:1000000000800020BD01000031A80000E9A7000029
:10001000E9A70000E9A70000E9A70000E9A70000A0
:10002000E9A70000E9A70000E9A7000031A8000047
:1000300031A80000E9A7000051C5000055C6000026
:1000400031A8000031A8000031A8000031A800004C
:1000500031A8000031A8000031A8000031A800003C
:1000600031A8000031A8000031A8000031A800002C
:1000700031A8000031A8000031A8000031A800001C
:1000800031A8000031A8000031A8000031A800000C
:1000900031A8000031A8000031A8000031A80000FC
:1000A0007DA3000089A3000031A8000031A8000052
:1000B00031A8000031A8000031A8000031A80000DC
:1000C00031A8000031A8000031A8000031A80000CC
:1000D00031A8000031A8000031A8000031A80000BC
:1000E00031A8000031A8000031A8000031A80000AC
:1000F00031A8000045AE000031A80000C9CB0000C7
:1001000031A80000F5CC000031A8000031A80000A3
:1001100031A8000031A8000031A8000031A800007B
:1001200031A8000031A8000031A8000031A800006B
:1001300031A8000031A8000031A8000031A800005B
:1001400031A8000031A8000031A8000031A800004B
:1001500031A8000031A8000031A8000031A800003B
:1001600031A8000005B1000031A8000031A800004E
:1001700031A8000031A8000031A8000031A800001B
:1001800031A8000031A8000031A8000031A800000B
:1001900031A80000E170000031A8000031A8000083
:1001A00031A8000031A8000031A8000031A80000EB
:1001B00031A8000031A800000DC30000564B4CF2DE
:1001C000205210B51A804DF628121A8000BF00BFC9
:1001D0000AF032FB514B4FF010621A60504A9A609D
:1001E000504ADA60504A136813F4807304D14F49BF
:1001F0000B604FF4A85313604D4B1A78110703D5C9
:100200001A7842F008021A704A4B4B492A221A7097
:100210004A4A4B4B8B4204D252F8040F43F8040B6A
:10022000F8E7484B484900228B4202D243F8042B9E
:10023000FAE74649464A002352F8230041F82300D2
:1002400001336F2BF8D1434B434A802103F8011B44
:100250009342FBD1414B3D4A1A60414B8A221A70AE
:10026000A3F5805324225A70A0221A709A7992071B
:10027000FCD59A79D406FCD43A4A937903F00C035E
:10028000082B384BF9D103221A7140225A719A79FE
:100290009006FCD5334A9179324B4906FBD5324A58
:1002A000324911600221516020221A709A7902F0BD
:1002B0000C020C2AFAD12E4B2E4A1A602E4B2F4AD2
:1002C0001A6000225A60072243F8042C2C4AC3F813
:1002D0000C2D62B60AF08CFC144B1B68DA0705D5AE
:1002E00028480AF0E9FB284B284A1A60284B1B785B
:1002F0005B0609D5244C254B22689A4204D121483B
:100300000AF0DAFB002323600DF064FD0AF09AFA8C
:100310000CF0B8FBFEE700BF0E2005403080044023
:10032000823F04000100002B10D0034014D0034092
:1003300002D0074000E0074030B2FF1FB8090100BB
:100340002097FF1F30B2FF1F94E1FF1F0092FF1F95
:100350000000000000E400E05FE400E008ED00E0E1
:100360000050064000400640448004400000030165
:1003700004800440C010050014E000E0FF76010096
:1003800000002020AC65345D1CE00340A5C3945AF6
:1003900000F00740FFFFFFFFFFFFFFFFFFFFFFFF32
:1003A000FFFFFFFFFFFFFFFFFFFFFFFFFFFFFFFF5D
:1003B000FFFFFFFFFFFFFFFFFFFFFFFFFFFFFFFF4D
:1003C000FFFFFFFFFFFFFFFFFFFFFFFFFFFFFFFF3D
:1003D000FFFFFFFFFFFFFFFFFFFFFFFFFFFFFFFF2D
:1003E000FFFFFFFFFFFFFFFFFFFFFFFFFFFFFFFF1D
:1003F000FFFFFFFFFFFFFFFFFFFFFFFFFFFFFFFF0D
:10040000FFFFFFFFFFFFFFFFFFFFFFFFDEF9FFFF23
:1004100010B5054C237833B9044B13B10448AFF33E
:1004200000800123237010BD30B2FF1F00000000C8
:10043000BC090100084B10B51BB108490848AFF3CF
:1004400000800848036803B910BD074B002BFBD0A0
:10045000BDE81040184700BF0000000034B2FF1F85
:10046000BC09010030B2FF1F0000000038B5074C86
:10047000074DC4F8C05204F5367009F0B7F82046AD
:1004800040F8185BBDE8384009F0B0B808C4FF1F59
:100490004805010070B5074C074EA4F5306544F8D7
:1004A000186C2046A4F5307409F0A0F8AC42F6D1DF
:1004B00070BD00BFF4BDFF1F4805010070B5324B91
:1004C0001B7882B0ABB9314D2C78012C31D01AD3C6
:1004D000022C0CD12E4B18780AF006FB01282FD0E5
:1004E0002C4A2D48642106F05FFF2C4B186002B0A7
:1004F00070BD2A4A2A4B1168274800221A7006F05C
:1005000057FF02B070BD224B18780AF0EDFA0028B0
:10051000EDD1244A244B12680092009919601D4ABB
:100520001D48142106F040FF1C4A012310602B7067
:10053000DDE7174E30780AF0D7FA08B9737823B19F
:10054000174B00221A7002B070BD164B164A1B687A
:1005500001931168019B40F2DB525B1A934207D86A
:100560000C4A0D48142106F01FFF0C4B1860BEE723
:100570000B4B084A1C700848022364212B7006F0BC
:1005800013FF064B1860B2E702C3FF1F88C9FF1FA5
:1005900050B2FF1FBD0400000CB3FF1F30C2FF1F8D
:1005A00048CAFF1F60DEFF1F90CEFF1F10B5044634
:1005B0000BF056FE204610BD10B51F4C2378EBB152
:1005C000012B1AD11D4A1E4B11681B681D48194486
:1005D00000781D4B11601B6820B3994203DB022099
:1005E000136019462070194806F068FD2378124AF6
:1005F000012B1AD00023137010BD10BD144A104BEC
:1006000011681B680D4A11480B441946136006F027
:1006100055FD012323700F4A0F481421BDE81040F7
:1006200006F0C2BE9942DEDCD9E70A4A0A48142124
:10063000BDE8104006F0B8BE8ACDFF1F08B3FF1F0B
:10064000F8B4FF1FACCEFF1FD8A4FF1F64CAFF1F62
:10065000009AFF1FB90500000CB3FF1F0A4B1B686F
:1006600083B110B5094C2168002904DD0848BDE8B4
:10067000104006F0C3BE1946064A054806F094FE2F
:10068000206010BD704700BF8CCDFF1FA4CEFF1FA0
:100690000CB3FF1F712C000008B5064A064840F64F
:1006A000B83106F081FE054A054B106001221A7030
:1006B00008BD00BF353700000CB3FF1FA8C0FF1FE7
:1006C0004CB2FF1F58B138B5054600240134012152
:1006D0000348E4B20BF096FBA542F7D138BD704752
:1006E00058FC0000032101480BF08CBB48F70000C8
:1006F00038B50F4C054607210E480BF083FB691CEB
:1007000020460CF025F80A210B480BF07BFB0B4B25
:1007100003EB0513204699890CF01AF803210848C9
:100720000BF070FB2046BDE838400BF0C1BF00BFA6
:10073000D0A7FF1F4CF7000054F7000000B5FF1FC3
:1007400060F70000F8B50E2106464FF430751948E1
:10075000194F05FB06F50BF055FB05F2932405F543
:1007600028753C443D4414F8010F0BF0CFFBAC421C
:10077000F9D10C2111480BF045FB0A220023314628
:100780000F480BF0A5FF06210E480BF03BFB4FF482
:10079000307303FB06760A48B6F8BA120BF0D8FF9E
:1007A000012109480BF02EFB0548BDE8F8400BF08D
:1007B0007FBF00BF64F700009CB5FF1F74F7000007
:1007C000D0A7FF1F84F700008CF700002DE9F04F41
:1007D00087B0DFF8C0819DF84040009498F8004051
:1007E000002C00F0C6800192002202930391824601
:1007F000DFF89C911746144605E0013498F8003064
:10080000E4B2A34248D94FF4307505FB04F509EB77
:100810000506002FF1D196F8AC32002BEDD1304611
:1008200007F0F4F8D446BCE80F0006F5257EAEE8E4
:100830000F009DF804309CE8030086F8AD329DF867
:10084000083086F8AE324FF0010B9DF8003086F884
:10085000BE328EE8030086F8AF7206F52571304689
:1008600086F8ACB207F006F9474B86F8BC421A6826
:100870000492464AB6F8BA3212780499C6F8B01211
:100880005B44A6F8BA32AAB9224698F8003001347F
:10089000E4B2A3425F46B6D897B13D4B4FF43071F6
:1008A00001FB02320120D2F8BA32039A136007B07A
:1008B000BDE8F08F2046FFF745FF5F4622469CE7E4
:1008C000002B56D0DFF8C8903C4605E0013498F87C
:1008D0000030E4B2A3424AD94FF4307505FB04F569
:1008E00009EB0506002FF1D196F8A8129AF81430FA
:1008F0009942EBD2304607F089F8D446BCE80F00A5
:1009000006F5257EAEE80F009DF804309CE8030054
:1009100086F8AD329DF8083086F8AE324FF0010B04
:100920009DF8003086F8BE328EE8030086F8AF727C
:1009300006F52571304686F8ACB207F09BF8124BED
:10094000B6F8BA221968114B05911978059886F8FE
:10095000BC425A44C6F8B002A6F8BA2269B9224687
:1009600098F800300134E4B2A3425F46B4D8002FB7
:1009700093D1002007B0BDE8F08F2046FFF7E2FEDC
:100980005F462246A2E700BF60DEFF1FE299FF1F1D
:100990009CB5FF1F20A0FF1F00B585B0002300936A
:1009A0001A4603A9FFF712FF05B05DF804FB00BF6C
:1009B00000B585B0002300911A4603A9FFF706FF92
:1009C00005B05DF804FB00BF044890F8BD3103B9E1
:1009D000704700F5D8700921FFF7EABF909CFF1F10
:1009E00000B583B0002300921A46FFF7EFFE03B074
:1009F0005DF804FB2DE9F04FDFF84C814D4E98F87F
:100A000000E04D4F4FF43075044683B005FB0E6097
:100A10008B469A46914687F800E006F0F7FF0FCC28
:100A200097F800E005FB0E6C0CF525750FC594E8F2
:100A30000300012285E803008CF8ADB28CF8BEA259
:100A40008CF8AC22AEF1020E3C4DB9F1000F35D05E
:100A50000EEB8E003A4905EBC00006F061FD3878D8
:100A6000DFF8ECA04FF4307404FB00F0311801F50E
:100A70002571304406F0FEFF3878DAF80030019333
:100A800004FB00632F49B3F8BA220978019C83F86C
:100A9000BC020132C3F8B042A3F8BA22B1B998F847
:100AA0000020294B022A0CBF032202221A70B9F13E
:100AB000000F0ED1012003B0BDE8F08F0EEB8E00C9
:100AC000224905EBC00006F02BFDC8E7FFF73AFE10
:100AD000E5E798F80000174FDFF86C804FF43074AA
:100AE00004FB006007F058FA0028E3D098F80000F3
:100AF0001349023800EB800005EBC000002206F02D
:100B00000FFDDAF80030009398F80030009A04FBEB
:100B100003730120002102F5C87283F8B802012096
:100B2000C3F8B42283F8AD1283F8BE1203B0BDE857
:100B3000F08F00BF9CB5FF1FE099FF1F84C1FF1F0E
:100B400016B70300E299FF1F7C9AFF1F5D74D10561
:100B500060DEFF1F01220B461146FFF74BBF00BFAF
:100B6000F8B50E2106464FF430751948194F05FBAC
:100B700006F50BF047F905F2932405F528753C447A
:100B80003D4414F8010F0BF0C1F9AC42F9D10C212E
:100B900011480BF037F90A22002331460F480BF0B9
:100BA00097FD06210E480BF02DF94FF4307303FB2F
:100BB00006760A48B6F8BA120BF0CAFD01210948B8
:100BC0000BF020F90548BDE8F8400BF071BD00BFFF
:100BD00090F700009CB5FF1F74F70000D0A7FF1F1F
:100BE00084F700008CF70000F8B50E2106464FF49C
:100BF00030751948194F05FB06F50BF003F905F29E
:100C0000932405F528753C443D4414F8010F0BF07E
:100C10007DF9AC42F9D1102111480BF0F3F80A220A
:100C2000002331460F480BF053FD06210E480BF010
:100C3000E9F84FF4307303FB06760A48B6F8BA12A7
:100C40000BF086FD012109480BF0DCF80548BDE8F2
:100C5000F8400BF02DBD00BF64F7000008C4FF1F73
:100C6000A0F70000D0A7FF1F84F700008CF700005A
:100C70002DE9F04FDFF84C814D4E98F800E04D4FD4
:100C80004FF43075044683B005FB0E608B469A46E0
:100C9000914687F800E006F0B9FE0FCC97F800E027
:100CA00005FB0E6C0CF525750FC594E803000122B9
:100CB00085E803008CF8ADB28CF8BEA28CF8AC22AB
:100CC0003D4DB9F1000F68D00EEB8E003B4905EBAE
:100CD000C00006F025FC3878DFF8F0A04FF430743F
:100CE00004FB00F0311801F52571304406F0C2FE16
:100CF0003878DAF80030019304FB00633049B3F828
:100D0000BA220978019C83F8BC020132C3F8B042D0
:100D1000A3F8BA22002948D198F80020294B42B9FB
:100D200001221A70B9F1000F08D1012003B0BDE80B
:100D3000F08F00221A70B9F1000FF6D098F8000079
:100D40001B4FDFF880804FF4307404FB006007F025
:100D500023F90028E9D098F80000184900EB80003A
:100D600005EBC000002206F0DBFBDAF80030009350
:100D700098F80030009A04FB03730120002102F56B
:100D8000C87283F8B8020120C3F8B42283F8AD1208
:100D900083F8BE1203B0BDE8F08F0EEB8E000A4957
:100DA00005EBC00006F0BCFB95E7FFF71DFFB3E7BE
:100DB00008C4FF1F4CC2FF1F74B4FF1F16B7030007
:100DC000E299FF1F08CEFF1F5D74D10560DEFF1F93
:100DD0000B4601220021FFF74BBF00BF01220B464B
:100DE0001146FFF745BF00BF00220B461146FFF733
:100DF0003FBF00BF002310B4104C41720261046079
:100E00000372C36041B1194600E0026942F8231041
:100E1000427A01339A42F8DC094B1A680AB90BE0AE
:100E20001A465369002BFBD1506100234361838034
:100E3000C380837210BC70471860F6E738F7000073
:100E4000F8DFFF1F13490A6838B50023124D05600B
:100E50000446437203610372C3600AB918E01A467C
:100E60005369002BFBD15461204600250B4B656173
:100E7000A580E580A57240F8183B08F0A5FB204648
:100E8000C4F88050C4F8845006F0A6FD204638BD52
:100E90000860E9E7F8DFFF1F38F7000048050100A8
:100EA00008B5124B5B7B4BB9114B5B7B33B9114BD4
:100EB000114A1B780021117063B908BD0F4B5B7B91
:100EC000002BF4D00E4B5B7B002BF0D00A4B0122A1
:100ED0001A7008BD0B480BF0EBFB26210A480AF0FC
:100EE00091FF0848BDE808400BF0E2BB90A4FF1F4B
:100EF000E499FF1FE299FF1F81CEFF1F9C9BFF1FFC
:100F0000809AFF1FD0A7FF1FB4F7000008B5114B50
:100F10005B7B33B1104B114A1B7801211170ABB9C7
:100F200008BD0D4A0D4912780B70002AF8D00C4804
:100F30000BF0BEFB0B482E210AF064FF08480BF0B3
:100F4000B7FB0748BDE808400BF0B2BB1C210648C0
:100F5000F2E700BFDCA4FF1FE299FF1F01C3FF1FE0
:100F6000D0A7FF1FFCF70000DCF70000092810B530
:100F7000044602D830200AF0C9FF214600230A2285
:100F80000248BDE810400BF0A3BB00BFD0A7FF1F75
:100F9000244A254B70B5A2FB0012A3FB0013234C7F
:100FA0009B09920BA4FB0215A4FB03146D094FF4DB
:100FB0007A71640901FB1300C5EB0515C4EB041439
:100FC000A2EB8505A3EB84040CF08AFC18490CF015
:100FD0008FFD002106460CF089FED0B130464FF05F
:100FE0007C510CF0C9FB0CF095FE0646E8B2FFF709
:100FF000BDFF01210F480AF005FFE0B2FFF7B6FF81
:1010000001210C480AF0FEFEF0B2BDE87040FFF787
:10101000ADBF30464FF07C510CF0ACFB0CF07AFECB
:101020000646E3E773B2E745D34D621089888888A6
:10103000000020412CF8000070B50646441E00F167
:101040000C0514F8010F0AF061FFA542F9D1062042
:10105000FFF738FB737B43B901210C480AF0D2FE3D
:101060000B48BDE870400BF023BB3069FFF790FFE1
:101070000620FFF727FB317D054800230A220BF0ED
:1010800027FB0348BDE870400BF012BB30F80000AE
:10109000D0A7FF1F10B53224012107480AF0B2FE85
:1010A000631E13F0FF04F7D104480BF001FBBDE809
:1010B00010400AF05BBF00BF30F80000D0A7FF1F50
:1010C00010B5154C84B020460BF0F2FAFFF7E2FFA2
:1010D000122112480AF096FE114B0A221978204676
:1010E00000230BF0F5FA20460BF0E2FA12210D482E
:1010F0000AF088FE68460C490BF096FC69462046CB
:101100000BF0B0FA20460BF0D3FAFFF7C3FF6846A6
:101110000BF04AFC04B010BDD0A7FF1F34F800004C
:101120008F9BFF1F48F800005CF8000038B512489C
:10113000124C0BF0BDFAFFF7ADFF0F2110480AF07B
:1011400061FE0D480BF0B4FAFFF7A4FF28210D480B
:101150000AF058FE08480BF0ABFAFFF79BFF04F5C6
:101160000B7554F8040FFFF767FFAC42F9D1024842
:10117000BDE838400BF09CBAD0A7FF1F68CAFF1F1C
:1011800064F8000074F8000010B53224012107480B
:101190000AF038FE631E13F0FF04F7D104480BF089
:1011A00087FABDE810400AF0E1BE00BF4CF900002C
:1011B000D0A7FF1F08B540B9022107480AF022FE58
:1011C0000648BDE808400BF073BAFFF78BFA0348F6
:1011D000BDE808400BF06CBAB8F80000D0A7FF1FBC
:1011E00038B5234C2348244D07210AF00BFE204636
:1011F0000BF05EFA0F2121480AF004FE286820490E
:101200000CF0C2FB0CF0ACFD00230A22C1B2204658
:101210000BF05EFA20460BF04BFA102119480AF049
:10122000F1FD686816490CF0AFFB0CF099FD002346
:101230000A22C1B220460BF04BFA20460BF038FAD6
:10124000162111480AF0DEFDA8680D490CF09CFB40
:101250000CF086FD0023C1B20A2220460BF038FABA
:1012600020460BF025FA2046BDE838400BF020BAA6
:10127000D0A7FF1FCCF80000C4A4FF1FD4F80000C3
:101280000000C842E4F80000F8F8000038B50F216B
:101290002448254C0AF0B6FD24480BF009FA012534
:1012A00009E0FFF71FFA013520480BF001FA072D7E
:1012B00004F1100423D007211D480AF0A3FD29469C
:1012C0001A480BF045FA05211A480AF09BFD2188BF
:1012D00016480BF03DFA052117480AF093FD618886
:1012E00012480BF035FA092114480AF08BFD2379D6
:1012F00013480221002BD4D10AF084FDD3E7112139
:1013000010480AF07FFD104B084819780A22002384
:101310000BF0DEF905480BF0CBF90448BDE8384086
:101320000BF0C6B910F9000000B5FF1FD0A7FF1FD2
:101330004CF7000020F9000028F9000030F9000007
:10134000B8F800003CF90000159CFF1F38B5174C99
:101350000125062116480AF055FD294615480BF0CF
:10136000F7F90D2114480AF04DFD218811480BF0C2
:10137000EFF9102111480AF045FD61880D480BF086
:10138000E7F911210E480AF03DFDA18809480BF04C
:10139000DFF9013507480BF08BF9042D04F1060441
:1013A000D7D10448BDE838400BF082B950C2FF1FC6
:1013B00050F90000D0A7FF1F58F9000068F900009D
:1013C0007CF9000008B50E212D480AF01BFD2D4BBD
:1013D00003F5F0715A7B1833002A37D18B42F9D1CB
:1013E0000E2129480AF00EFD28480BF061F90E2164
:1013F00027480AF007FD274B03F5F0715A7B183395
:101400006AB98B42FAD10E211F480AF0FBFC1F4833
:101410000BF04EF91D48BDE808400BF049B9142106
:101420001D480AF0EFFC1D4B1B782BBB02211C480A
:101430000AF0E8FC01211B480AF0E4FC13480BF019
:1014400037F91248BDE808400BF032B914211248B0
:101450000AF0D8FC144B1B785BB9022110480AF043
:10146000D1FC01210F480AF0CDFC08480BF020F90F
:10147000BDE7FFF737F9F4E7FFF734F9DAE700BF24
:1014800090F90000D0A0FF1F1CF80000D0A7FF1F9C
:10149000A0F90000B0A2FF1FB0F90000A0C3FF1F19
:1014A000B8F800008CF70000C4B4FF1F10B5182175
:1014B00082B030480AF0A6FC2F480BF0F9F8212141
:1014C0002E480AF09FFC2E4B1878FFF773FE25215B
:1014D0002C480AF097FC2C4B186800283AD00CF0E6
:1014E000FBF92A490CF004FB0BF01CFE0124024618
:1014F0000B46009420480BF033F9082124480AF0E9
:1015000081FC1D480BF0D4F8182122480AF07AFC1F
:10151000214B1B7833BB092120480AF073FC164885
:101520000BF0C6F80F211E480AF06CFC1D4B124848
:1015300019780A2200230BF0CBF801211A480AF08F
:1015400061FC0D480BF0B4F80B4802B0BDE8104048
:101550000BF0AEB8032115480AF054FC06480BF016
:10156000A7F8D1E70C2112480AF04CFC02480BF016
:101570009FF8D7E7C8F90000D0A7FF1FE4F90000E3
:101580002CC2FF1F08FA00008CCDFF1F00606A47C5
:1015900030FA000040FA00008B9BFF1F6CFA00003D
:1015A00078FA00008D9BFF1FC8F800003CFA00008D
:1015B0005CFA000038B5324C3248334D0E210AF047
:1015C00021FC20460BF074F8102130480AF01AFC78
:1015D0002F4B1878FFF7EEFD10212E480AF012FC71
:1015E0002D4B204619880BF0B3F8032128460AF04A
:1015F00009FC20460BF05CF8102128480AF002FC98
:10160000274B204619880BF0A3F8032128460AF03F
:10161000F9FB20460BF04CF80C2122480AF0F2FBB3
:10162000214B0A221978204600230BF051F80C2197
:101630001E480AF0E7FB1E4B204619680BF088F89D
:1016400006211C480AF0DEFB1B4B0A2219782046B3
:1016500000230BF03DF80B2118480AF0D3FB184B80
:10166000204619680BF074F8042116480AF0CAFBEA
:1016700020460BF01DF82046BDE838400BF018B8A6
:10168000D0A7FF1F88FA000060F7000098FA00005A
:10169000ACCEFF1FACFA000062CEFF1FC0FA000004
:1016A0009ECEFF1FD4FA00008A9BFF1FE4FA0000C1
:1016B000009AFF1FF4FA00008C9BFF1FFCFA000049
:1016C000D8A4FF1F08FB0000013838B50D461446AA
:1016D000072817D8DFE800F03C42484E045E701738
:1016E0000C2167480AF08EFB294600230A22654830
:1016F0000AF0EEFF022C75D0032C00F09180012C33
:1017000000F0948038BD0B215F480AF07BFB012D6F
:1017100007BF29465D485E480121013C0AF072FB83
:10172000082CEFD801A353F824F000BF15180000CF
:101730000517000005170000051700000517000039
:101740000517000009180000FD170000F117000040
:101750000C215048BDE838400AF054BB0B214E48DC
:10176000BDE838400AF04EBB0D214C48BDE838407A
:101770000AF048BB07214A480AF044FB29460023E7
:101780000A2240480AF0A4FF05214648BDE8384037
:101790000AF038BB062144480AF034FB013C2946D4
:1017A00000230A2237480AF093FF052CAAD8DFE865
:1017B00004F04943375B554F0B213C480AF022FBAC
:1017C000294600230A222F480AF082FF022C09D062
:1017D000032C4FD0012C95D105213548BDE8384068
:1017E0000AF010BB05213348BDE838400AF00ABBB7
:1017F0000C213148BDE838400AF004BB0E212F48C7
:10180000BDE838400AF0FEBA0A212D48BDE838404C
:101810000AF0F8BA0A212B48BDE838400AF0F2BABB
:1018200007212948BDE838400AF0ECBA06212748CC
:10183000BDE838400AF0E6BA04212548BDE8384042
:101840000AF0E0BA03212348BDE838400AF0DABACA
:1018500006212148BDE838400AF0D4BA10211F48BB
:10186000BDE838400AF0CEBA0F211D48BDE8384027
:101870000AF0C8BA07211B48BDE838400AF0C2BACE
:101880004CFB0000D0A7FF1FC8FB0000D4FB0000EA
:10189000D8FB000010FB000020FB00002CFB000028
:1018A0003CFB000044FB000050F90000ACFB0000D2
:1018B000B8FB000064FB000004FC0000F4FB000027
:1018C000E8FB0000DCFB00006CFB00005CFB0000A0
:1018D00078FB000074FB0000A4FB000090FB0000FC
:1018E00080FB0000C0FB0000F8B50D214848494CC2
:1018F0000AF088FA48480AF0DBFE0125082147482B
:101900000AF080FA294644480AF022FF022144489E
:101910000AF078FA637D002B54D0082141480AF080
:1019200071FA617A3C4800230A220AF0D1FE0B21A9
:101930003D480AF067FAE379002B54D10135364867
:101940000AF0B6FE062D04F11804D7D13248374FFD
:101950000AF0AEFE102136480AF054FA2E480AF07A
:10196000A7FE3B784BB3334E002408212B480AF0E6
:1019700049FA04EB8403F518F15C274800230A2296
:101980000AF0A6FE05212C480AF03CFA00230A22A0
:10199000697821480AF09CFE032128480AF032FAAF
:1019A0002A79E978A878FFF78FFE1B480AF080FEB5
:1019B00001343B78E4B2A342D7D81748BDE8F840D9
:1019C0000AF076BE11211E480AF01CFAA37D012BF5
:1019D00018D012D3022B0BD10D211A480AF012FA9B
:1019E000E379002BAAD0132117480AF00BFAA5E7D8
:1019F000072116480AF006FA9DE7042114480AF068
:101A000001FA98E70C2113480AF0FCF993E700BFAC
:101A100014FC000050B2FF1FD0A7FF1F24FC0000E1
:101A20009CF9000030FC00003CFC000098B5FF1F52
:101A3000A0FC0000F4CCFF1FB4FC0000A0F80000E4
:101A400048FC000074FC00008CFC000084FC0000DA
:101A50005CFC000064FC000070B50546A8B1441EA3
:101A6000E4B2013905290FD8DFE801F0033C597DC4
:101A7000118F784B2C2000FB043005F029F9764BB0
:101A80001B78002B40F0AF8070BD0446E9E7714E33
:101A90002C2303FB0466304605F05CF9002800F0B7
:101AA0009780304605F07AF96B4B1B78002BEBD012
:101AB000304605F04FF90446002800F0A7800621C3
:101AC00066480AF09FF9294600230A2264480AF072
:101AD000FFFD0F2163480AF095F96148BDE87040A9
:101AE0000AF0E6BD5B4B2C2000FB043005F00AF940
:101AF000594B1B78002BC7D0062158480AF082F9B1
:101B0000294600230A2256480AF0E2FD04215648DD
:101B10000AF078F95248BDE870400AF0C9BD4D4A54
:101B20002C2303FB0424204605F006F94A4B1B78BE
:101B3000002BA9D0204605F099F804460621474815
:101B4000002C76D00AF05EF9294600230A22444888
:101B50000AF0BEFD0A2145480AF054F94048BDE8A4
:101B600070400AF0A5BD424B3A4804EB440203EB37
:101B700042032C269A88598806FB040005F05CF97C
:101B8000354B1B78002B9AD170BD324B384A04EB91
:101B900044012C2000FB043032F8111005F0FAF853
:101BA0002D4B1B78002B3FF46FAF06212B480AF01A
:101BB00029F9294600230A2229480AF089FD06212D
:101BC0002C480AF01FF92648BDE870400AF070BDA5
:101BD000274B04EB440403EB44043046A28861889D
:101BE00005F02AF960E706211C480AF00BF929469E
:101BF00000230A221A480AF06BFD03211E480AF04E
:101C000001F91748BDE870400AF052BD062113489B
:101C10000AF0F8F8234629460A2211480AF058FD2E
:101C20000E2116480AF0EEF80D48BDE870400AF0A3
:101C30003FBD0AF0E7F8234629460A2208480AF081
:101C400047FD0B210E480AF0DDF80548BDE870405D
:101C50000AF02EBD8CC9FF1FE299FF1F50F900004A
:101C6000D0A7FF1FE0FC0000C0FC0000C8FC000083
:101C700050C2FF1F00FD0000BCFC0000F0FC000093
:101C8000D4FC00002DE9F041104C4FF0020804F1A3
:101C90007807002540F2DC562078022108F032FF58
:101CA0000322012365706680A680A5712572E57107
:101CB00084F80A80E56025612575A57562726375F3
:101CC0001834BC42E8D1BDE8F08100BF50B2FF1F1C
:101CD00010B50F4C0F492078042208F02DFE207E0D
:101CE0000D49042208F028FE94F830000B49042224
:101CF00008F022FE94F848000949042208F01CFE6E
:101D000094F8600007490422BDE8104008F014BEB2
:101D100050B2FF1FC11D0000C91D0000D11D0000F1
:101D2000D91D0000E11D000010B5124C20782228BA
:101D300028BFFF2008F07CFE207E222828BFFF203D
:101D400008F076FE94F83000222828BFFF2008F023
:101D50006FFE94F84800222828BFFF2008F068FE94
:101D600094F86000222828BFFF20BDE8104008F04A
:101D70005FBE00BF50B2FF1F70B5044608F0C8FE3A
:101D800004EB44030C4ADB00D518A97901B170BDFE
:101D90000646D05C08F0A8FE30B1EE60002CF6D10B
:101DA000064B01221A7070BDEB68EE60F61A012333
:101DB000AE80AB7170BD00BF50B2FF1F02C3FF1FEA
:101DC0000020FFF7D9BF00BF0120FFF7D5BF00BF3C
:101DD0000220FFF7D1BF00BF0320FFF7CDBF00BF38
:101DE0000420FFF7C9BF00BF10B5114C2378012BA9
:101DF00016D00BD3022B06D10E4804F083FF0D48FA
:101E000005F050F823780C4A137010BD094804F00F
:101E100079FF084805F02AF8074A2378137010BDA7
:101E2000044804F055FF044A2378137010BD00BF26
:101E30008BCDFF1FC0C2FF1F73C3FF1FF0B51D4A2C
:101E40001D4B126883B00192019A1A6008F060FE7F
:101E50001A4B4FF080421A6072B6194B194E00218E
:101E600003F178058E4602271A69821AB24201F1FF
:101E7000010406D95A78012AE1B204BF5F7083F8E1
:101E800014E01833AB42EFD162B60F4B4FF08042F3
:101E900005291A6009D00D4B1B780D4A12789A4219
:101EA00001D0FFF7A1FF03B0F0BD084A0223137071
:101EB000F3E700BF60DEFF1FD4C1FF1F88E100E031
:101EC00050B2FF1FA086010008E100E08BCDFF1F8C
:101ED00073C3FF1F2DE9F04F4FEA400CDFF854E1C8
:101EE0000CEB00030EEBC3035F885D7AC7F57A74D1
:101EF000002CB8BF6442012D40F38780DFF838B171
:101F0000DFF838A1DFF83891012242F20F73002682
:101F1000A91E04290AD8DFE801F02F372821030081
:101F20003BF91230DB1B002BB8BF5B42A342B8BFAA
:101F3000D6B202F10102B8BF1C46AA42E9D101366D
:101F4000F6B260440EEBC000C3792BB3023D042D02
:101F500022D8DFE805F034523A4624003AF912302C
:101F6000DB1B002BB8BF5B42E0E739F91230DB1B0B
:101F7000002BB8BF5B42D9E72C4B33F91230DB1B87
:101F8000002BB8BF5B42D1E7294B33F91230DB1B82
:101F9000002BB8BF5B42C9E73046BDE8F08F012E89
:101FA00041D0022E39D0032E31D0042E32D0052E4E
:101FB00036D0062E14BF30460120BDE8F08F012E2A
:101FC00014BF01200220BDE8F08F012E1FD0022E89
:101FD00020D0032E24D0042E14BF30460120BDE8AB
:101FE000F08F012E19D0022E11D0042E18D0052EFC
:101FF00014BF30460120BDE8F08F012E0AD0032E19
:1020000014BF30460120BDE8F08F012699E7042077
:10201000BDE8F08F0320BDE8F08F0520BDE8F08F0C
:102020000220BDE8F08F0620BDE8F08F3CF70000ED
:1020300040F7000050B2FF1F4C02010040020100B7
:1020400038020100013805281BD8DFE800F0070A34
:102050000E12160340F6055008F03ABE094808F083
:1020600037BE44F6206008F033BE42F2107008F02C
:102070002FBE41F2883008F02BBE40F2836008F09A
:1020800027BE70478038010008B5064B064819681E
:1020900005F014F8054B064A19880648BDE80840C3
:1020A00005F082B9009AFF1F64CAFF1F62CEFF1FAE
:1020B000B90500000CB3FF1F38B51E4B1B78DBB110
:1020C0001D4A1E4B10681B681D4CC01A0BF008FC03
:1020D0001C4B054618880BF0FFFB1B490BF008FD55
:1020E000014628460BF004FD4FF07C510BF044FBF9
:1020F0000BF010FE206038BD104A0F4B10681B68B3
:102100000F4CC01A0BF0ECFB0E4B054618880BF079
:10211000E3FB0D490BF0ECFC014628460BF0E8FC14
:102120004FF07C510BF028FB0BF0F4FD4042206097
:1021300038BD00BFACCEFF1FD8A4FF1F009AFF1F01
:10214000F8B4FF1F9ECEFF1F0000A04170B51F4BCB
:1021500018780BF0C1FB1E490BF00CFB1D490BF06E
:1021600013FC1D4B054618780BF0B6FB18490BF015
:1021700001FB18490BF008FC184B1B780446284655
:10218000BBB91749174E184D0BF0F6FA4FF07C51BA
:102190000BF0F2FA0BF0BEFD1449306020460BF054
:1021A000EBFA4FF07C510BF0E7FA0BF0B3FD28602F
:1021B00070BD0E490B4E0C4D0BF0DEFA4FF07C510A
:1021C0000BF0DAFA0BF0A6FD0549E6E78A9BFF1F44
:1021D0000000C8420000A0408C9BFF1FACCEFF1F38
:1021E0000000FA44009AFF1FD8A4FF1F00007A44A1
:1021F000F8B55B4D00222B4605F1960E012702260D
:102200001A705A709A70DF701E71053373454FF063
:1022100000014FF001004FF00204F1D1514E524A3B
:10222000B075032386F87640AB71AB72EB732B75F8
:102230006B75EB7705270723717586F875100426F3
:102240002C706870A8706C71EC71E87268732C74F3
:10225000AC74EC74EC752876A876287768772E73C2
:102260006E76AE776F74AF75EB7685F8203040F2FE
:10227000DC5685F82140DFF830E185F822004FF484
:102280007A7441F270704FF47A6741F288354FF4F6
:10229000FA5C168014864FF4FA6640F6B8348EF86D
:1022A0000030A2F852001346A2F822C002F16000EA
:1022B0005780A2F84270168256865582A2F8505076
:1022C0001484A2F8404019715971996099811033B2
:1022D00098424FF00004F6D1244D2549254A2C7030
:1022E00019250D70244F254B2548DFF8C0E00470F8
:1022F0004FF07C5111605160916005223A70214984
:102300002148224FDFF8A8C0214E8CF800401E2241
:102310005A809A801A801A815A81DA80DA811A8268
:102320009A81C8230B804FF448731A491A4AAEF8B1
:1023300000306423037001254FF4FA603B704FF4C2
:102340007A73136008603570FFF700FFFFF7B4FE83
:102350001249134B134A34700D701A60F8BD00BF58
:10236000F4CCFF1F50B2FF1F00B5FF1FC4B4FF1F06
:10237000159CFF1FC4A4FF1F8D9BFF1F50C2FF1F92
:10238000A0C3FF1F62CEFF1F8A9BFF1F8C9BFF1FF6
:102390008B9BFF1F009AFF1FD8A4FF1F2CC2FF1F9B
:1023A0008CCDFF1FC0D4010098B5FF1F9ECEFF1F2C
:1023B000ACCEFF1F2DE9F04F87B0544D019550244E
:1023C000534B544A54490094544804F0A5FB05F17A
:1023D00018030193524A4E4B4F4900944F4804F062
:1023E0009BFB05F1300301934E4A494B4A49009447
:1023F0004A4804F091FB05F1480301934A4A444BD3
:1024000045490094454804F087FB05F160030193BA
:10241000163D3F4B40490094444A404804F07CFB41
:102420002F4605F178012B4600209A7D02B15875A0
:1024300018339942F9D13E4C354B3E4A3E490194FE
:1024400050260096354804F023FB04F1180301934D
:102450003A4A2F4B38490096304804F019FB04F1F2
:1024600030030193364A2A4B334900962B4804F037
:102470000FFB04F148030193324A254B2E49009685
:10248000264804F005FB04F1600301930096204BFD
:102490002D4A2949214804F0FBFA7B7D002B40F0AE
:1024A000DD8297F82D30002B40F0E68297F845301A
:1024B000002B40F0F08297F85D30002B40F0FA825C
:1024C00097F87530002B40F00483DFF884900022E9
:1024D0004B4609F19606012402201A705A709A7030
:1024E000DC7018710533B3424FF00001F5D1174B82
:1024F0000B2619704FF0010805AF6B7D002B78D0CB
:102500006B7A002B75D0012425E000BF66B2FF1F57
:10251000B8C3FF1F08FD000014FD0000B4CDFF1F6D
:1025200024FD000030FD00003CFD000048FD0000DF
:1025300057B2FF1F54FD000060FD000074FD000055
:1025400080FD00008CFD000098FD000098B5FF1F85
:10255000F4CCFF1F1446601E56FA80F000230A22B6
:1025600004A980B205930BF07FFC502302468DE84E
:102570008800AC49AC4BAD4804F000FB631CDAB2F8
:10258000DFF82CC390B39CF80000DFF828B31E28B6
:1025900000EB800E2AD80599A54B0391A3FB013AC5
:1025A0004FEA5A3A1FFA8AF30BFB0313A14909F8C1
:1025B0000E80A1FB03135FFA8AFA0399C3F3471352
:1025C000CAEB0A1B01EB0B1103EB830BCE44C3EBED
:1025D000CB0B013001EB8B018CF800008EF8014031
:1025E0008EF804308EF802A08EF803106B7AA342A6
:1025F000B0D80A36B6B208F101083D2E5FFA88F865
:1026000005F118057FF479AF50248B4D01950094A6
:10261000854B8A4A8A49854804F0A2FAAB1C00948B
:102620000193884A804B8649804804F099FA2B1D13
:1026300000940193844A7C4B81497C4804F028FA39
:1026400005F1100300940193804A774B7C49774849
:1026500004F086FA05F11203009401937C4A724B50
:102660007749724804F07CFA05F114030094019351
:10267000784A6D4B72496D4804F00AFA05F120035F
:1026800000940193744A684B6D49684804F068FAF5
:1026900005F1220300940193704A634B6849634833
:1026A00004F05EFA05F12403009401936C4A5E4B3A
:1026B00063495E4804F0ECF905F13003009401939E
:1026C000684A594B5E49594804F04AFA05F1320309
:1026D00000940193644A544B5949544804F040FA19
:1026E00005F1340300940193604A4F4B54494F481D
:1026F00004F0CEF905F14003009401935C4A4A4B83
:102700004F494A4804F02CFA05F142030094019322
:10271000584A454B4A49454804F022FA05F144031A
:1027200000940193544A404B4549404804F0B0F9A5
:102730002B1900940193514A3B4B41493B4804F00B
:102740000FFA05F15203009401934D4A364B3C4970
:102750003648543504F004FA8DE83000324B494ACB
:102760003749324804F094F9474B00940193474AA3
:102770002D4B33492D4804F0CFF98DE890002A4BBA
:10278000434A44492948FF248DF8144004F0C4F911
:102790009DF81400A04209D06428A8BF64200BF063
:1027A0009BF83D493D4C0BF0A3F9206050238DE888
:1027B0008800FF241C4B3A4A36491C488DF81440C7
:1027C00004F0AAF99DF81400A04209D06428A8BF1B
:1027D00064200BF081F83049304C0BF089F96060CF
:1027E00050238DE88800FF240F4B2E4A29490F48BB
:1027F0008DF8144004F090F99DF81400A04209D01F
:102800006428A8BF64200BF067F82349234C0BF021
:102810006FF9A0605024244D01950094FF26024BCF
:10282000224A49E0E0FD0000B8C3FF1FB4CDFF1FFE
:102830005917B7D11F85EB5100B5FF1FF8FD0000F8
:1028400000FE000010FE000018FE000020FE000048
:1028500028FE000030FE000038FE000040FE0000B0
:1028600048FE000050FE000058FE000060FE000020
:1028700068FE000070FE000078FE000080FE000090
:1028800088FE000090FE0000159CFF1F98FE0000CF
:10289000A4FE0000ACFE00000000C842C4A4FF1F5C
:1028A000B4FE0000BCFE000050C2FF1FC4FE0000CA
:1028B00098B5FF1FF0D8FFFF8B498C488DF8146046
:1028C00004F04EF9AB1C01930094894B894A864968
:1028D0008648894E894F04F043F92B1D01930094DB
:1028E000834B874A8049814804F03AF9AB1D019334
:1028F00000947F4B834A7C497C4804F031F905F110
:102900000803019300947A4B7F4A7749774804F093
:1029100027F905F10A0301930094754B7B4A72492C
:10292000724804F01DF905F10C0301930094704BFB
:10293000774A6D496D4804F013F905F10E030193D0
:1029400000946B4B734A68496848103504F008F9E5
:102950008DE83000664B704A6349644804F000F922
:102960006E4B01930094624B6D4A6E495F4804F0D0
:102970008FF86D4B019300945D4B6C4A69495B483D
:1029800004F086F86A4B01930094594B694A6A49EE
:10299000564804F07DF8694B01930094544B684A03
:1029A0006549524804F0DCF8664B01930094504BA3
:1029B000654A61494D4804F0D3F8644B0193009493
:1029C0004B4B634A5C49494804F0A6F8614B624AA4
:1029D000594901930094464B444804F09DF8FFF791
:1029E000B5FBFFF769FB5D4B5D48196804F066FBBA
:1029F0005C4B019300943E4B5B4A5C493B4804F0BE
:102A000047F85B4B01930094394B5A4A5749374872
:102A100004F0B4F8584B01930094354B574A584989
:102A2000324804F035F8324B564A55492F488DE864
:102A3000500004F071F830780AF04EFF52490BF064
:102A400057F852490AF0A0FF4FF07C510AF094FE6B
:102A50000BF060F9387007B0BDE8F08F0234244BFA
:102A6000019400964A4A4B49204804F055F897F8DB
:102A70002D30002B3FF41AAD474B019350230093A8
:102A8000464A1B4B4349194804F046F897F845302D
:102A9000002B3FF410AD424B019350230093414A69
:102AA000134B3C49114804F037F897F85D30002B80
:102AB0003FF406AD3C4B0193502300933B4A0C4B33
:102AC00034490A4804F028F897F87530002B3FF491
:102AD000FCAC374B019350230093364A044B2D49ED
:102AE000024804F019F8F0E4D0FE0000B4CDFF1F56
:102AF000B8C3FF1FD8FE00008D9BFF1FCCA0FF1F97
:102B0000E4FE0000F0FE0000FCFE000008FF0000F4
:102B100014FF000020FF00002CFF0000C4B4FF1FC2
:102B200038FF000044FF0000A0C3FF1F50FF00005B
:102B3000ACCEFF1F5CFF00006CFF000062CEFF1FE9
:102B400074FF00009ECEFF1F80FF00008A9BFF1FC6
:102B50008CFF00008C9BFF1F98FF0000D8A4FF1F74
:102B600064CAFF1F2CC2FF1FA4FF0000A4FE0000C8
:102B70008CCDFF1FB0FF00008B9BFF1FBCFF000030
:102B8000CCFF0000D8FF00000000C84200007F43D7
:102B9000A4FD0000ACFD000071B2FF1FC0FD0000ED
:102BA00089B2FF1FC8FD0000A1B2FF1FD0FD0000C9
:102BB000B9B2FF1FD8FD000038B51F4C1F4A23785B
:102BC00013708342207007D0022B06D0022811D048
:102BD00001281DD0082812D038BD194B1B78012BB5
:102BE000F4D1184B1B68F3B90228F1D1FDF736FD7B
:102BF0002078EDE7124B1B78012BF7D038BD0F2161
:102C0000114809F0FFF81148BDE8384009F050BDFF
:102C10000C210F4809F0F6F80C4809F049FD20781E
:102C20000828D9D1EBE70B4D0B48296804F0C0FB0D
:102C300000232B602078C9E782CEFF1FA1CEFF1FA3
:102C400043CAFF1F8CCDFF1FF8FF0000D0A7FF1F56
:102C5000E8FF0000A4CEFF1F0CB3FF1F034B1B783F
:102C600003B170470120FFF7A7BF00BF82CEFF1F4F
:102C7000044B1B7813F0F70F02D00820FFF79CBF1E
:102C8000704700BF82CEFF1F174B184A1B78107089
:102C9000012B174B1B780ED063B1164B1B78012B01
:102CA00007D9082B05D0A0B9052B1AD0033B012B5F
:102CB00014D970477047002BFBD00F4B1B78002BAB
:102CC000EBD00C4B1B78002BE9D10328F1D9FFF78F
:102CD000C5BF022BEDD10320FFF76EBF0620FFF723
:102CE0006BBF0720FFF768BF43CAFF1F74C3FF1FF6
:102CF00081CEFF1F82CEFF1F2CC2FF1FF8B5154EDD
:102D00004FF4307505FB0065044628460F4604F075
:102D10007DFE114B1B7833B92FB195F8AC3213B14E
:102D20000E4B1B788BB94FF4307000FB046000230E
:102D300080F8AE3280F8AF3280F8BE3280F8AC3224
:102D400080F8AD3280F8B832F8BD2046FDF708FFB4
:102D5000E9E700BF9CB5FF1F48CAFF1FE299FF1FAC
:102D60002DE9F0432C4B93F8CD4083B0002C3DD09F
:102D7000DFF8B890DFF8B88099F90240B9F8003070
:102D80004FF4307000FB0480B0F8BA229A423DD074
:102D9000224D0FCD4FF4307707FB04F608EB060EFB
:102DA0000EF525740FC495E80300012384E80300A1
:102DB00000240EF525718EF8AC3270468EF8AD42C7
:102DC0008EF8BE4204F056FE154A99F90200154BE2
:102DD0001268019207FB0087134A1B780199C7F814
:102DE000B012147063B903B0BDE8F0830F4B01213A
:102DF0009878FFF783FF0C4B1C7003B0BDE8F0839D
:102E0000C0B2FDF79FFC03B0BDE8F08304F0FEFD07
:102E100099F90240BCE700BF909CFF1F509DFF1F27
:102E200060DEFF1FE299FF1FA0CEFF1FA0C0FF1FA3
:102E30009CB5FF1FF8B5264C264E257815BB337878
:102E4000002B35D0244B0227384629461F70FFF748
:102E500055FF03202946FFF751FF2048204A437BB6
:102E600017705BBB1F4A204B12781B781F4813FB5F
:102E700002F31B1203EB430300EBC300437B1BBBBA
:102E800001232370317899B91948457B8DB92946BA
:102E90000220FFF733FF29460320FFF72FFF1049D9
:102EA0000D4B0220042208701A7000232370F8BD15
:102EB000F8BD03230122FDF79DFDF6E701232A4615
:102EC0002946FDF797FDDBE73946FDF743FED7E7D7
:102ED000FDB4FF1FD4C0FF1F20A0FF1FB4A0FF1F21
:102EE0007C9AFF1F34C2FF1F94CEFF1FDCA4FF1F7C
:102EF00024A0FF1F70B50A4C06460025237E2046FD
:102F0000314604F5307413B10BF02EFE28B10135B3
:102F1000042DF3D14FF0FF3070BD68B270BD00BF1B
:102F200030B8FF1FF0B50138C4B2194B04EB4405AB
:102F300003EBC50583B00E4628461746FFF7DAFFB8
:102F40001EB100280ADB03B0F0BD0028FBDBC0B2D5
:102F5000012103B0BDE8F040FFF7D0BE6B7B5FB14D
:102F6000002BF0D00B490023284601EB840100938D
:102F70000122FDF72BFCE6E7002BE4D005493A4699
:102F8000284601EB840103B0BDE8F040FDF728BD01
:102F90000098FF1F68C2FF1F022810D0032804D02A
:102FA000012800D07047FDF70FBD0A4890F8ED31B9
:102FB000002BF7D000F5F0700B21FDF7F9BC0548A8
:102FC00090F8D531002BEDD000F5E4700A21FDF723
:102FD000EFBC00BF909CFF1F022816D003280BD027
:102FE000012800D070470D4890F84D32002BF9D0E1
:102FF00000F51070FDF7D0BC084890F87D32002B2A
:10300000F0D000F51C70FDF7C7BC044890F865329D
:10301000002BE7D000F51670FDF7BEBC909CFF1F9B
:1030200000B5012885B006D00F4A92F8AD3273B9C9
:1030300005B05DF804FB0C4890F8AD32002BF7D0DA
:1030400000F52870FDF7A8FC05B05DF804FB002131
:103050000346009102F5287003A90122FDF7B6FB93
:1030600005B05DF804FB00BF909CFF1F20B109482C
:1030700090F8DD324BB97047064890F8F532002BD6
:10308000F9D000F53A70FDF787BC00F53470FDF714
:1030900083BC00BF909CFF1F2DE9F047414C84B0DA
:1030A0002378A0B183B9404890F8E530002B59D07F
:1030B000D83003223D49FDF793FC002855D0012369
:1030C00023703B4B00221A7004B0BDE8F087002B40
:1030D000FAD0374F3B78002BF6D1334B93F815518C
:1030E000002D48D0DFF8C4A0DFF8D4909AF9024050
:1030F000BAF800304FF4307000FB0490B0F8BA22F8
:103100009A4249D02B4D0FCD4FF4307808FB04F68E
:1031100009EB060E0EF525740FC495E80300012394
:103120000422002584E803008EF8BE228EF8AC321B
:103130000EF5257170468EF8AD523B7004F09AFC86
:103140001D4A9AF902001D4B1268039208FB009871
:103150001B78039AC8F8B022002BB5D0C0B2FDF797
:10316000F1FAB1E790F8FD206AB9114B00221A700C
:1031700004B0BDE8F0870D4B29469878FFF7BEFDF7
:1031800025703D70A0E70093F03001220749FDF75C
:103190001DFB002893D1E8E704F038FC9AF90240BF
:1031A000B0E700BF40CAFF1F909CFF1FA4C0FF1FD5
:1031B00064C2FF1F989DFF1F60DEFF1FE299FF1F83
:1031C0009CB5FF1F2DE9F047424C84B06378A8B14D
:1031D0008BB9414890F82D31002B5AD000F59070F2
:1031E00005223E49FDF7FCFB002855D00123637002
:1031F0003B4B00225A7004B0BDE8F087002BFAD098
:10320000374F7B78002BF6D1334B93F85D51002D6F
:1032100048D0DFF8C8A0DFF8D8909AF90240BAF891
:1032200000304FF4307000FB0490B0F8BA229A429C
:103230004AD02C4D0FCD4FF4307808FB04F609EB43
:10324000060E0EF525740FC495E80300012306222F
:10325000002584E803008EF8BE228EF8AC320EF50D
:10326000257170468EF8AD527B7004F003FC1E4A47
:103270009AF902001D4B1268039208FB00981B7814
:10328000039AC8F8B022002BB5D0C0B2FDF75AFAA5
:10329000B1E790F845216AB9114B00225A7004B089
:1032A000BDE8F0870D4B29469878FFF727FD65703C
:1032B0007D70A0E7009300F59C7001220749FDF79F
:1032C00085FA002892D1E7E704F0A0FB9AF90240C2
:1032D000AFE700BF40CAFF1F909CFF1FF0CCFF1F4D
:1032E00064C2FF1FE09DFF1F60DEFF1FE299FF1F0A
:1032F0009CB5FF1F2DE9F047424C84B0A378A8B1DC
:103300008BB9414890F87531002B5AD000F5B47054
:1033100007223E49FDF764FB002855D00123A37026
:103320003B4B00229A7004B0BDE8F087002BFAD026
:10333000374FBB78002BF6D1334B93F8A551002DB6
:1033400048D0DFF8C8A0DFF8D8909AF90240BAF860
:1033500000304FF4307000FB0490B0F8BA229A426B
:103360004AD02C4D0FCD4FF4307808FB04F609EB12
:10337000060E0EF525740FC495E8030001230822FC
:10338000002584E803008EF8BE228EF8AC320EF5DC
:10339000257170468EF8AD52BB7004F06BFB1E4A6F
:1033A0009AF902001D4B1268039208FB00981B78E3
:1033B000039AC8F8B022002BB5D0C0B2FDF7C2F90D
:1033C000B1E790F88D216AB9114B00229A7004B0D0
:1033D000BDE8F0870D4B29469878FFF78FFCA57064
:1033E000BD70A0E7009300F5C07001220749FDF70A
:1033F000EDF9002892D1E7E704F008FB9AF90240C2
:10340000AFE700BF40CAFF1F909CFF1F68C1FF1FAE
:1034100064C2FF1F289EFF1F60DEFF1FE299FF1F8F
:103420009CB5FF1F02280AD0032805D0012800D030
:1034300070470846FFF730BE0846FFF75BBF0846F7
:10344000FFF7C0BE2DE9F0415C4C84B02378A8B1F1
:103450008BB95B4B5B481B78002B74D190F85530CF
:10346000002B00F08180483001225749FDF7B8FA5F
:1034700008B10123237004B0BDE8F081002BFAD01D
:103480004F4E50483378002B46D190F88520002AC3
:1034900042D0DFF834814D4F98F90250B8F800203F
:1034A0004FF4307303FB0573B3F8BA329A427BD002
:1034B000DFF828E1BEE80F004FF4307606FB057612
:1034C00006F525760FC69EE8030086E803004FF454
:1034D000307606FB05F57B190122002583F8AC2226
:1034E00003F52571184683F8AD5283F8BE5204F0F7
:1034F000C1FA374A98F90200364B1268039206FB6C
:1035000000771B78039A2570C7F8B022002BB2D041
:10351000C0B2FDF717F9AEE790F83D50EDB1DFF816
:10352000A8802A4F98F90250B8F800104FF4307272
:1035300002FB0572B2F8BA228A4235D0002BB7D00E
:10354000DFF89CE0B6E7437BA3B101221E491D488A
:10355000FDF746FA00288CD18DE71B4B01219878A6
:10356000FFF7CCFB257086E7437B002BEDD190F86D
:103570006D207AB990F82530002B3FF47CAF002302
:103580000093012210491448FDF720F900287FF428
:1035900070AF70E70093603001220B49FDF716F918
:1035A00000287FF466AF66E74FF4307000FB0570CB
:1035B00004F02CFA337898F90250BFE7C5B4FF1F26
:1035C00081C1FF1F909CFF1F58C3FF1F9CB5FF1FA9
:1035D00060DEFF1FE299FF1FA89CFF1F089DFF1FD1
:1035E000C09CFF1F90B110B5124C237882B05BB91C
:1035F000114890F89D307BB1903002220F49FDF7C1
:10360000EFF908B10123237002B010BD094B1B78FC
:103610000BB1FFF7A5BB704790F8B520002AF3D097
:103620000093A83001220549FDF7D0F80028E9D120
:10363000EAE700BFA0CEFF1F909CFF1FA0C0FF1FA6
:1036400010B5114C82B0237830B13BB90F4890F8D7
:10365000952262B902B010BD002BFBD00C4B0121AA
:103660009878FFF74BFB0023237002B010BD009346
:1036700000F5227001220649FDF7A8F80028E9D0DC
:1036800001232370E6E700BFA3CEFF1F909CFF1F1E
:10369000BCC2FF1F38B5144A144C154D216815489B
:1036A00000235371537582F8253082F8353082F843
:1036B000453082F855302B7003F0BAFE78B90E4BC6
:1036C0001B7813B10D4B1B7803B938BD0C210C4886
:1036D00008F098FB0B48BDE8384008F0E9BF2168C6
:1036E000044803F065FEEAE700B5FF1FA8C0FF1F0E
:1036F0004CB2FF1F0CB3FF1FE299FF1F28C1FF1F31
:1037000008000100D0A7FF1F10B5084A084B126837
:1037100082B000011C180192019A185A6188A260B7
:1037200009F038F9A08102B010BD00BF60DEFF1FB4
:1037300000B5FF1FF8B5154B1B78C3B1144D154EDE
:10374000002401272B79E0B2013423B16B7913B93E
:1037500096F80D3363B9062C05F1100506F118062D
:10376000F0D10D4B1B7813B10C4B1B7823B9F8BD6E
:103770006F71FFF7C9FFEEE70D21094808F042FB22
:103780000848BDE8F84008F093BF00BF4CB2FF1FE7
:1037900000B5FF1F909CFF1FE299FF1F28C1FF1F6C
:1037A00018000100D0A7FF1F134B03EB00135B7938
:1037B000B3B110B500F120030446104803EB4303F6
:1037C00000EBC300437B63B92046FFF79DFF0C4B22
:1037D0001B7803B910BD2046BDE81040FCF788BF38
:1037E0007047FDF7D9F82046FFF78EFF044B1B7892
:1037F000002BEFD0EFE700BF00B5FF1F909CFF1F2D
:10380000E299FF1F70B50C4D0C4E82B000246B790D
:10381000E0B24BB133680193019BA968AA895B1A96
:10382000934201D3FFF7C0FF0134062C05F11005C8
:10383000EDD102B070BD00BF00B5FF1F60DEFF1FFD
:10384000F0B5244A13788A2B83B0044639D822482D
:10385000591C40F823401170204605F03DFD0546F7
:1038600018B90025284603B0F0BD1C481C4E04F0D2
:10387000CDF82146194804F0FDF833680093174845
:10388000009F04F089FB60B9206980B93368019317
:10389000019BDB1B052BE4D8104804F07DFB0028BE
:1038A000F2D00E4804F08EFB20610028EED03228C2
:1038B000D7D901236373094804F0A8F8284603B058
:1038C000F0BD3C21074808F09DFA074808F0F0FEDB
:1038D000C2E700BF48CEFF1F6CCAFF1F9CB5FF1F89
:1038E00060DEFF1F28000100D0A7FF1F10B50024D5
:1038F000E0B200210134FFF701FA042CF8D10548A9
:1039000004F084F8044804F081F8044B00221A7093
:1039100010BD00BF08C4FF1FC8C6FF1F08CEFF1F91
:10392000F8B51546126804460E46EAB900292BDDA3
:1039300001464FF0FF370AE00A6028680132013083
:103940009642286003F1180301F104010AD0587B64
:103950000028F1D1013296420F6003F1180301F102
:103960000401F4D12B687BB1304609F00FF804EB69
:10397000800354F82000421CF6D02A684FF0FF3133
:103980000A442A601960F8BD4FF0FF30F8BD00BF4F
:1039900010B50A4C0A4A0B4823460521FFF7C0FF21
:1039A000002805DB00EB400004EBC000437B03B9BB
:1039B00010BDBDE81040FCF7EFBF00BF3CA0FF1FEB
:1039C000D8C1FF1F78C3FF1F10B50D4C0D4A0E481C
:1039D00023461421FFF7A4FF00EB400304EBC304CC
:1039E0000A4A637B106023B120460E220849FCF787
:1039F000F7FF0849084B0E20012208701A7010BD0D
:103A0000D0A0FF1F64CEFF1FDCC1FF1FA8CEFF1F89
:103A1000989BFF1F8E9BFF1FA2CEFF1F70B5564BBA
:103A20001B78013B072B12D8DFE803F0331112118A
:103A30001104532A514B1B78002B60D0504B5B7BF9
:103A4000002B5CD000214E48FDF7C8F952E070BD54
:103A50004C4C4D4A4D4823460521FFF761FF40B2CB
:103A600000286FDB00EB400004EBC000437B13B188
:103A70000221FDF7ADF90420BDE87040FFF79CB8C6
:103A80004348437B002B59D10020BDE87040FFF72D
:103A900093B8404C2578002DD9D13F483F4E03F0D4
:103AA000B5FF3F4803F0B2FF3E4A33781570002B54
:103AB00037D03D4B5B7B002B3BD13C4B5B7B1BB141
:103AC00001213A48FDF790F900220123327023705A
:103AD00070BD374C374A384823460521FFF720FF91
:103AE00040B20028A6DB00EB400004EBC000437BA3
:103AF000002B3DD10220BDE87040FFF75DB82F4C90
:103B00002F4A304823460521FFF70AFF00EB40000B
:103B100004EBC000437B002BECD00021FDF75EF9E5
:103B2000E8E7224B5B7B002BCAD11F4B5B7B002B52
:103B3000CAD001211C48FDF757F9C5E70421FDF75C
:103B400047F9A1E7204A214B12781B78204813FB44
:103B500002F31B1203EB430300EBC300437B13B1DF
:103B60000321FDF73BF90520BDE87040FFF724B8BD
:103B70000121FDF72DF9BDE782CEFF1FA1C3FF1F75
:103B8000ACA4FF1F049AFF1F98CDFF1FA4C3FF1F03
:103B9000709BFF1F81C1FF1F08C4FF1FE199FF1F1A
:103BA000C8C6FF1F08CEFF1F90A4FF1FE499FF1F88
:103BB000189CFF1F94B5FF1F38C2FF1F9C9BFF1F5F
:103BC00044CAFF1F10CAFF1F74C3FF1F54C3FF1F47
:103BD000809AFF1F2DE9F0477C4C7D4EDFF818825C
:103BE0007C4F86B004F5B06594F8AC322BB394F8F2
:103BF000BE32042B21D8DFE803F03903688E27009A
:103C0000204604F0C9F9C0B1204604F0CDF9D4F83B
:103C1000A432A3F5C87398420FD36F4B1B78002BC7
:103C200000F095806D48437B002B00F090800021D0
:103C3000FDF7D4F80220FEF7BFFF04F53074AC4264
:103C4000D2D106B0BDE8F087204604F0A5F90028DF
:103C5000F3D133680293029BD4F8B0229B1A042B51
:103C6000EBD984F8AC0288F80000E6E7204604F0BF
:103C700093F968B933680393039BD4F8B0229B1A75
:103C8000042B05D994F8AD32002B71D184F8AC32F5
:103C9000204604F081F90028CFD094F8AC32002BF4
:103CA000CBD094F8B832002BC7D033680593059B6E
:103CB000D4F8B4229A42C0D0204603F0A7FE0023D5
:103CC00084F8AC3284F8B832B7E7204604F064F9DF
:103CD0000028B2D0204604F067F9D4F8A432A3F546
:103CE000C8739842A9D33E4A3E4B11781B783E4A8E
:103CF00011FB03F31B1203EB430002EBC0005FFA5E
:103D000083F9437B002B3ED1384B052083F800908C
:103D1000FEF752FF91E73B78052B8ED1314B304AAD
:103D20001B781278DFF8C49012FB03F31B1299F88A
:103D300000205FFA83FA52452DD02B4803EB430352
:103D400000EBC300437B13BB89F800A075E7DFF8E5
:103D5000AC90274A27484B460521FFF7E1FD00EBD1
:103D6000400009EBC000437B002B3FF463AF5EE7EC
:103D700004F52571204603F07DFE33680493049B0F
:103D8000C4F8B03284E70321FDF728F8BCE703212B
:103D9000FDF724F8D8E7204604F0FEF800287FF469
:103DA0004CAF33680093009BD4F8B0229B1A042BCD
:103DB0007FF643AF04F52571204603F05BFE3368C0
:103DC0000193019BC4F8B03237E700BF08C4FF1F5E
:103DD00060DEFF1F82CEFF1FA1C3FF1FACA4FF1F29
:103DE00054C3FF1F74C3FF1F809AFF1F68CEFF1FBD
:103DF00044CAFF1F10CAFF1F81C1FF1F9C9BFF1FEA
:103E00002DE9F047614C624EDFF89881614F86B032
:103E100004F5B06594F8AC326BB394F8BE32032B62
:103E200029D8DFE803F06C4B022F5B4B5B4A1B7811
:103E30001278DFF8749112FB03F31B1299F800203B
:103E40005FFA83FA524540F08880204604F0A4F8D7
:103E500088B933680093009BD4F8B0229B1A042BD6
:103E600009D904F52571204603F004FE3368019357
:103E7000019BC4F8B03204F53074AC42CAD106B02C
:103E8000BDE8F087204604F087F881460028F2D18B
:103E900033680293029BD4F8B0229B1A042BEAD910
:103EA00001460220FEF72AFF49460320FEF726FFBF
:103EB0000222042388F800203B70DCE7204604F04F
:103EC0006BF80028D7D0204604F06EF8D4F8A4325E
:103ED000A3F5C8739842CED32F4A304B12781B7883
:103EE0002F4813FB02F31B1203EB430300EBC30049
:103EF000437B002BBFD00221FCF72CFEBBE7204602
:103F000004F04AF860B933680393039BD4F8B022F5
:103F10009B1A042B04D994F8AD3263BB84F8AC32FD
:103F2000204604F039F80028A5D094F8AC32002BD4
:103F3000A1D094F8B832002B9DD033680593059B2F
:103F4000D4F8B4229A4296D0204603F05FFD0023B5
:103F500084F8AC3284F8B8328DE7114803EB4303A0
:103F600000EBC300437B13B989F800A083E702216B
:103F7000FCF7F0FDF8E704F52571204603F07AFD23
:103F800033680493049BC4F8B032C9E71CBBFF1F1D
:103F900060DEFF1F20A0FF1F34C2FF1F94CEFF1F53
:103FA000DCA4FF1F7C9AFF1FECCCFF1F10B5002480
:103FB0000134E4B2002220461146FEF7B3FF142C70
:103FC000F6D110BD38B558B3012826D1174B1D883E
:103FD00093F90200002820DB154B1C78F4B1013C5A
:103FE000E4B24FF43072134B04FB02221A4403E094
:103FF00003F53073934210D093F8AC42002CF7D005
:10400000B3F8BA12A942F3D193F9BC128142EFD1AD
:10401000C0B20021FEF772FE00E00024204638BD49
:10402000054B1D8893F90200D4E700BFFC99FF1FE0
:1040300020A0FF1F9CB5FF1F989BFF1F10B50446D3
:10404000FFF7C0FF90B994B1012C00D010BD164B02
:104050001B785BB1154B16481B6803EB430300EB61
:10406000C300437BCBB9134B01221A7010BD124B16
:104070001B78002BFAD0114B11481B6803EB43034C
:1040800000EBC300437B23B10E4B0F491A78FCF7BA
:10409000A7FC0E4B01221A7010BD0D4B0D491A786A
:1040A000FCF79EFCDFE700BFB8C2FF1F84CEFF1FF6
:1040B000B0A2FF1FD4CCFF1F80CEFF1FA8CEFF1FD2
:1040C000D0A0FF1F8E9BFF1F989BFF1FA2CEFF1F3C
:1040D000149CFF1FFC99FF1FF8B5054600283CD033
:1040E000012838D13F4B1B78002B35D03E4B3F4940
:1040F0001A780F68002A5ED13D4E18702846FFF7E7
:1041000061FF002F36D1002404EB440306EBC30308
:104110005B7B002B3BD10134E4B2142C30D1002F57
:1041200010DD0024234603EB430206EBC202527B60
:104130001AB1002D45D0012D2CD00133DBB2BB428A
:104140001C46F0DB25212B4807F05CFE2A48BDE821
:10415000F84008F0ADBAF8BDF8BD284B1B78002B2D
:10416000FAD0274B27491A780F6832B3264E2846D3
:10417000FFF728FF122FC6DC7C1CE4B2132CCED82C
:1041800004EB440306EBC3035B7B002BC3D0C5B138
:10419000012DC0D1164B04EB440003EBC000437B60
:1041A0001BB10F221949FCF71BFC104A184B146075
:1041B0000F221A70F8BD0E4ED9E701221A70124E66
:1041C0009CE7114B04EB440003EBC000437B1BB1A5
:1041D0000C221049FCF704FC0A4A0F4B14600C2215
:1041E0001A70F8BDB8C2FF1FD4CCFF1F84CEFF1FCA
:1041F000B0A2FF1F68000100D0A7FF1F80CEFF1FE5
:10420000A2CEFF1FA8CEFF1FD0A0FF1FFC99FF1F4B
:10421000149CFF1F989BFF1F8E9BFF1F70B548B318
:10422000012825D1274B1B781BB3274A274B14683D
:1042300018700546FFF7C6FE002C254E29DD013C0F
:10424000E4B204EB440306EBC3035B7B002BF6D024
:104250000DB3012DF3D11E4B04EB440003EBC00062
:10426000437B53BB184A1B4B146010221A7070BD5D
:1042700070BD70BD184B1B78002BFAD0174A184B35
:104280001468184E01221A700546FFF79BFE002C99
:10429000D5DC1324D5E7134B04EB440003EBC0003B
:1042A000437B2BB90D4A104B14600D221A7070BD60
:1042B0000D220E49FCF794FBF4E710220C49FCF7A1
:1042C0008FFBCFE7B8C2FF1F84CEFF1FD4CCFF1FE8
:1042D000B0A2FF1F149CFF1F80CEFF1FA8CEFF1FA0
:1042E000A2CEFF1FD0A0FF1F8E9BFF1F989BFF1F1A
:1042F000FC99FF1F10B50446FFF764FEC4B1012C02
:1043000015D1104C104A114823461421FFF708FB21
:1043100000EB400304EBC3040D4A637B10605BB900
:104320000C490D4B1120012208701A7010BD10BDF0
:10433000BDE81040FFF748BB204611220749FCF7B3
:104340004FFBEDE7B0A2FF1F04B3FF1F04C3FF1F25
:1043500084CEFF1F149CFF1FD4CCFF1FFC99FF1FAE
:104360002DE9F04FB74F3B7889B0002B3AD0B64ECD
:10437000DFF8F482DFF8F492002404E001343B78A3
:10438000E4B2A3422ED94FF4307505FB046595F8CD
:10439000AC32002BF2D0284603F0FEFD0028EDD110
:1043A000D8F800300093009BD5F8B0229B1A042B5C
:1043B000E4D995F8BE32013B102B00F29281DFE880
:1043C00013F028010A01EC00E200C400BA008C00DE
:1043D00082007A0072006A005D00510041003200E4
:1043E0002300140009B0BDE8F08F4FF4307303FBD5
:1043F000046399F80020002183F8AC12002ABDD094
:104400000120FFF777FFB9E74FF4307303FB046334
:1044100099F80020002183F8AC12002AAED00120C8
:10442000FFF7FCFEAAE74FF4307303FB046399F82F
:104430000020002183F8AC12002A9FD00120FFF752
:104440004BFE9BE7814A4FF4307303FB0463127801
:10445000002083F8AC02002A90D0FFF7B3FDFFF7ED
:10446000B3FA8BE7794A4FF4307303FB0463127895
:10447000002083F8AC02002A80D0D1E7734A4FF4C1
:10448000307303FB04631278002083F8AC02002A27
:104490003FF474AFD3E76E4A002319469370204669
:1044A000FEF72CFC6AE76A4A00231946537020463F
:1044B000FEF724FC62E7664A002319461370204683
:1044C000FEF71CFC5AE76349634A00238B702046C1
:1044D00001219370FEF712FC50E7DFF894C1BCE8AD
:1044E0000F004FF4307B0BFB04FB06EB0B0A0AF5C5
:1044F000257EAEE80F009CE803008EE803000AF575
:104500002571284603F0B6FAD8F80020534B0592DF
:104510001A78059BCAF8B032012100238AF8AD123F
:104520008AF8AE328AF8BE32002A3FF427AF20461E
:10453000FCF708F922E74749474A00234B70204619
:1045400001215370FEF7DAFB18E7DFF828C1BCE859
:104550000F004FF4307B0BFB04FB06EB0B0A0AF554
:10456000257EAEE80F009CE803008EE803000AF504
:104570002571284603F07EFAD8F80020374B0492C4
:104580001A78049BC6E73349334A00230B70204650
:1045900001211370FEF7B2FBF0E6DFF8DCC0BCE8E7
:1045A0000F004FF4307B0BFB04FB06EB0B0A0AF504
:1045B000257EAEE80F009CE803008EE803000AF5B4
:1045C0002571284603F056FAD8F80020234B0392B1
:1045D0001A78039B9EE7DFF8A4C0BCE80F004FF4F5
:1045E000307B0BFB04FB06EB0B0A0AF5257EAEE8DD
:1045F0000F009CE803008EE803000AF525712846A9
:1046000003F038FAD8F80020144B02921A78029B73
:1046100080E7134B1B789BBB124B93F86D207AB34A
:1046200003F1600EBEE80F004FF4307C0CFB046C0D
:104630000CF5257CACE80F009EE803008CE8030035
:104640002EE000BF20A0FF1F9CB5FF1FC4B4FF1FBA
:1046500070C3FF1F40CAFF1F64C2FF1FE299FF1F04
:1046600081C1FF1F909CFF1F60DEFF1FA0C3FF1FC3
:10467000109EFF1FC89DFF1F809DFF1F389DFF1FBD
:10468000DFF8E0C0BCE80F004FF4307E0EFB046E94
:104690000EF5257EAEE80F009CE803008EE80300CF
:1046A0004FF4307303FB04FA06EB0A0101F52571A0
:1046B000284603F0DFF9D8F80030284A019306EBCA
:1046C0000A031178019AC3F8B0220120002283F86E
:1046D000AD0283F8AE2283F8BE2200293FF44EAE2D
:1046E00025E74FF4307303FB04F306EB030A9AF853
:1046F000AD22A2B19AF8AE12A1B19AF8AF2201325E
:10470000D2B291428AF8AF221AD800238AF8AC328A
:104710008AF8AD328AF8AE328AF8AF322EE68AF8DD
:10472000AC222BE60E4AD11801F52571284603F07C
:10473000A1F9D8F800300693069BCAF8B0321DE6FE
:10474000074AD11801F52571284603F093F9D8F8E6
:1047500000300793079BCAF8B0320FE6E299FF1FBB
:104760009CB5FF1FA89CFF1F10B50F4C0F480021E0
:1047700007F048FB204607F09BFFFCF78BFC12215B
:104780000B4807F03FFB204607F092FFFCF782FC46
:104790001B21084807F036FB204607F089FFBDE8DB
:1047A0001040FCF777BC00BFD0A7FF1FE00001005E
:1047B00090000100A400010038B50E4D0E4C002100
:1047C000284607F01FFB204607F072FFFCF762FC4B
:1047D00010210A4807F016FB204607F069FFFCF796
:1047E00059FC2846002107F00DFB2046BDE8384063
:1047F00007F05EBFE0000100D0A7FF1FC00001006E
:1048000070B50646441E00F10C0514F8010F07F0C0
:104810007DFBA542F9D10620FBF754FF737B7BB9E2
:1048200001210D4807F0EEFA0D20FBF74BFF09219F
:104830000A4807F0E7FA0A48BDE8704007F038BFB9
:104840003069FCF7A5FB0620FBF73CFF0C2105486F
:10485000BDE8704007F0D6BA30F80000E40001006F
:10486000D0A7FF1FD4000100F0B53A4885B003F08F
:1048700093FB10B9384C237823BB364803F08CFBEC
:10488000F0B9354C2378DBB9344F354A3B68029395
:10489000029B12689B1AB3F5487F11D9314D324EF5
:1048A000B5F9003056F8230004F016FD002844D175
:1048B000B5F90020012356F822002370FFF7A0FF6E
:1048C00005B0F0BD254E294A33680093009B12685D
:1048D0009B1A642BD1D9264A13788BB9214D01211B
:1048E000B5F9003011703268019201331C4A019908
:1048F00011601BB200228A2B227014DC2B80BCE7D3
:10490000184D194AB5F9003052F82320527B002A7D
:10491000E9D00421174807F075FA174807F0C8FED8
:10492000B5F90030DFE714482A8007F0C1FEFCF734
:10493000B1FB114807F0BCFE9FE7B5F90030054810
:1049400056F8231003F096F83B680393074B039A3D
:104950001A60ADE79CB5FF1FD4A4FF1F60DEFF1FE8
:10496000B0CDFF1F889BFF1F6CCAFF1F9CC0FF1F9D
:1049700060CEFF1FF0000100D0A7FF1F10B50C4A4A
:104980000C4B127819789142044607D01D210A4831
:104990001A7007F037FA094807F08AFE204608F037
:1049A0009BFF0749074C09F0A3F8206010BD00BF2A
:1049B000D5A4FF1F35C2FF1FF8000100D0A7FF1FBD
:1049C0000000C84270B4FF1F38B543780F3B442B3A
:1049D0004CD8DFE813F0CC014B004B004B004B00F0
:1049E0004B004B004B004B004B004B004B004B006F
:1049F0004B004B004B004B004B004B004B004B005F
:104A00004B004B004B004B004B004B004B004B004E
:104A1000C301B801B301AE01A901A401A001940131
:104A200088017E01700164015F015A0155014C014A
:104A3000400136012C012201190115010301F0008A
:104A4000DE00D200CD00C800BD00B400A8008C007C
:104A50007D0075007100A100960053004C00D1014B
:104A6000C378C74A003318BF0123137038BD837859
:104A7000002B00F0B681012BF2D038BDC3788078CE
:104A8000013B003018BF0120082BEFD801A252F8DB
:104A900023F000BFD54D00006D4A00006D4A0000B4
:104AA0006D4A00006D4A00006D4A0000CD4D0000C7
:104AB000C54D0000BD4D0000BDE83840FEF768BFA1
:104AC0008078003018BF0120BDE83840FEF7CEBA2C
:104AD0008378C578AB4C642BA8BF6423184608F0D4
:104AE000FBFEA94909F004F844F8250038BD837895
:104AF000A64A1370002B00F07181A54B01221A7099
:104B000038BDA44890F86532002BAFD000F5167080
:104B1000BDE83840FBF740BF83789F4A003318BF99
:104B20000123137038BD9D4B5B78002B9ED09C4BAE
:104B3000587800289AD1BDE83840FEF743BB974B20
:104B40005B78002B92D10120BDE83840FEF73ABBDC
:104B5000904890F8C532002B88D000F52E70BDE843
:104B60003840FBF719BF8078BDE83840FFF706BF33
:104B70008078BDE83840FEF753BA864890F8AD32E9
:104B8000002B3FF473AF00F52870BDE83840FBF709
:104B900003BFC378013BDBB2052B3FF667AF8178DB
:104BA000804A814802EB03130A1C18BF012201212D
:104BB0001A71017038BDC378013BDBB2052B3FF69B
:104BC00055AF8278774902EB820202EB82025200F3
:104BD00001EB031302F5FA725A8038BDC378013B2A
:104BE000DBB2052B3FF642AF82786E4902EB8202C0
:104BF00002EB820252001B0102F5FA72CA5238BD62
:104C0000BDE83840FEF746BD684B1B78002B7FF4AB
:104C10002DAFBDE83840FBF73FBDC07814283FF604
:104C200025AF00221146BDE83840FEF77BB9C078B9
:104C300014283FF61BAF01221146BDE83840FEF7AD
:104C400071B9C07814283FF611AF00220121BDE8E8
:104C50003840FEF767B94F4890F84D32002B3FF4CB
:104C600005AF00F51070BDE83840FBF795BE504B1E
:104C70001B78002B3FF4FAAEBDE83840FEF770B861
:104C80000120BDE83840FEF7ADBC0020BDE838404B
:104C9000FEF7D8BB0120BDE83840FEF7D3BB3D4846
:104CA00090F81D32002B3FF4E1AE00F50470BDE832
:104CB0003840FBF771BE394B1B78002B3FF4D6AE62
:104CC000374B187800287FF4D1AEBDE83840FEF7A6
:104CD000E3B9324B1B78002B7FF4C8AE0120BDE84E
:104CE0003840FEF7D9B92B4890F83532002B3FF405
:104CF000BDAE00F50A70BDE83840FBF74DBE254853
:104D000090F80532002B3FF4B1AE00F5FC70BDE821
:104D10003840FBF741BEBDE83840FBF755BE0020E8
:104D2000BDE83840FEF78CBC0120BDE83840FEF7F6
:104D300087BC0020BDE83840FDF7A6BF8078BDE8FD
:104D40003840FDF7A1BF1B4B1B7813F0F70F3FF462
:104D50008DAE0820BDE83840FDF72EBF164B1B78FE
:104D6000002B3FF483AEBDE83840FDF777BF807875
:104D7000BDE83840FDF766B9BDE83840FFF716B921
:104D8000A0C3FF1FC4A4FF1F0000C84234C2FF1FFE
:104D9000D4C0FF1F909CFF1FA1C3FF1F40CAFF1F6D
:104DA00064C2FF1F00B5FF1F28C1FF1F4CB2FF1FC9
:104DB000A0CEFF1F82CEFF1F81CEFF1FBDE838406F
:104DC000FFF798BABDE83840FFF728BABDE8384089
:104DD000FFF782B9BDE83840FFF730B9044A1370D5
:104DE00038BDC378034A003318BF0123137038BDA0
:104DF000D4C0FF1FC4B4FF1FF0B52A4C2A4D2B4E60
:104E000085B0012705F0DAFF002833D005F0E6FF72
:104E1000C0B2DA2827D02B78244A2349002BF1D0BE
:104E200094F800E00EF10103DBB2042B06F80E004B
:104E30002370E7D91E4D507813789778D6782B7069
:104E400003443B44334468701079AF7003F07F0330
:104E50009842EE70287113D00020002313700B705D
:104E6000237005B0F0BD2F703070277005F0A6FFDD
:104E70000028CBD12378042BF3D90B490B4AD9E76F
:104E80000C480D4B00680390039E0C481E608DE893
:104E9000060001F01DFF2846FFF796FD01209DE862
:104EA0000600DAE788CEFF1F00C3FF1F90CDFF1F6B
:104EB00098CEFF1F60DEFF1F4CCAFF1FC0C2FF1F3E
:104EC00010B50C4A0C4B127819789142044607D061
:104ED00019210A481A7006F095FF094807F0E8FB07
:104EE000204608F0F9FC0749074C08F001FE206055
:104EF00010BD00BFCCA5FF1F35C2FF1F1801010068
:104F0000D0A7FF1F0000C84270B4FF1F2DE9F04773
:104F10004100BE4C01EB000804EBC808074698F8B6
:104F200015309BB3FCF7D6FF98F80A30C0B2834225
:104F30004FD0DFF80C9388F80A0099F80030002B66
:104F400047D0B34E0137002405E0013499F8003012
:104F5000E4B2A34246D9A2001319F118F35CBB4294
:104F6000F3D1487898F80A309842EED18B7891F8CE
:104F700003A0013B072BE8D8DFE813F0420039001B
:104F800036009E00B500D000DA00ED00B8F802301F
:104F9000B3F57A7F1FDA4FF47A752B46CA1904EB02
:104FA000C202907D5580012831D0022811D165219F
:104FB000A3F57A73974C107A01FB03F384FB03414A
:104FC000DB17C3EB2123C11A0029B8BF49420529C9
:104FD0005FDCBDE8F087B3F5FA6FA8BF4FF4FA6362
:104FE0009DB2DBE7BDE8F0878B4B1B7843B18B4B61
:104FF0001B7813F0F70FA8D00820FDF7DDFDA4E71C
:10500000874B1B78002BA0D0FDF728FE9DE7854835
:10501000007888B3A3F2DC5383EAE372A2EBE37275
:10502000814B120283FB0203D217C2EBA313DBB244
:10503000CA1904EBC202127AD21A002AB8BF52422D
:10504000032A7A4A127803DC9A42C2D9002302E08A
:105050009A4288BF00230F4404EBC704184623720A
:10506000FDF712FE237A724A1370002B40F0A080E5
:10507000704A1370BDE8F087D279A3F57A737AB1DC
:10508000644A1B0282FB0302DB17C3EB2223DBB261
:10509000CEE7DBB213721846BDE8F047FFF710BF4A
:1050A000A3EBC3135B4A5B0082FB0302DB17C3EB7A
:1050B0002223FF33DBB2BBE70AF1FF335E4AD15C48
:1050C00000297FF442AF01215046D154FDF764FF1F
:1050D00006215046FCF7C0FCBAF1010F7FF435AF52
:1050E000FCF7D2FF31E7131933441D79022D00F08C
:1050F000A980032D7AD0012D7FF427AF4F4B534465
:1051000013F8013C002B7FF420AF29465046FEF7F0
:1051100089F950460421FCF79FFC16E72244B51894
:1051200029794B1E022B48D95046FCF795FC0CE719
:1051300013193344197902294ED0032942D0012989
:105140007FF403AFBAF1140F3FF6FFAE50460022D2
:10515000FDF7E8FEF9E6131933441AF1FF301B7925
:1051600003F1FF3318BF0120082B3FF6EEAE01A27A
:1051700052F823F0AB5100004B4F00004B4F0000A2
:105180004B4F00004B4F00004B4F0000A55100005B
:105190009F51000099510000FFF7ACF8D5E6FFF7EA
:1051A0003DF8D2E6FEF798FFCFE6FEF747FFCCE6E4
:1051B000204B01221A70BDE8F0875046FDF70CFF26
:1051C0002979B1E7BAF1140F3FF6BFAE012250467C
:1051D0001146FDF7A7FEB8E6BAF1140F3FF6B5AEDB
:1051E000002250461146FDF79DFEAEE6134B534498
:1051F00013F8013C002B39D050460021FEF712F97C
:1052000050460221FCF728FC9FE600BF50B2FF1F6A
:10521000F4CCFF1F9F74784181C1FF1F82CEFF1F16
:1052200081CEFF1F8B9BFF1F41DDB320CCA0FF1F52
:1052300034C2FF1FD4C0FF1F70C3FF1F40CAFF1F2F
:1052400098B5FF1F0AF1FF33094AD25C002A3FF4E8
:105250007CAE084AD15C00297FF477AE5046FEF759
:10526000E1F829465046FCF7F7FB6EE601214DE7D1
:1052700040CAFF1F64C2FF1F2DE9F8433D4FDFF80E
:105280000491DFF804813C4607F160060025A3790C
:10529000E8B2A3B3A388A3F54872B2F5AF6F35D8CF
:1052A0006178E2686380012922615FD055D30229C9
:1052B0004ED000222F4BA2714FF0010E5978587E2C
:1052C000884208BF0EF1010E03F1180308BF5FFA10
:1052D0008EFE012908BF01229E42EFD197F861306E
:1052E000012B26D0BEF1050F2AD02ABB022388F855
:1052F000003099F800209A4201D0FCF775FD013585
:10530000052D04F11804C2D1BDE8F883E3682269D1
:1053100019499B1A8B42CCD9184B1B78A3B9184B4F
:105320001B78012B14BF0023022363700023237515
:10533000BFE7BEF1050F03D0012388F80030D8E79E
:105340007B7888F80030D4E7002DE8D16570EDE770
:105350000022012362702375ABE7237D0133DBB2AA
:10536000042B2375A5D901236370A2E7FFF7CEFDB7
:105370009FE700BF50B2FF1FA086010048CAFF1F71
:1053800043CAFF1F73C3FF1F8BCDFF1FF8B5154E18
:10539000154C164F172005F0A9F93278237893425F
:1053A000054614D03B68C31A002BB8BF5B424B2B99
:1053B0000CDD1B210E48227006F024FD0D4807F07D
:1053C00077F9227833789A4201D0F8BDF8BD2846A3
:1053D00008F086FA4FF06A5108F0D6FA064C3D60A4
:1053E0002060F8BD80C1FF1F35C2FF1FC8B2FF1F7C
:1053F00034010100D0A7FF1F70B4FF1F084B1B78BA
:10540000012B07D005D3032B08D801210E2005F06E
:1054100065BB70470021052005F060BB704700BFE9
:105420008F9BFF1F074B1978012907D005D303294C
:1054300007D800210E2005F051BB7047052005F06C
:105440004DBB70478F9BFF1F2DE9F04F83B00023AA
:105450000193FFF79BFFA54B93F8AC2222B993F879
:105460006C45002C00F0DD80A14B00211868012460
:105470008DF8044008F080F905469E4F97F8ACA2DD
:1054800097F86C35BAF1000F75D0002B40F06781AA
:105490004FF07E56984ADFF894B292F800900BF1E4
:1054A000100830469549B9F1000F00F0D48008F09B
:1054B00027FC9349934A60B9304608F003FC4FF04B
:1054C0008F41914A28B9304608F05EFA08F022FC74
:1054D0000246CBF800200BF1040BD845E1D1844BF8
:1054E0002846596801238DF8053008F045F9874BA7
:1054F0001B7801340546E4B2002B42D0844B1B7864
:10550000002B40F0828097F82C387A4A002B00F06C
:105510003C81774B2846996808F02EF94FF07E576A
:105520000546754B7B4E93F8009006F110084FF43A
:10553000803A38467149B9F1000F00F0918008F0C7
:10554000DFFB6F496F4B60B9384608F0BBFB4FF08B
:105550008F416D4B28B9384608F016FA08F0DAFB8F
:105560000346336004364645E3D101340123E4B2F7
:105570008DF806300EE0002B8AD1644B1B78002B8F
:10558000BCD197F82C385B4A002B4CD192F8EC3AFE
:10559000002B48D1604B93F8303053B1544B284620
:1055A000D96808F0E9F8013401230546E4B28DF822
:1055B00007305A4E5A4B3068196808F08DFB0028A6
:1055C00040F0CA80002C4ED1FFF718FF554C3568CB
:1055D00004F110064949284608F092FB4849494B16
:1055E00060B9284608F06EFB4FF08F41464B28B952
:1055F000284608F0C9F908F08DFB034644F8043F3B
:10560000A642E7D103B0BDE8F08F394B2846996830
:1056100008F0B2F8013401230546E4B28DF80630F3
:10562000B8E7002529E7BAF1000F0BD097F86C35E1
:1056300043B12F4B2846596808F09EF84FF07C572D
:1056400005466EE72A4B2846596808F095F84FF052
:105650007E57054665E74FF48033CBF800303AE7D4
:10566000C6F800A07EE7FFF7DDFE012CAED90021D1
:10567000284608F045FB00287CD04FF07E51284694
:1056800008F020FB00287DD11B4BD6F8009093F842
:1056900000A0254E164F01AC0DF1080814F8013B8F
:1056A00003B3BAF1000F43D03968484608F06CF9EB
:1056B000294608F01DFA1149834608F021FB98B9E4
:1056C0000F49584608F0FEFA00284BD00E483060CB
:1056D000444506F1040607F1040793D014F8013B92
:1056E000002BDED13360F3E70648F0E708C4FF1F64
:1056F000C4A4FF1F9CB5FF1FFCB4FF1F00FEFF46A4
:1057000000FEFFC60000FF7F0000018001C3FF1FF5
:1057100081C1FF1FE4B2FF1F60B5FF1F70B4FF1F00
:105720008CCEFF1F4CB4FF1F50B4FF1F24CEFF1FB1
:105730001949484608F0E4FA0028D5D117494846E7
:1057400008F0C0FA0028C1D14FF08F41484608F058
:105750001BF908F0DFFABAE7FFF750FE85E74FF0D4
:105760007C5697E64FF08F41584608F00DF908F047
:10577000D1FAACE70A4B9861D8611862586203B05D
:10578000BDE8F08F4FF07E557EE792F8EC3A002BA3
:105790007FF4BFAEFEE600BF00FEFF4600FEFFC680
:1057A00038B4FF1F594B70B500221A60FFF74CFE4A
:1057B000FFF724FE5648574CFEF742F85648FEF7CE
:1057C0003FF804F1780520461834FEF739F8A54271
:1057D000F9D15248524CFEF733F804F178052046CF
:1057E0001834FEF72DF8A542F9D14E4C4E4E04F177
:1057F000F0052046FEF724F8183410B13378013351
:105800003370A542F5D1494C04F17805204618348F
:10581000FEF716F8A542F9D14548464C464EFEF72C
:105820000FF84648FEF70CF804F1F0052046FEF7A5
:1058300007F8183410B1337801333370A542F5D12D
:105840003F48404CFDF7FCFF04F5647520461834D2
:10585000FDF7F6FFA542F9D13B4C04F1780520464F
:105860001834FDF7EDFFA542F9D1384C04F5F07579
:1058700020461834FDF7E4FFA542F9D1344C04F575
:10588000F07520461834FDF7DBFFA542F9D1314C05
:1058900004F5F07520461834FDF7D2FFA542F9D182
:1058A00000212D4B0A4683F8BC1201310024042943
:1058B00083F8AC2283F8AD2283F8AE2283F8AF22BE
:1058C000A3F8BA2283F8B82283F8BE42204603F533
:1058D0003073E8D1214B012283F8BC0283F8BE0269
:1058E00083F87E0583F87C2583F8AC4283F8AD020B
:1058F000A3F8BA4283F8B80283F86C0583F86D0503
:10590000A3F87A4583F8780570BD00BF70B4FF1F17
:1059100090A4FF1F9C9BFF1FE499FF1FACA4FF1FD7
:10592000049AFF1F809AFF1F54C3FF1F189CFF1F7C
:10593000709BFF1FDCA4FF1F94CEFF1FB4A0FF1FAE
:1059400024A0FF1F909CFF1F3CA0FF1F0098FF1F7B
:10595000D0A0FF1FB0A2FF1F9CB5FF1F08C4FF1FF0
:10596000F0B541F2883091B005F0B2F9022106207D
:1059700005F0C8F80221092005F0C4F80A2005F056
:10598000E9F8062005F0B0F8002800F03081AE4BB1
:10599000AE4AAF4FAF4CB04D1A6001260E220F2316
:1059A0000021AE4822702B703E7001F0B5FF32200E
:1059B00005F0D0F83146052005F0A4F80520314661
:1059C00005F08CF80A2005F0C5F80C21A44806F073
:1059D0001DFBFFF739FDA34B2A7883F860201220C6
:1059E000112110221325187683F8301083F84820EF
:1059F0001D70FCF747F9FCF76BF9002215219A4856
:105A000001F056F900221421984801F051F90022C2
:105A10000521974801F04CF900220421954801F036
:105A200047F900220321944801F042F9012108209E
:105A300005F068F80821914801F03AFB022117208F
:105A400005F060F80B218E4802F00EFE0C218C4808
:105A500002F052FE0D218A4802F092FE01212078C8
:105A600005F050F82078012105F038F8207803F08F
:105A7000FBFDF0B92822834D7B48114601F0DCF98B
:105A80002B680193019C2E46774801F025FA2B687C
:105A90000293029B1B1BB3F57A7FF5D936217A4816
:105AA00006F0B0F9794806F003FE33680393039CCF
:105AB000EAE7774C4FF4FA7005F04CF8FFF772FE06
:105AC0002378002B40F0B380FBF7EAF9FBF71EFACE
:105AD000704B03F5F07101E08B4203D05A7B183311
:105AE000002AF9D06C496D4B0A7003F5F07101E0A2
:105AF0008B4203D05A7B1833002AF9D06849694B8E
:105B0000694C0A7000221A705A709A70FCF770FB88
:105B100094F84130032B03D804F11C0003F09CFDE2
:105B200003A8A27E604903F0FFFA9DF81050059883
:105B30009DF818105D4B84F8205010AA079D6062F4
:105B400084F828100898099912F80F6DE56220630F
:105B50000A9D0B9861639DF8301084F84160A5633D
:105B600003F10D06E06384F8401012F8011F03F8FA
:105B7000011BB3424C4CF8D103A803F037FD94F855
:105B80004130032B40F2A28001230A214848E376EA
:105B900006F038F9474B1C68204609F0B1F9014678
:105BA000204606F02FF91021434806F02BF937481C
:105BB00006F07EFD4149424A424C4FF480330E20AC
:105BC000A361E361236263628B61CB610B624B6211
:105BD0009361D3611362536204F088FD06F0D0FE36
:105BE000214801F043F9FAF769FC11B0F0BD092032
:105BF00004F07AFF164B18B302221A70124B324A85
:105C0000144C154D1A600A260F2301210E20237013
:105C10002E7004F077FF01210E2004F05FFF304664
:105C200004F098FF02210D4801F076FECDE6FBF767
:105C300047FA2378002B3FF447AFFBF777FA43E7A7
:105C400003221A70DAE700BF8CCEFF1F0AD7A33CED
:105C50008F9BFF1F909BFF1FA8A4FF1F24CAFF1F3D
:105C60000082FF1F50B2FF1FC8B4FF1FC0C2FF1F3A
:105C70008CC9FF1FB8C9FF1FE4C9FF1F64CAFF1FFB
:105C8000D0A5FF1F60DEFF1F50010100D0A7FF1F3E
:105C9000E299FF1FD0A0FF1F80CEFF1FB0A2FF1F01
:105CA000B8C2FF1F40CAFF1FB4CDFF1FF6CDFF1FB4
:105CB00088010100949BFF1F940101000CCEFF1F7F
:105CC000CCB2FF1FB0CEFF1FA69BC43B00235022C7
:105CD0002449E376204600F071FD68B3224B01228F
:105CE0001A70FCF767FBFBF7D5F922211F4806F075
:105CF00089F81F4806F0DCFC16211E4806F082F8E1
:105D00001B4806F0D5FCFBF7C5F9FBF769FAFBF772
:105D1000BDFAFBF71BFBFBF755FBFBF7C7FBFBF7DC
:105D200049FCFBF7E1FDFBF72FFA114806F0C0FC38
:105D30000F4806F0BDFC3DE70A210F4806F062F867
:105D4000204609F0DDF80146204606F05BF80D21FB
:105D50000A4806F057F80122E17E204600F02CFFA9
:105D600028E700BFB8C3FF1FF4B4FF1FB80101004C
:105D7000D0A7FF1FDC01010088010100A80101007C
:105D800030B55D4C2378012B83B05CD04AD3022B15
:105D90005A4D31D05A4801F043FA5A4801F09CF864
:105DA000594801F099F8594801F096F8584801F01F
:105DB00093F8584801F090F8FFF746FB2B783BB179
:105DC000554B1A78002A4CD0FEF74EFD03B030BD7B
:105DD000514A117800295AD1FDF720FEFDF7FAFE4D
:105DE0004E4B1B78002B49D1FEF70AF8FEF7B8FAA4
:105DF000FDF708FD03B030BD2B78002B54D042488E
:105E000000F0A8FF0028C5D1454B464A1B68009307
:105E1000009B12689B1AB3F57A7FBBD93A4801F010
:105E200025F8B7E7FEF7E8FFFFF726FA3E4B1B78A9
:105E3000012B3CD03B4B1B68002B44D12378002B1B
:105E400039D12E4DA6E7FFF717FA354B374A1B68B5
:105E50000193019B12689B1A642BF2D9FBF7EEFFAA
:105E6000EFE7012227481A7000F098FF264800F05B
:105E700095FFFDF73BFDFEF777FCA5E7FCF7DAFFA2
:105E8000FDF7BEFFFEF76CFAFDF7BCFCB2E7284851
:105E9000137001F0BBFDFEF78FFC2378002B9BD124
:105EA000184800F0E3FF97E7FEF7A6FFA7E7214AAF
:105EB0002370137893B91348104D00F06FFF124808
:105EC00000F006FF66E702232370FBF72DFF194B56
:105ED0001B78002BB2D01921174801E01748152173
:105EE00005F090FF164806F0E3FB154806F0E0FBCE
:105EF000134806F0DDFBA1E743CAFF1F48CAFF1F96
:105F00000CB3FF1FC8B4FF1FC0C2FF1F8CC9FF1F07
:105F1000B8C9FF1FE4C9FF1FFEB4FF1F01C3FF1F65
:105F200060DEFF1F4CCAFF1F8BCDFF1FD4C1FF1FB8
:105F30009CB5FF1FE299FF1F0C020100F401010054
:105F4000D0A7FF1F2DE9F04F7148DFF81C92714E6A
:105F5000DFF818B28BB001F037F96F4B6F48196852
:105F600000231A4600F0AEFB6D4A6E496B4807F0FD
:105F700017FF6D48FAF766FF6C48FAF763FF6C4845
:105F8000FAF760FF6B48FAF75DFF654A6A4900203F
:105F900007F006FF6948FAF755FF6948FAF752FF1C
:105FA0005F4A6849002007F0FBFED9F80020C6F8D8
:105FB00000B00023737233613372F3600AB961E396
:105FC0001A465369002BFBD1566100245E4F5F4B8C
:105FD00050487461B480F480B472B461F461346286
:105FE000B484DFF88CA133604FF0FF3502F028F95C
:105FF00007F1240201213846FAF7FCFE07F14C02B2
:106000000121C7F800A0BD6107F12800FAF7F2FEF0
:106010004F4BC7F828A003F12402184601213D6424
:10602000FAF7E8FE4A4BDFF84C81C3F800A003F111
:106030004C029D6103F128000121FAF7DBFE454B7C
:1060400003F128021846424B0421C3F828A01D641E
:10605000FAF7D0FE404B414D03F1280218463D4B64
:106060004FF4803A0421C3F80080C3F818A0C3F8A5
:106070001CA0C3F820A0C3F824A0FAF7BBFE384B3D
:1060800003F128021846344B0421C3F80080C3F8FA
:1060900018A0C3F81CA0C3F820A0C3F824A0FAF7E6
:1060A000A9FE304B03F1280218462D4B0421C3F8FA
:1060B0000080C3F818A0C3F81CA0C3F820A0C3F840
:1060C00024A0FAF797FE27492C72012005F1180247
:1060D0002346C1F80080C1F818A0C1F81CA0C1F87F
:1060E00020A0C1F824A0EC602146C5F800B0687279
:1060F0002A612C4600E0226942F823106A7A174888
:1061000001339A42F7DCD9F80020174BAABBBCE256
:106110000CB3FF1F60B5FF1F949BFF1FB4CDFF1F83
:10612000FC97FF1F016700009CB5FF1F5CB8FF1FB5
:106130001CBBFF1FDCBDFF1F9504000008C4FF1F30
:10614000C8C6FF1F6D04000074B4FF1F5405010092
:1061500084C1FF1FB0CEFF1F0CCEFF1F24CAFF1F3C
:10616000CCB2FF1F38B4FF1FF8DFFF1F38F7000065
:1061700024050100300501001A465369002BFBD1AC
:1061800055610024DFF8ACA3DD4B6C61AC80EC8082
:10619000AC72DC482B6001F017FBDB4BCAF8003017
:1061A00050468AF80840CAF804708AF80940CAF8CC
:1061B0000C408AF8104006F01FF8D44AD449DFF8A2
:1061C00078B3DFF87893DFF87883504607F0E8FD7E
:1061D000CD4B8BF809408BE8880058464FF00103FF
:1061E000CBF80C408BF810408BF8083006F004F820
:1061F000C54BC64AC649584603F5307A07F0D0FD6C
:10620000C44BC9F804304846C9F800A089F80840D2
:1062100089F80940C9F80C4089F8104005F0ECFFF6
:10622000BA4ABB49DFF81CB3484607F0B9FDB94B81
:10623000DFF81493C8F8043040464FF0010388F8A3
:106240000830C8F800A088F80940C8F80C4088F861
:10625000104005F0D1FFAD4AAD49DFF8F0A240464D
:1062600007F09EFDAC4BC9F80430484689F8084059
:10627000C9F8007089F80940C9F80C4089F8104045
:1062800005F0BAFFA14AA249DFF8C482A34F4846ED
:1062900007F086FD9F4BCAF800309F4BCAF80430C8
:1062A00050464FF001038AF809308AF80840CAF8CE
:1062B0000C408AF8104005F09FFF944A9449DFF89B
:1062C0009492504607F06CFD954BC8F80430404658
:1062D00088F8084088F80940C8F80C4088F8104051
:1062E000C8F8007005F088FF884A8949DFF868A27D
:1062F000404607F055FD8A4BC9F8043048464FF038
:10630000010389F8083089F80930C9F80070C9F824
:106310000C4089F8104005F06FFF7D497B4ADFF89B
:106320003C82484607F03CFD07F530790223584689
:106330007B4A8BF80930CBF80090CBF804208BF81F
:106340000840CBF80C408BF81040019305F054FF47
:106350006E4A6F49584607F023FD714BCAF8043066
:1063600050464FF001034FF0030B8AF80830CAF88B
:106370000090CAF80C408AF810408AF809B005F07D
:106380003BFF624A6249DFF8D891504607F008FDAA
:1063900007F5B06A634BC8F804304046C8F800A05F
:1063A00088F8084088F80940C8F80C4088F8104080
:1063B00005F022FF554A5649404607F0F1FC594B7B
:1063C000DFF8A081C9F8043048464FF0010389F88E
:1063D0000830C9F800A089F80940C9F80C4089F8CC
:1063E000104005F009FF494A4949DFF87CA14846B9
:1063F00007F0D6FCDFF8749188F8084007F50467C9
:106400004046C8F8007088F80940C8F80C4088F881
:106410001040C8F8049005F0EFFE3C4A3C49404665
:1064200007F0BEFC4FF001035046DFF844818AF8C4
:106430000830CAF80070CAF804908AF80940CAF80F
:106440000C408AF8104005F0D7FE304A3049364FEC
:10645000504607F0A5FCA9F128034046C8F80030D3
:10646000324BDFF810A1C8F8043088F8084088F8EB
:106470000940C8F80C4088F8104005F0BDFE234ADA
:106480002349404607F08CFC284BCAF8043050469C
:106490004FF00103DFF8E0808AF80930CAF8009075
:1064A0008AF80840CAF80C408AF8104005F0A4FEAB
:1064B000164A1749DFF8C490504607F071FC164B96
:1064C000C8F8003040461A4BC8F8043088F8084035
:1064D00088F80940C8F80C4088F8104005F08CFE98
:1064E0000A4A0B49DFF898A0404607F059FC4FF0E4
:1064F00001037B720A4B3B6038460D4B7B6041E0E9
:106500003C05010024CAFF1F08C4FF1FFC97FF1FA2
:10651000AD0500009CB4FF1FB0CEFF1F9CB5FF1F50
:106520000CCEFF1F84C1FF1F9CCDFF1FCCB2FF1FED
:1065300038B4FF1FACC0FF1FC0C0FF1F5CC3FF1FEC
:10654000D8C0FF1FECC2FF1FECC0FF1F50CAFF1FC7
:1065500000C1FF1F14C1FF1F98CCFF1FACCCFF1F51
:106560002CC1FF1FD8CCFF1F40C1FF1FACC1FF1FB4
:1065700054C1FF1F8CC3FF1FC0CCFF1F4CCEFF1F99
:106580006CC1FF1F3C72FC603C7405F035FE404A54
:106590004049DFF82C81384607F002FC019B8AF85D
:1065A00009303D4BCAF8003050463C4BCAF8043025
:1065B0008AF80840CAF80C408AF8104005F01CFE22
:1065C000334A3449504607F0EBFB344BC9F80430EA
:1065D0004846C9F8006089F80840C9F80C4089F8B5
:1065E000104089F809B005F007FE294A29494846B4
:1065F00007F0D6FB294B88F80840404688E8280079
:1066000088F80940C8F80C4088F8104005F0F4FDFF
:106610001F4A2049224D234C404607F0C1FB224A25
:10662000224813680693DDF818C013680793DDF855
:106630001CE013680893089F13681D49099380E8BC
:1066400000501C4B2D78099E25700F604E6003F1A1
:10665000840511680491049811680591059943F81F
:106660002C0C43F8281C2C33AB420F4CF1D11248B0
:1066700000F0A2FC23680393039A104B1A600BB03E
:10668000BDE8F08FC9F800609FE4186079E500BFAD
:10669000FC97FF1FAD050000CCB2FF1F38B4FF1FF1
:1066A00080C1FF1F35C2FF1F60DEFF1FC8B4FF1F80
:1066B000C0C2FF1FB8C9FF1F64CAFF1F44CEFF1F1F
:1066C0006CCEFF1FF8B50D4604461C3017461E461B
:1066D00002F07AFF284608F013FC1A2806D9002396
:1066E0002370A77684F850602046F8BD421C2946E6
:1066F000204603F04FFEA77684F850602046F8BD90
:1067000010B504461C3002F071FF204610BD00BFDA
:106710002DE9F04190F82550032D02D90220BDE863
:10672000F081022A02D80320BDE8F0810F461968E3
:1067300004461E46154602F063FF10B90420BDE86A
:10674000F0812A463946204602F052FF804618B9A9
:1067500038700720BDE8F081013D3A46002306E08D
:106760000D2928D00133984516D0AB4214D01178AA
:106770000A29964602F10102F2D10D245A1C00208A
:106780008EF80000BD5C3168A54218BF1A46013181
:106790000A443260BDE8F081236820461B699847AF
:1067A00020B907F808000720BDE8F08100237B55D9
:1067B0000320BDE8F0810A24E0E700BF2DE9F041A5
:1067C00082B002AC002344F8043D80460F461646D2
:1067D00000F11C052346324639462846FFF798FF4C
:1067E0000028F7D0072805D088F81B00002002B049
:1067F000BDE8F0810023012088F81B3002B0BDE81D
:10680000F08100BF70B5054608F07AFB01382C18FE
:106810000AD2002603E004F80169A54204D82078D2
:1068200007F000FB0028F6D170BD00BF2DE9F0474E
:1068300080461C468A46914619461C300A9B089A97
:10684000FFF766FF074638B1072805D0012488F80E
:106850001B002046BDE8F0872578284626460134EF
:1068600007F0E0FA0028F7D13B2D19D0232D17D0DF
:10687000BAF1000F01D05B2D18D03D21304608F051
:1068800003F9054660B1002303703046FFF7BAFFF5
:1068900098F85040494630467CB108F065F9B8B1E7
:1068A000072F03D000242046BDE8F08706230124EB
:1068B00088F81B302046BDE8F08708F0C1F80028B2
:1068C000EED1099B01351D6088F81B400124EAE7E1
:1068D000099B01351D6088F81B00E4E72DE9F843AA
:1068E000804629B3144689461A462146089B1C3027
:1068F000FFF70EFF074630B1072804D088F81B00C9
:106900000120BDE8F883264614F8015B284607F00D
:1069100089FA0028F7D13B2D08D0232D06D05B2D16
:106920000CD0072F04D00020BDE8F883052FFAD142
:10693000052388F81B300120BDE8F8830136344672
:106940000136207807F06EFA05460028F7D15D2160
:10695000204608F099F80028E3D005702046FFF79C
:1069600051FF98F85030494620464BB908F068F876
:106970000028D6D1002388F81B300120BDE8F88319
:1069800008F0F2F80028CCD1F4E700BFF0B587B0EA
:1069900007460D9C2679012E1D461AD00FD3022ED4
:1069A00008D196460AB11678FEB90623FB76012077
:1069B00007B0F0BD0823C376012007B0F0BD002961
:1069C0004FF000000CBF022301232371206007B0A9
:1069D000F0BD1A4600940C9BFFF780FF68B1F87E6B
:1069E0000028E4D102232371E7E702940C9C05AE52
:1069F0008DE85000FFF71AFF10B9002007B0F0BD76
:106A0000FB7E002BD3D1059C26460134307807F05D
:106A100009FA0028F8D130460596FFF7F3FE059BEA
:106A20001A7842B10133059313F8012C05F8012BB4
:106A30001A78002AF6D100232B70B8E72DE9F04729
:106A400084B00025DDF830A002950446884617463C
:106A50001E468DF80C500DF1080906E0CDF80490A3
:106A6000CDF800A0FFF792FF68B994F84150032DCC
:106A700033463A4641462046F0D90223E3760020C9
:106A800004B0BDE8F087E07EB0FA80F04009F7E797
:106A900030B583B01D46069C0094FFF7CFFF044637
:106AA000F0B11749284607F0CBFFE0B11549284659
:106AB00007F0C6FFB8B11449284607F0C1FF90B1EE
:106AC0001249284607F0BCFF98B11149284607F043
:106AD000B7FF70B128460F4907F0B2FF48B1002454
:106AE000204603B030BD079A01232046137003B03F
:106AF00030BD079A00232046137003B030BD00BF9D
:106B000058020100600201006402010068020100F5
:106B1000700201007402010030B583B01D46069C6E
:106B20000094FFF78BFF044620B1284607F03EF99A
:106B3000079B1870204603B030BD00BF30B583B04E
:106B40001D46069C0094FFF779FF044620B12846B5
:106B500007F030F9079B1860204603B030BD00BF36
:106B600010B584B0069C009403AC0194FFF7E6FFD7
:106B700010B1079A039B138004B010BD30B585B0E7
:106B80001D46089C0094FFF759FF18B900242046C1
:106B900005B030BD04460A2203A9284608F0B8FB18
:106BA000039B9D42F2D01B78002BEFD1099B18600C
:106BB000204605B030BD00BF10B5144608293AD8AC
:106BC000DFE801F00B342A2F161B202505000D21CC
:106BD0001B4805F017F934B910BD0821194805F014
:106BE00011F9002CF8D01848BDE8104005F060BD40
:106BF0000A21164805F006F9EDE71121144805F0C1
:106C000001F9E8E70D21134805F0FCF8E3E70B2153
:106C1000114805F0F7F8DEE70D21104805F0F2F80D
:106C2000D9E710210E4805F0EDF8D4E70E210D4804
:106C300005F0E8F8CFE713210B4805F0E3F8CAE7C1
:106C4000F402010078020100D0A7FF1FB802010082
:106C5000C4020100D8020100E80201009402010010
:106C6000A4020100840201000403010008B5C37AF4
:106C7000807A2BB903F038FF003018BF012008BD1F
:106C800003F032FFB0FA80F0400908BDC37A807A81
:106C900013B9012103F022BF002103F01FBF00BF81
:106CA000C17A807A09B903F019BF012103F016BF38
:106CB00010B50446C27281720846012103F022FF1A
:106CC0002046FFF7EDFF00236373237310BD00BF61
:106CD00010B5037B82B0044663B1FFF7E1FF084BB8
:106CE0001B680193019B2360002323736373A373C9
:106CF000238223812046FFF7C9FF02B010BD00BFE9
:106D000060DEFF1F10B5037B82B0044663B1FFF75E
:106D1000C7FF084B1B680193019B2360002323736B
:106D20006373A373238223812046FFF7B9FF02B068
:106D300010BD00BF60DEFF1F10B5847A204603F04F
:106D4000D3FEB0FA80F149092046BDE8104003F0B7
:106D5000C5BE00BF007B7047F0B50D4E028283B008
:106D600033680193490000230139019F0373012512
:106D7000437303818173076085740446FFF786FFC0
:106D800033680093009B2573236003B0F0BD00BF00
:106D900060DEFF1F0A460121FFF7DEBF10B582B09B
:106DA0000446FFF77DFF064B1B680193019B2360A0
:106DB000002323736373A3732382238102B010BD66
:106DC00060DEFF1F84B02DE9F04182B009AC84E899
:106DD0000E00DFF860809DF83CE0D8F800300093AA
:106DE00005460FCC009E2E60002705F114062F7378
:106DF0006F732F81AF740FC694E8030046F8040B3D
:106E0000BEF10A0FAB8A318028BF4FF00A0E2B82E9
:106E1000284685F80EE0FFF739FFD8F800300193D7
:106E2000019B2B6001232B7302B0BDE8F04104B03D
:106E3000704700BF60DEFF1F30B58BB001238DF8B7
:106E400024300AABADF81010ADF81220044613E957
:106E5000070002256B46039503C304A91A80204648
:106E60000EC9FFF7AFFF0BB030BD00BF30B58BB020
:106E700001238DF824300AAB044613E907000225EC
:106E80006B46039503C340F2EE21ADF81010ADF848
:106E9000121004A91A8020460EC9FFF793FF0BB009
:106EA00030BD00BF30B58BB001238DF824300AAB64
:106EB000044613E9070002256B46039503C3282106
:106EC000ADF81010ADF8121004A91A8020460EC9B2
:106ED000FFF778FF0BB030BD70B5038988B004466A
:106EE000ABB1344D41682A680092009A521A93421D
:106EF0000DD2FFF7D5FE2B680193019B2360002381
:106F000023736373A3732382238108B070BD238A24
:106F1000002BFAD0274D21682A680292029A521A51
:106F20009342F2D2637BA27B0133DBB29A4263735A
:106F300014D9DB07204622D4FFF7A8FEA67C002E3A
:106F40002CD1637B0A2B2ED82A68049204EB4303CE
:106F5000049A9B8A2382226008B070BD94F828604E
:106F600086B92046FFF79CFE2B680793079B267384
:106F70006673A67326822681236008B070BDFFF772
:106F80008FFEDBE7A38A2382002363732046FFF78B
:106F90007DFE2B680693069B2360B6E72B6805935E
:106FA000059B2360B1E72046FFF77AFE2B68039329
:106FB000039BDCE760DEFF1F70B40F4E00233588B3
:106FC00003710C21012215424FEA42040AD00379D1
:106FD000013903F10103A2B20371F4D1FF2303715C
:106FE00070BC704705490B88154323EA02023580BF
:106FF0000A8070BC704700BFF2CEFF1FE8CEFF1FB3
:10700000F8B504790B2C01D92046F8BD0646CCB260
:10701000204601211F46154603F074FD1A4A3079B7
:107020001A4913880C544FF0010E194C0EFA00F156
:107030000B4321681380174BED00FF0042F6E0621E
:1070400011EA0E013580778023F8102015D12368CE
:107050001148124A124F134D43EA0E03236003787E
:10706000114C43F080030370032311603B60452102
:107070002023C5F800E0116023700C4B4FF4001280
:107080001A6034792046F8BDE8CEFF1F0CCFFF1FF1
:1070900038800440F4CEFF1F00500640000004403A
:1070A000040004400800044055E400E008E100E06A
:1070B0004FF416634FF40872FFF7A2BF0388C900AC
:1070C000994203DB43888B42A8BF0B4602790B2A07
:1070D0009CBF024921F81230704700BFF4CEFF1F59
:1070E000F8B5304E304D96F900202B881341DC075F
:1070F00050D42E4C94F900300B2B0EDC298841FA29
:1071000003F2D00702D52CE0D20729D401335BB2B9
:107110000C2B41FA03F2F7D1237025480268C2F51F
:107120001C3101F58071B1F5487F16DB4EF6602306
:107130008B42A8BF0B461A441E4902600E681E4DC2
:107140001E4A1B4F3344C5260B602E6003689342D2
:1071500002D900233B602370F8BD4FF44873EAE77F
:107160002370174A0121D05C03F0B8FC94F9003079
:107170000F4A14490F4831F81350116833702944ED
:10718000116002680C492A440133C52502600D6074
:107190002370F8BD0A4B0021985C03F09FFC0C2380
:1071A0003370A6E7CDA5FF1FE8CEFF1FF0CEFF1F6F
:1071B000ECCEFF1F0800044000000440FF700200F6
:1071C0000CCFFF1FF4CEFF1FF0B5144B83B01B682C
:1071D00001938446012300220198CCF824310CF15C
:1071E000C7070CF12406ACF104050CF19C040CF16A
:1071F000F801134601320A2A07F8013F4FF0000E4A
:1072000046F8043F45F8040F44F8043F41F8043FB2
:10721000F0D16046CCF828E103B0F0BD60DEFF1F7E
:107220002DE9F047434B82B01B68019300F1D00673
:107230000746DDF804C0314600F1240300F1C8041C
:1072400000F1F8054FF0000E4FF001084FF0020971
:1072500005E0C1F80080A94204F1010426D053F8EA
:10726000042F41F804EF002AF5D053F8280C9A6A4D
:10727000C0EB0C0A92450244EDD3207843F8282C49
:107280000028E8D01A6D002AE3D0986F824200F1FE
:10729000010AE0DD5245C1F80080C3F878A0D8BFEC
:1072A000C1F80090A94204F10104D8D107F12804E3
:1072B00007F150084FF0000956F8043F012B19D090
:1072C000022B11D123689847D7F828E1BEF1000FAF
:1072D0000AD0D4F8D4002A46002352F8041F88426A
:1072E0000ED001330A2BF8D104344445E4D102B066
:1072F000BDE8F0872368043498474445DCD1F6E7BD
:1073000007EB83018A6A002AEED03B4404340EF175
:10731000FF324445C1F8289083F8C890C1F8D49052
:10732000C1F85090C1F8A090C1F8FC90C7F828218E
:10733000C2D1DCE760DEFF1FF0B5D0F82871092F5D
:1073400083B008DC00F12405002455F8046F3EB139
:1073500001340A2CF9D14FF0FF32104603B0F0BDD2
:10736000002AF8D00F4D2D68019500EB840500EB45
:10737000040E2965019EAB670121AA628EF8C81030
:1073800040F82460D0F82421C5F8FC205318002BC5
:107390000F44D8BF0B46C0F82871C0F824311046FE
:1073A00003B0F0BD60DEFF1F0123FFF7C5BF00BFC4
:1073B00030B4D0F828514DB100F1F802002352F852
:1073C000044FA14204D001330A2BF8D130BC7047DE
:1073D00000EB8302916A0029F8D003440021013DAB
:1073E000916283F8C810C2F8D4101165C2F8A010D9
:1073F000C2F8FC10C0F8285130BC704710B400F13E
:10740000F80283B0002352F8044FA14205D00133A3
:107410000A2BF8D103B010BC7047044A12680192DD
:10742000019A40F8232003B010BC704760DEFF1FB4
:1074300010B400F1F802002352F8044FA14205D025
:1074400001330A2BF8D1002010BC7047034410BC54
:1074500093F8C800704700BF2DE9F84F8469002CED
:1074600040D0631C06464FF0000147D004F0A2FE56
:10747000834600283BD0D6F81CE096F82050274FD2
:1074800002300BF5817804E0964534D2744480458F
:107490001DD0230E5A1C37F9139037F9121030F90A
:1074A000022FC4F30F2ACAF5803309FB03F30AFB4A
:1074B00001331B1402FB03F3DB13E2430380002DB3
:1074C000E2D1A64515D28045CEEB0404E1D1304689
:1074D000B4610022594604F047FE5846BDE8F84F13
:1074E00004F018BE214604F059FE0028F6D1BDE88C
:1074F000F88F2C46CBE74FF0FF34C8E704F04EFE80
:1075000004460028F3D030462146002204F02CFE29
:107510002046BDE8F84F04F0FDBD00BF1803010090
:1075200072B683694BB1013304BF6FF0010383610D
:10753000C16180F8202062B6704701238361C16178
:1075400080F8202062B6704710B5044604F084FF2E
:10755000204610BD024A0349034806F021BC00BF83
:10756000FC97FF1F4975000018CFFF1F38B5074D66
:10757000074C08482A46214606F012FC2A462146B6
:107580000548BDE8384006F00BBC00BFFC97FF1F64
:107590004975000020CFFF1F28CFFF1F024A034973
:1075A000034806F0FDBB00BFFC97FF1F49750000B4
:1075B00030CFFF1F024A0349034806F0F1BB00BF6A
:1075C000FC97FF1F4975000038CFFF1F024A03498F
:1075D000034806F0E5BB00BFFC97FF1F497500009C
:1075E00040CFFF1F024A0349034806F0D9BB00BF42
:1075F000FC97FF1F4975000048CFFF1F2DE9F84396
:107600004FF00008064600F118054746414630464F
:10761000002F4FD004F0C2FDF0B12C68B4F5803FCC
:1076200007F1040100F1040E07F5827C27D05EF813
:10763000042B34FB02F334FB12F903F30F0209F3BA
:107640000F03C2EA03430A6893FA12F341F8043BBA
:107650008C45ECD804F05EFD08F10108B8F1040F88
:1076600005F10405D2D1002F40D030463946002222
:1076700004F07AFD3846BDE8F84304F04BBD07F14D
:107680000C0100F10C0451F8083C54F8082C93FA52
:1076900012F341F8083C54F8042C51F8043C93FAD6
:1076A00012F38C4541F8043C04F1080401F108018F
:1076B000E9D8CFE704F07EFD07460028CCD0286843
:1076C000B0F5803FC8D0391D07F582740B6830FBD8
:1076D00003F230FB13F302F30F0203F30F03C2EACA
:1076E000034341F8043B8C42F0D8B5E7BDE8F8838A
:1076F000024A0349034806F053BB00BFFC97FF1F33
:107700004975000050CFFF1F10B5002104F046FD61
:1077100070B172B60A4B1A6872B10A490C6844B16A
:107720001C60086062B61046BDE8104004F0F2BC70
:1077300010BD086062B610BD186062B610BD00BF13
:1077400068CFFF1F58CFFF1F38B5184B18491A686C
:10775000184C12681B79184D0B70A242286836BF6E
:107760002246A4F5807202F58074C0B1011D31F982
:10777000023B03F500431B1122F8023B9442F6D86A
:1077800004F0C8FC0D4B0022196829601A600C4BEC
:107790001B781BB10B4B4FF080421A6038BD4FF481
:1077A000006322F8023B9442FBD8F0E75CCFFF1F56
:1077B0001F800040308FFF1F68CFFF1F58CFFF1F73
:1077C00064CFFF1F08E200E0F8B501214248434EB4
:1077D00004F0DEFD424A43491368802043F480539D
:1077E00013600024087040F6080534800120083436
:1077F00003F0B0F9A3B2AB421CB2F6D13A4B1B680E
:107800005B0208D5394B1A6848F6A273134048F654
:10781000A27293424FD03449344A0B68344F354DED
:107820003548364C43F480030B604FF0010E40F2B4
:107830003F4648F6A37140F20113C7F800E02E60FE
:10784000116014600360244C2D4A236823491A6098
:1078500002259D802279196102F1804202F50432ED
:10786000284EDE6040F20111D9804FF48070002173
:107870000627B026D8829D60D88399829F8399611C
:107880001170167004F02AFD22791F4B1F4E1870DC
:1078900053119B0003F160431D4C327003F56143AB
:1078A00002F1100002F01F0701211A4D44F8205088
:1078B000B9401960F8BD0F4B1A6840F23F439A4235
:1078C000A9D10B4B1B68012BA5D10B4B1A6840F2B9
:1078D00001139A429FD1B6E75CCFFF1F00C00C4056
:1078E0002C80044021C00C403C80044000600340D8
:1078F0000C6003400460034010600340A28F01004D
:10790000308EFF1F00FEFFFF64CFFF1F1B80004073
:107910000092FF1F49770000044A137802290CBF28
:1079200003F0BF0343F040031370704721C00C40C5
:10793000024A0349034806F033BA00BFFC97FF1F11
:10794000497500005CCFFF1F024A0349034806F057
:1079500027BA00BFFC97FF1F497500006CCFFF1FBF
:10796000024A0349034806F01BBA00BFFC97FF1FF9
:107970004975000074CFFF1F024A0349034806F00F
:107980000FBA00BFFC97FF1F497500007CCFFF1F97
:10799000024A0349034806F003BA00BFFC97FF1FE1
:1079A0004975000084CFFF1F024A0349034806F0CF
:1079B000F7B900BFFC97FF1F497500008CCFFF1F70
:1079C000024A0349034806F0EBB900BFFC97FF1FCA
:1079D0004975000094CFFF1F38B50446D0F88000E9
:1079E0000D23002584F88F3284F89032656718B132
:1079F00004F090FBC4F88050D4F8840020B104F067
:107A000089FB0023C4F8843038BD00BF38B572B696
:107A100090F88F320D2B27D0044600230D22D0F88A
:107A20008000D4F88450C4F88030C4F8843084F8DE
:107A30008F2262B608B104F06DFB15B1284604F040
:107A400069FB04F1180001F007FE084A13882BB9FE
:107A50005E210748BDE8384000F0EEBD013B9BB217
:107A60001380002BF4D038BD62B638BD9CCFFF1F09
:107A7000D0A5FF1F70B5314D8EB00E460446FFF7FE
:107A8000C5FF5E212E4800F0C1FD2B8801332B80FD
:107A900072B60022314601A801F046FB9DF808109D
:107AA000039B9DF81060059821770EAA0699236222
:107AB000079B84F82460A062089E0998E162236312
:107AC0009DF8281012F80F3DA06384F83D306663DE
:107AD00084F83C1004F13E0304F14B0012F8011F3E
:107AE00003F8011B8342F9D101A801F07FFD62B6C2
:107AF00094F83D30032B09D92B88104AC3B95E2175
:107B00000F4800F099FD00200EB070BD0D2000233D
:107B10001421082284F890020120A4F88C32A4F8E1
:107B20008A3284F88E32616784F88F220EB070BD7D
:107B3000013B9BB21380002BE1D0E4E79CCFFF1FF9
:107B4000D0A5FF1FC36C9AB2012A01D00020704754
:107B5000026D4AF644418A4222D045F222618A42AD
:107B60001BD042F611318A42F0D10F4904221B0C7E
:107B7000012B04D0022BE9D1490842F00102B0F8F0
:107B80005A30082B04D0102BE0D1490842F00202F1
:107B9000C16780F890220120704704490422E6E77B
:107BA00003490022E3E700BF34EE35171AF79A0BBA
:107BB0008D7BCD052DE9F04FB0F88A6200F18A0780
:107BC00083B03E44E9B1DFF8CCB304460D464FF034
:107BD000080A4FF0000994F88F320D2B00F25F81F4
:107BE000DFE813F00F000F00D5009E000F000F001C
:107BF0000F000F001D0113004500710087000F00EA
:107C00006267002003B0BDE8F08F626F94F88E3297
:107C1000AA4204F14C0028BF2A4618443146904637
:107C200002F0B8FB94F88E12B4F88A22636F4144D4
:107C3000C8EB0303424484F88E12A4F88A226367D7
:107C40000193002BDDD12046FFF77CFF002800F0D8
:107C500026810A22019BC4F874A0C8EB050546449E
:107C600084F88E3284F88F22002DB4D1C9E7626F78
:107C700094F88E32AA4204F14C0028BF2A461844D8
:107C80003146904602F086FB94F88E12B4F88A22B0
:107C9000636F41444244C8EB030384F88E12A4F896
:107CA0008A226367002BACD1E16C226D6267594573
:107CB0004644C8EB050500F008810B2384F88F3299
:107CC000002D88D19DE7626FB4F88A329542C0F0EA
:107CD000578113440A21AD1AC4F874A0164484F8DD
:107CE0008E92A4F88A3284F88F12002D7FF473AF3D
:107CF00087E7626FB4F88A1295422B4628BF134675
:107D00001944D21AA4F88A127FF47AAFED1A1E44ED
:107D1000C4F874A084F88FA2002D7FF45CAF70E7E4
:107D2000636F94F891129D4228BF1D465A1B6267EB
:107D3000002900F0BD80D4F88010B4F88830E06CE1
:107D400001EB430C4FF0000EACF8040084F891E214
:107D5000D4F8840096F801C016F802EB00EB43005B
:107D600001339BB24EEA0C2E7F2BA4F88830A5F18C
:107D70000205A0F804E000F2E180002D40F09880B8
:107D8000002A00F09B8084F8915228463AE7636FFE
:107D9000D4F880109D4228BF1D46C5EB030C023667
:107DA000C4F874C003E00236002D00F0A680B4F8D9
:107DB000882016F8020C16F801EC531C9BB201EB5C
:107DC000420240EA0E207F2BA4F88830A5F102057C
:107DD0009080E8D90022204604F0C6F90122D4F8A8
:107DE0008010204604F0C0F9D4F8800004F092F925
:107DF000636FD4F884001D44F61B0023A4F88A6244
:107E00006567C4F8803010B104F084F9656F15B966
:107E10000D2384F88F32012003B0BDE8F08F626F2C
:107E200094F88E32AA4204F14C0028BF2A46184426
:107E30003146904602F0AEFA94F88E12B4F88A22D7
:107E4000636F41444244C8EB030384F88E12A4F8E4
:107E50008A226367002B7FF4D4AEE26C4C498A42DD
:107E60001DD1626DA1F57001A1F2FB718A4216D19C
:107E700001F15B41A26D01F5F11101F60F418A425A
:107E800030D00C23E26D84F88E3284F88F32C8EB48
:107E9000050546446267002D7FF49DAEB1E60D23D3
:107EA000002084F8903284F88F3203B0BDE8F08F60
:107EB000023D307896F801E024D17ABB0D230020F2
:107EC00084F88F3203B0BDE8F08F94F8901284F8F4
:107ED0009132CB0784F88F1227D4A267002D7FF44C
:107EE0007AAE8EE6E26DA2F110011829D7D80921E9
:107EF00084F88E3284F88F12C9E7BCF1000F7FF44A
:107F000080AEDBE7D4F88010B4F8883001EB430C86
:107F100040EA0E200236ACF8040019E73388E36427
:107F20000223284684F891326CE604F09FF8C4F8E6
:107F3000840000283FF465AE626FCEE70022204641
:107F400004F012F94FF00008D4F8800004F0E2F8D1
:107F50000122D4F88410C4F88080204604F004F98B
:107F6000D4F8840004F0D6F8606FC4F88480F61B5F
:107F70002844A4F88A62606700283FF449AF4AE7C2
:107F8000521B1D446267A4F88A5200203AE600BFE3
:107F9000524946466461746190F88F0207288CBF8D
:107FA00000200120704700BF90F88F32072B07D8C0
:107FB000836F426FC16F9B1AA3FB01231846704762
:107FC0000020704790F88F32072B05D8836FC26F5F
:107FD000A3FB0223184670470020704790F88F32A9
:107FE0000D2B00F0B6802DE9F041044604F03EF878
:107FF000C4F88000002800F09A8094F88F32072B94
:1080000040F297800023C4F88430B4F88C32B4F87E
:108010008A120022591A9142A4F8882005DD2046D0
:10802000FFF7C8FD002840F09B8094F88F320D2B9D
:1080300004F1180625D0304601F09AFA08B304F18D
:108040008A074FF000080FE0A4F88A8294F88F5254
:10805000FFF7B0FD94F88F32002866D10D2B10D0B9
:10806000072D1ED9072B1CD839464FF40072304615
:1080700001F0BEFA83B219462046A4F88C32002BD8
:10808000E2D1304601F0E8FA3A4A1388002B61D178
:108090005E21394800F0D0FA0D2384F8903284F83C
:1080A0008F32D4F8800000B3B4F88830C3B17F2B8E
:1080B00009D800EB4303023300F58175002223F851
:1080C000022FAB42FBD101460022204604F04CF8BF
:1080D00094F88F32072B01D8DB0743D5D4F8800002
:1080E00004F018F80023C4F88030D4F88400F0B10C
:1080F000B4F8883093B17F2B09D800EB43030233E7
:1081000000F58175002223F8022F9D42FBD1014624
:108110000122204604F028F8D4F8840003F0FAFF86
:108120000023C4F88430BDE8F0810D2BA9D0BDE850
:10813000F081DA077FF566AF03F098FFC4F884009A
:1081400000287FF462AFD4F88000BDE8F04103F06E
:10815000E1BF7047013B9BB21380002B98D09BE797
:10816000BDE8F0810122D4F88010204603F0FCFF26
:10817000B4E700BF9CCFFF1FD0A5FF1F90F83030A1
:1081800003B9704770B5054603F070FF0646002836
:1081900050D0EB69296A8B4227D901F5807293424E
:1081A00038D2A8695C1A22460844311D01F08EFDC0
:1081B0002B6AEA6A1919630822447F2B2962EA6252
:1081C00009D806EB4303023306F58171002223F838
:1081D000022F8B42FBD128463146002203F0C4FF18
:1081E0003046BDE8704003F095BF134A13885BB971
:1081F0005E21124800F020FA002385F83030304626
:10820000BDE8704003F086BF013B9BB21380002B9A
:10821000F2D1EDE7A8694FF480720844311D01F0F6
:1082200055FD2A6AEB6A02F5807203F580732A62B3
:10823000EB62D0E770BD00BF9CCFFF1FD0A5FF1F32
:10824000002380F830308362C362704710B4047F2B
:108250004160022CC26002D010BC04F017B98368E0
:1082600010BC18472DE9F0410468E56815F0807FDF
:10827000794D256052D1DF0740F1B380002900F02D
:10828000E3800D78012B18BF45F00045656301318F
:1082900090F8248003F1FF3C48EA0828BCF1000F65
:1082A00000F0A88021B14D7811F8028B45EA08282A
:1082B00045682E7ABCF1020F06F1FF364FEA06360A
:1082C0000CBF48F0805548F01045B6B26563ACF17C
:1082D000020C08E00AB114700132013B05F470454C
:1082E000B54216D90468E56A15F0F00FF6D0A46B14
:1082F00013F0010F17464FEA242EEBD11AB107F8FD
:1083000002EB54703A4605F47045B542A3F10203FE
:10831000E8D8BCF1000F6DD00468C3E7DD074CD589
:10832000002900F089800D78012B18BF45F0004529
:108330006563013103F1FF3E90F824C0BEF1000FE8
:1083400041D029B191F801C00D78023145EA0C2CD9
:1083500045682E7ABEF1020F06F1FF364FEA063667
:108360000CBF4CF080554CF01045B6B26563AEF1D1
:10837000020E08E00AB114700132013B05F47045A9
:10838000B54215D90468E56A15F0F00FF6D013F080
:10839000010F1746A46BEDD122B107F8024B24124E
:1083A00054703A4605F47045B542A3F10203E9D88A
:1083B000BEF1000F07D00468C3E79E4690F824C0C2
:1083C000BEF1000FBDD11BB30468E16A11F0F00FDC
:1083D000FBD0A16BDC071DD50AB111700132013B46
:1083E000F1E790F824809C4648EA0828BCF1000F89
:1083F0007FF458AF63B10468E16A11F0F00FFBD06D
:10840000DE07A16B0FD50AB111700132013BF1E714
:10841000BDE8F0812AB114460D1204F8021B557014
:108420002246023BCFE72AB114460D1204F8025B44
:1084300051702246023BDDE790F82450012B18BF13
:1084400045F00045656375E790F82450012B18BF8F
:1084500045F0004565631BE700041F80F0B4464B00
:10846000464A186BDC6A01791170454922790A7015
:108470009A6A00790870002A46D05968C9688A4209
:108480003ED82168CC8B240402F1FF3065D4C0F3C0
:108490000E00C883C88B80B2C882196B0968C88B6C
:1084A000000452D4C2F30E00C883C88B002480B2EB
:1084B00012F1FF32C88218BF01229C62D96A2E488D
:1084C00009680D6800F12404A54236D00068C4682C
:1084D00014F0804F0C680D6815BF2488247802358D
:1084E000013544F000440D604463196B254B097954
:1084F0001970214912B1CA6A12791A70F0BC70471A
:10850000521A9A620122D9E7586B196805681E4C05
:108510000A63CC62CC682D681C4E24F0804403278B
:10852000B542CC6083F825701FD1037F4260022BD7
:10853000C2601ED0F0BC03F0A9BF016890F824000F
:10854000CC6840F000404863CFE7CC8BC2F3080012
:1085500004F47E442043C883A7E7CC8BC0F3080013
:1085600004F47E442043C88394E72B461146F0BCB4
:1085700018478368F0BC1847D0A5FF1F1F80004034
:108580001C8000401B80004000000FFF4D82000057
:1085900090E80C00F0B41C6859682568164F174E17
:1085A00029432160164D17491760D6601561116087
:1085B000417A154A5C180A3194F8244053F8215046
:1085C00002EBC40149680D60017A5C1803EB81017C
:1085D000247ECD6902EBC40149680D60817A581888
:1085E00003EB810390F83000596B02EBC002F0BC42
:1085F00053681960704700BF01401F000110003828
:108600000110007800001F80840601005E2911D847
:1086100030B44A09C57A012303FA02F42C4300EB73
:108620008202C472D06801F01F0103FA01F1014314
:10863000D16030BC704700BF5E2913D830B44D09FB
:1086400000EB850401F01F01E368012202FA01F149
:1086500023EA0101E16021B9C37AAA4023EA0202B8
:10866000C27230BC704700BF204A43689A42F0B4DF
:108670000FD0427A1A4492F82420914207D093F8FE
:1086800024408C4215D093F825408C422AD0F0BC6F
:1086900070470B2907D00729EBD1154C227842F0FF
:1086A00001022270E5E7124C227822F001022270CA
:1086B000DFE7002421461E685D6836682E420FD031
:1086C0000C4D05EBC202002756685A18376092F825
:1086D000242005EBC2050A316A6853F82130136083
:1086E0004472D4E701242146E5E700BF58050100A4
:1086F0004CE0FF1F840601001E4A43689A42F0B412
:108700000CD0027A1A44127E914205D01C7E8C4213
:1087100014D05C7E8C422AD0F0BC70470C2907D064
:108720000829EED1144C227842F002022270E8E7C8
:10873000114C227822F002022270E2E70024214646
:108740001E685D6836682E420FD00C4D05EBC202E4
:10875000002756685A183760127E063105EBC205AD
:1087600003EB81036A685B6813600472D4E7012439
:108770002146E5E7580501004CE0FF1F8406010093
:10878000204A43689A42F0B40FD0827A1A4492F891
:108790003020914207D093F830408C4215D093F8A6
:1087A00031408C422BD0F0BC70470D2907D00E29E8
:1087B000EBD1154C227842F004022270E5E7124C0E
:1087C000227822F004022270DFE7002421461E688E
:1087D0005D6836682E4210D00C4D05EBC2020027B2
:1087E00056685A18376092F830200C3105EBC205F4
:1087F00003EB81036A685B6813608472D3E701242A
:108800002146E4E7580501004CE0FF1F8406010003
:108810000BB1FFF727BD7047DFF8F0C02DE9F0413D
:10882000DCF80040002C53D003686BB1D3F8004251
:108830008C4231D072B6046894F80832013B84F857
:10884000083262B60023036072B6DCF800800025AF
:1088500043462E462F460BE093F808E2D3F8044235
:10886000BEF1000F04BF3D461E461F46BCB1234665
:10887000D3F80042A142EFD13FB1D3F80422C7F8A8
:108880000422CCF80030C3F8048293F808220132A5
:1088900083F8082262B603601846BDE8F08192B101
:1088A0008EB13DB1D6F80432C5F80432CCF8006080
:1088B000C6F8048201220023C6F8001286F80822B6
:1088C00086F80932066062B603681846BDE8F08192
:1088D00072B60D4B4FF0FF3703F6546EC3F80072BB
:1088E00083F8084283F8094203F5037373454FF098
:1088F000000643F8083C044DF0D1C5F84C6ECCF8A6
:10890000005062B690E700BFA4CFFF1FA0CFFF1FAB
:10891000F8B5314CE37A0E461746EBB172B6E37AFE
:10892000DD071A4606D52D49E2680D682A40A26186
:108930000A601A46990706D5294923690D68E27A23
:108940002B40E3610B60520705D5264A6369116825
:108950000B402362136062B62368DA68B2F1384FC5
:1089600009D021491960214A4FF038454FF078412C
:10897000DD6019611A6001223146FFF74DFF48B3EF
:1089800090F80932DB07054616D5E37A12491A46F4
:1089900083B1D80703D5164A896911601A46990729
:1089A00003D5144BE169E27A1960530702D5124BE3
:1089B000226A1A602846F8BD3046294600F018FAA7
:1089C00040B11FB9012385F80932DEE7052385F898
:1089D0000932DAE70025D8E7D0A5FF1F80E100E0E3
:1089E00084E100E088E100E001403F0000003F80BA
:1089F00000E100E004E100E008E100E02DE9F041E1
:108A0000494CE37A054688461746EBB172B6E37ADD
:108A1000DE071A4606D54549E26808680240A261A9
:108A20000A601A46980706D5414923690868E27A20
:108A30000340E3610B60510705D53E4A6369116845
:108A40000B402362136062B62368DA68B2F1384FD4
:108A500009D039491960394A4FF038404FF0784110
:108A6000D86019611A60002241462846FFF7D4FEFB
:108A7000064600284BD090F80932DA0718D4404651
:108A8000394600F0B5F9E37A5BBB96F8093213F08A
:108A900001030FD12A68002A33D072B6296891F8F1
:108AA0000822013A81F8082262B62B60BDE8F08105
:108AB000E37AABB9314638464FF4007201F06AFCF4
:108AC0002B68002B2CD072B62A6892F80832013B32
:108AD00082F8083262B600232B600120BDE8F081E5
:108AE0000120DB0702D5164BA2691A60E37A0E4A11
:108AF000990708D45B0702D5124B226A1A60002E30
:108B0000C3D1BDE8F0811049D2690A60F2E740465E
:108B1000394600F06DF9E37A002BE2D1BDE8F0812F
:108B20000120BDE8F08100BFD0A5FF1F80E100E07B
:108B300084E100E088E100E001403F0000003F8068
:108B400000E100E008E100E004E100E003684BB16F
:108B500072B6026892F80832013B82F8083262B6B7
:108B600000230360704700BF184A194B70B41B689C
:108B7000156801264FF00044021285F80061DC629E
:108B80005A63DA6A002AFCDA0A0C42F080524FF08B
:108B900000449D6BDC625A63DA6A002AFCDA89B20F
:108BA00041F080514FF000429C6BDA625963DA6AFF
:108BB000002AFCDAC0B24FF00042996BDA625863C7
:108BC000DA6A002AFCDA9B6B70BC7047F8DDFF1F85
:108BD000D0A5FF1F38B5002144F29500FFF7C4FF70
:108BE000104B1A6809214FF00045FF24D5625463E9
:108BF000D36A002BFCDA906B030603D54B1E13F0EF
:108C0000FF01F3D1084B1C6801254FF00041FF2301
:108C100084F88050D1625363D36A002BFCDA936BE3
:108C2000C0B238BDD0A5FF1FF8DDFF1F38B54FF427
:108C3000D57144F68700FFF797FF1E4B1A6809218C
:108C40004FF00045FF24D5625463D36A002BFCDA51
:108C5000906B030603D54B1E13F0FF01F3D1C0B296
:108C6000012810D04FF00040134B1C6801254FF035
:108C70000041FF2384F88050D1625363D36A002BF4
:108C8000FCDA936B38BD4FF000410C4BD16253635B
:108C9000D36A002BFCDA916B084B4FF00040D06296
:108CA00009045363D36A002BFCDA906B80B208434B
:108CB000DAE700BFD0A5FF1FF8DDFF1FFFFF0010A0
:108CC000F8B5254C0021054647F2FF70FFF74CFF31
:108CD000226809214FF00046FF20D6625063D36A14
:108CE000002BFCDA936B1F0603D54B1E13F0FF011C
:108CF000F3D11A4E306801274FF00041FF2380F86E
:108D00008070D1625363D36A002BFCDA294646F6A1
:108D1000FF10936B4FF00045FFF726FF22680921F3
:108D2000FF24D5625463D36A002BFCDA906B0306F0
:108D300003D54B1E13F0FF01F3D1346801254FF02A
:108D40000041FF2384F88050D1625363D36A002B23
:108D5000FCDA936BC0B2F8BDD0A5FF1FF8DDFF1F92
:108D600038B5002147F6FF20FFF7FEFE1D4B1A68BD
:108D700009214FF00045FF24D5625463D36A002BCC
:108D8000FCDA906B030603D54B1E13F0FF01F3D101
:108D900010F0FF0F23D14FF00041134BD16253630A
:108DA000D36A002BFCDA916B0F4B4FF00040D0627E
:108DB00009045363D36A002BFCDA906B80B208433A
:108DC0000A4B1C6801254FF00041FF2384F88050B6
:108DD000D1625363D36A002BFCDA936B38BD002059
:108DE000EEE700BFD0A5FF1FFFFF0010F8DDFF1F5B
:108DF000F8B5444B444D1B78012B98BF40020C46FC
:108E0000014645F2FF10FFF7AFFE2B6809214FF036
:108E10000047FF26DF625E63DA6A002AFCDA986B9D
:108E2000020603D54A1E12F0FF01F3D110F0FF0F26
:108E30001DD14FF00040FF21D8625963DA6A002A41
:108E4000FCDA9A6BD2B2FE2A21D0FF2AF4D02F4A44
:108E5000106801244FF00041FF2280F88040D96261
:108E60005A63DA6A002AFCDA9B6B0020F8BD274AB5
:108E7000106801244FF00041FF2280F88040D96241
:108E80005A63DA6A002AFCDA9B6B0020F8BD204B9B
:108E9000204E5E631A4618465E63A11C04F50077F7
:108EA000D36A13F0F00FFBD04663836B01F8013CEB
:108EB0001B0A01F8023C0231B942F1D11449CA6AD5
:108EC000134B12F0F00FFAD09A6B84F8FF21120ABC
:108ED00084F8FE21DA6A0E4912F0F00FFAD00B4B3B
:108EE0002A6818688B6B01244FF00041FF2380F83B
:108EF0008040D1625363D36A002BFCDA936B01206C
:108F0000F8BD00BFFCDDFF1FD0A5FF1FF8DDFF1F70
:108F100000C00240FFFF001000207047002310B483
:108F20000361CB6943618A8A4B8B43EA02438361C5
:108F3000C361CB7A03F01003002B14BF022300237C
:108F400080F825304C1E00F126032E3014F8012F36
:108F5000202A19D003F8012B9842F7D10B7A202B45
:108F600016D02E2303700B7A43704B7A202B14D02B
:108F700083708A7A202A00F1030301D0C270031D96
:108F800000221A7010BC704718460B7A202BE8D1CB
:108F9000034600221A7010BC7047831C00221A700E
:108FA00010BC70472DE9F04F0C7887B0BCB32F2C64
:108FB00035D003AF01313D460DF1170C05AE4FF032
:108FC000200E0DF1150810E07E2C07D8A4F16103E6
:108FD000192B9CBF203CE4B22C700135654513D29F
:108FE00011F8014BFCB12F2C1DD02E2CECD1B54229
:108FF000F4D22B4603F801EBB342FBD16B1CC3EB5D
:1090000008031D446545EBD390F82530032B13D09E
:10901000022B42D00024204607B0BDE8F08F03AFFA
:109020003D460DF1170C202305F8013B6545FBD3A8
:1090300090F82530032BEBD14369D0F818904FEA14
:10904000532A904683460126BAF1000F4CD00AEB12
:10905000090301930022494602A80292FFF758FC37
:1090600090B3044600250AE043B3E52B26D0DBF895
:10907000103001352033102DCBF810302CD00B22BE
:109080003946204605F0EAF9002843D023782034F9
:10909000002EE9D1C3B10026E9E721498369214CBB
:1090A00009782568C361023B8B40012403EB050965
:1090B00004FA01FA904683460126C5E7C8F82090D5
:1090C00088F82450002BE6D1002402A8FFF73EFDCB
:1090D000204607B0BDE8F08F02A8FFF737FD019BDF
:1090E00009F101094B45B5D19BF82520032A91D000
:1090F000584600F005F900288CD0094BDBF81C20FD
:10910000084993F800900968023A02FA09F202EB62
:10911000010999E721464046FFF700FF0124D4E703
:1091200008DEFF1F04DEFF1F2DE9F0419AB00C4658
:10913000074600F049FA664B664A00921A469D6857
:1091400052F8261FCDF8261050689168127BCDF892
:109150002A00CDF82E10187B19698DF832205A6933
:109160001E7902958DF80C009D69D86904910592CD
:10917000196A93F8242093F825308DF80460069539
:10918000079008918DF824208DF825300DF13308D3
:1091900023782F2B3CD0002B6DD00DA800F014FAB3
:1091A000207830B10DAA21466846FFF7FBFE00E0AB
:1091B00083B314F8013F2F2BFAD160B312A80FC864
:1091C0009DF838E00F9E9DF840C0119D8DF804E099
:1091D00002969DF858E09DF85960079208938DF823
:1091E0000CC00495059006918DF824E08DF825605B
:1091F0000DF159020DF1260312F8011F03F8011BAE
:109200004345F9D10DA800F0F1F923782F2BC2D1F5
:109210000134BDE748B90DA800F0E8F9684600F050
:10922000E5F938461AB0BDE8F0811AAA9DF8383041
:1092300012F80F1D0F9C9DF8400087F825103B7118
:109240001199129BBC603873139C149839617B612F
:1092500015999DF85830F86187F82430BC6139625F
:1092600007F1260307F1330012F8011F03F8011B71
:109270009842F9D1CFE71AAA9DF8044012F8435D4D
:1092800002989DF80C10049B87F825503C71059DB1
:10929000069CB8603973079808993B619DF82430A3
:1092A000F86187F824307D61BC61396207F12603DB
:1092B00007F1330012F8011F03F8011B9842F9D19E
:1092C000684600F093F938461AB0BDE8F08100BF57
:1092D0000CDEFF1FD805010010B58EB0014600223C
:1092E00001A8FFF721FF9DF8294001A8032C8CBF9E
:1092F0000024012400F07AF920460EB010BD00BF12
:1093000070B51B4B1B4A1B781168C46982B00022E0
:10931000102B0646019201AD17D001EBD41128465F
:109320000122FFF7F5FAD8B104F07F0450F8243099
:10933000114AF36114682846A3428CBF002401241B
:10934000FFF704FC204602B070BD01EB1421284653
:109350000122FFF7DDFA18B1E4B230F81430E7E784
:109360002846FFF7F3FB0024204602B070BD00BF83
:1093700044DEFF1F40DEFF1F48DEFF1F90F8253050
:10938000012B1CBF0123037100207047704700BFF1
:109390002DE9F04F03694669C3EB0609914528BFE3
:1093A000914685B0B9F1000F4DD0DFF858B1544C5B
:1093B00080460D46C1699BF80000246800F109024F
:1093C000012707FA02F20239013A1A40814021448A
:1093D000C2F3080301EB5224002B39D11E460DF1D4
:1093E0000C0AC6EB090703E04E45A7F5007726D225
:1093F0000023B7F5007F2A462146504603934BD3FE
:10940000FFF7FCFA013405F5007500283DD0D8F8C7
:10941000103003F50073C8F810305046FFF796FB84
:109420009BF80030012202FA03F3013B234206F5C8
:109430000076D9D14046FFF763FF0028D4D13046EB
:1094400005B0BDE8F08F4E46304605B0BDE8F08F60
:109450000DF1100A00224AF8042D214650460193CE
:10946000FFF756FA002849D0019BC3F500764E4518
:1094700000EB030124D928464A4600F08BFFD8F8B8
:1094800010304B44C8F810304E465046FFF75EFB94
:10949000304605B0BDE8F08F1A46FFF739FA0028CC
:1094A000F3D001463A46284600F074FFD8F8103051
:1094B0001F44C8F8107050464E46FFF747FBE7E7D9
:1094C0003246284600F066FFD8F810303344C8F81A
:1094D00010305046FFF73AFB9BF8003007FA03F3D1
:1094E0000134013B234203D04E45A8D2354478E7EE
:1094F0004046FFF705FF0028F6D1A0E70646C4E77F
:1095000004DEFF1F08DEFF1F90F82530012B02D973
:109510004FF0FF30704770B582B001220DF10701A6
:1095200004460669C569FFF733FF012805D19DF898
:1095300007002661E56102B070BD4FF0FF30FAE729
:1095400090F82530012B02D94FF0FF30704700B55D
:1095500083B001220DF10701FFF71AFF012804D1A2
:109560009DF8070003B05DF804FB4FF0FF30F9E70A
:1095700090F82530012B01D900207047436900691C
:10958000181A48BF6FF00040704700BF10B504685C
:109590000C4A646882B094428DF8071008D190F8A4
:1095A0002520012A0AD001220271002002B010BD3C
:1095B00001220DF10701A04702B010BD002002B04A
:1095C00010BD00BF7D9300004FF47A7210B4064CBA
:1095D000826004210022046080F825100271027369
:1095E00080F8262010BC7047D8050100704700BFE6
:1095F00090F82530012B01D900207047FFF7C8BE35
:10960000F8B590F82530012B01D90020F8BD436949
:109610008B42FAD30F4B02691B78C769093321FAD1
:1096200003F422FA03F3E31A0DD41C460E46054652
:1096300014B90BE0013C09D02846FFF761FE002871
:10964000F8D1EF61F8BD8369C361EFE72E610120B6
:10965000F8BD00BF08DEFF1F0422002380F825208C
:1096600080F82630704700BF2DE9F04F754A764BE1
:10967000764D52F830202A60012489B021461C70B2
:10968000DFF8E8B101F03EFA2B68584683F88040D5
:10969000FEF77EFF9BF80B302BB372B69BF80B30B6
:1096A000DE07194608D56A48DBF80C10046821402B
:1096B000CBF81810016019469D0709D56548DBF8FD
:1096C000103004689BF80B102340CBF81C3003606B
:1096D0004C0707D56049DBF8143008680340CBF825
:1096E00020300B6062B6DBF80010CB68B3F1384F66
:1096F00009D05A4808605A4B4FF038444FF0784030
:10970000CC6008610B60574D05204FF00044CC62DF
:109710004D63CB6A002BFCDA013810F0FF008B6B35
:10972000F5D1514C514E23680493049DDFF848A1B4
:10973000DFF82491DFF81C81454FFFF74BFA012831
:1097400057D09BF80B301A466BB1D80703D5484A5F
:10975000B16911601A4699073AD4530744BFDBF840
:109760002030CAF8003023680593059B5B1BFA2B59
:1097700063D89BF80B30D3B172B6F37AD8071A4688
:1097800005D53968F2680A40B2613A601A4699070D
:109790000AD5D8F80010DBF810309BF80B200B40EE
:1097A000CBF81C30C8F80030530718D462B6DBF889
:1097B0000030DA68B2F1384FBFD0284919604FF055
:1097C0003841D960264A4FF0784119611A60B4E7F0
:1097D0002849DBF81C309BF80B200B60BDE7D9F85B
:1097E0000020DBF814301340CBF82030C9F80030EB
:1097F000DCE70190FFF71AFAB0F1004F019B3DD072
:10980000B0F5D57F00F0E0809BF80B301748194683
:109810009BB1DD0703D516498069086019469C078E
:1098200005D5144BDBF81C009BF80B10186048079B
:1098300003D5114BDBF820201A600024204609B024
:10984000BDE8F08F84060100FDDDFF1FF8DDFF1F7E
:1098500080E100E084E100E088E100E001403F00B9
:1098600000003F80FFFF001060DEFF1FD0A5FF1F3C
:1098700000E100E004E100E008E100E0964D002690
:109880002B7023680693069FDFF86882DFF878A2C2
:10989000DFF878923046FFF713FA002863D09BF880
:1098A0000B301A46A3B1D90704D58C4AD8F8181042
:1098B00011601A46990705D58949DBF81C309BF8D9
:1098C0000B200B60530703D5864ADBF8203013606A
:1098D0000128B2D823680793079B40F2DC52DB1BB8
:1098E0009342AAD89BF80B3043B372B698F80B306A
:1098F000D8071A4609D57C4A1168D8F80C200A40C6
:109900007949C8F818200A601A4699070AD5D9F883
:109910000010DBF810309BF80B200B40CBF81C300C
:10992000C9F80030530708D5DAF80020DBF8143006
:109930001340CBF82030CAF8003062B6DBF80030B4
:10994000DA68B2F1384FA5D0684919604FF0384154
:10995000D960674A4FF07841196130461A60FFF7C5
:10996000AFF900289BD12B785B4C022B32D09BF8AF
:109970000B30604819469BB1DC0703D55749806915
:10998000086019469A0705D5554BDBF81C009BF873
:109990000B1018604B0703D5524BDBF820201A60E0
:1099A00008AD002445F8144D224628462146FEF70E
:1099B000AFFFB0F8FE214AF655239A4211D0002499
:1099C0002846FFF7C3F839E7434D02232B704FF0C9
:1099D000804656E7FFF7C4F9800F032808BF2070C0
:1099E000C5E790F8C231062B68D00B3B012B65D937
:1099F0002846FFF7ABF8002221462846FEF788FFED
:109A0000B0F8FE214AF655239A42D8D1B0F80B306F
:109A1000B3F5007FD3D1037C022BD0D1B0F80EC0B8
:109A2000BCF1000FCBD0437B334AC68AB3FA83F331
:109A3000C3F11F0882F8008006B9466AB0F81170B9
:109A4000B0F8132007F10F01090902B9026ADFF823
:109A5000C0E06444CCEB02035B1A32193144DFF8F6
:109A6000B4C0CEF800401144DFF8ACE0234CCCF891
:109A70000010A3EB460323FA08F340F6F471CEF886
:109A800000208B4203F1010EC4F800E097D94FF695
:109A9000F4718B421A4B1B4913D87F0132440324C3
:109AA00010205F619A6183F82540087000212846E4
:109AB000DA6119610124FFF749F881E7D0F8C6415E
:109AC00096E7C26A9A610026022420205E6183F82C
:109AD00025400870EAE700BFFCDDFF1F00E100E061
:109AE00004E100E008E100E080E100E001403F0027
:109AF00000003F80D0A5FF1F08DEFF1F48DEFF1FCC
:109B00000CDEFF1F44DEFF1F88E100E084E100E07F
:109B100040DEFF1F04DEFF1F00DEFF1F10B5054CF7
:109B20002046FFF751FD2046034A0449BDE8104096
:109B300004F036B90CDEFF1FFC97FF1FED95000007
:109B4000014B024A1A6070474CDEFF1F01100138BA
:109B5000524ADFF868C12DE9F04F514D514CDFF802
:109B60006081DFF860B1DFF860E11646D17A09B3B1
:109B700072B6F37AD807194607D5DBF80000F1680A
:109B80000140B161CBF8001019469B0707D5DCF8FE
:109B900000001369D17A0340D361CCF800304F073D
:109BA00006D5D8F8001053690B401362C8F800308E
:109BB00062B6D17A1368D868B0F1384F0AD04FF046
:109BC00078404FF03849C3F800E0C3F80C901861B2
:109BD000354818602078D5F800A04FF001098007BB
:109BE0008AF800914FF000492DD57020C3F82C90D1
:109BF0005863D86A0028FCDA4FF0004900209F6BB8
:109C0000C3F82C905863D86A0028FCDA01209B6BBB
:109C10008AF8800081B1CF0703D5244F9069D17AAB
:109C20003860880703D5224FD069D17A3860490758
:109C300002D52048116A01601B0697D51E4B0022F1
:109C40001A70BDE8F08F0520C3F82C905863D86ACD
:109C50000028FCDA4FF0004900209F6BC3F82C90DD
:109C60005863D86A0028FCDA01209B6B8AF88000D0
:109C700081B1CF0703D50D4F9069D17A386088073D
:109C800003D50B4FD069D17A3860490702D509480E
:109C9000116A0160DB073FF569AFCFE7D0A5FF1F71
:109CA00054DEFF1F50DEFF1F00003F8000E100E098
:109CB00004E100E008E100E051DEFF1F84E100E084
:109CC00088E100E080E100E001403F002DE9F04F35
:109CD0000E4685B0002181463046154604F054FCFE
:109CE000984B994ADB7A11780291002B25D072B6F5
:109CF000944BDB7ADC07194608D5944891490468EF
:109D0000C96821408F4CA16101601946980709D5A7
:109D10008F488C4B04681B698A492340894CC97A57
:109D2000E36103604B0707D58A49864B08685B6986
:109D30000340844803620B6062B6824B1B68D9689B
:109D4000B1F1384F09D0844818604FF03840D860DE
:109D500082494FF07840186119608148DFF804B2F9
:109D60000178039100297ED1DBF80020029800F0F1
:109D7000080A00F001015FFA8AFA01914FF0010828
:109D800009EB0507BAF1000F40D1544682F8008173
:109D9000019A002A4DD04FF000410322D9625A6344
:109DA000DA6A002AFCDA4FEA194242F080524FF098
:109DB0000041986BD9625A63DA6A002AFCDA1FFA0A
:109DC00089F949F080524FF00041986BD9625A638B
:109DD000DA6A002AFCDADFF86C919B6B3246314676
:109DE0002B464846FEF714FDDBF800202E4482F88F
:109DF00080800121002C00F0B780524B2546B946E7
:109E00001B6809EB0507BAF1000FBED07C1E84EA7F
:109E1000090414F07E44B9D029F07E4182F8008113
:109E2000019AC1F100716C1A09EB01070D46002A75
:109E3000B1D1C9F3074242F0805242F440724FF070
:109E40000041D9625A63DA6A002AFCDA1FFA89F9FA
:109E500049F080524FF00041986BD9625A63DA6A38
:109E6000002AFCDAB7E71178DBF8002001248F071D
:109E700082F800414FF0004440F1B8807021DC626C
:109E80005963D96A0029FCDA4FF0004400219F6B26
:109E9000DC625963D96A0029FCDA996B090600F182
:109EA000B880039B0121022B82F8801000F2BE8053
:109EB000244B82F800111B684FF000400621D86245
:109EC0005963D96A0029FCDA01209C6B82F8800072
:109ED00020210139FDD102994C0740F10C810399F1
:109EE00081420CBF8521752101244FF0004082F88A
:109EF0000041D8625963D96A0029FCDA986B02984C
:109F0000012110F0020F82F880104FF0004082F81B
:109F1000001100F0DD807021D8625963D96A0029F0
:109F2000FCDA996B4FF000440020DC625863D96A78
:109F30000029FCDA996B0906F7D5012182F8801017
:109F400014E700BFD0A5FF1F50DEFF1F80E100E037
:109F500084E100E088E100E001403F0000003F8034
:109F600051DEFF1F54DEFF1F039B23B3D9F80030DF
:109F700082F800114FF000400621D8625963D96A77
:109F80000029FCDA01209C6B82F880002021013935
:109F9000FDD102994C0743D47A2101244FF00040AF
:109FA00082F80041D8625963D96A0029FCDA01219C
:109FB0009B6B82F88010554B5449DB7A1A4693B15B
:109FC000D80703D5524A896911601A46990704D502
:109FD0004E4A504BD169D27A1960530703D54B4A88
:109FE0004D4B126A1A6005B0BDE8F08F0521DC62A6
:109FF0005963D96A0029FCDA4FF0004400219F6BB5
:10A00000DC625963D96A0029FCDA996BCF073FF506
:10A0100048AF0021012482F8804001700391A5E639
:10A020000399814214BF7A218A21B6E7374B37481A
:10A03000DB7A19469BB1DC0703D535498069086096
:10A0400019469F0705D5314B32483049DB69C97A3B
:10A0500003604C0703D52D492F4B096A1960019203
:10A06000FFF776FD294B2949DB7A019AEBB172B6ED
:10A07000CB7AD8071A4640D49B0709D52749234BEA
:10A0800008681B69214A03402048D27AC3610B60EB
:10A09000570707D5224A1D4B11685B690B401B49C6
:10A0A0000B62136062B6DBF80020184B1B68D9689E
:10A0B000B1F1384F09D01B4818604FF03840D860D4
:10A0C00019494FF0784018611960002103914DE65D
:10A0D0000521D8625963D96A0029FCDA996B4FF0DF
:10A0E00000440020DC625863D96A0029FCDA996BCD
:10A0F000CF07F7D421E77521F6E60C48CA68046853
:10A1000022408A6102601A46B6E700BFD0A5FF1F51
:10A1100000E100E004E100E008E100E084E100E0AB
:10A1200088E100E001403F0000003F8080E100E066
:10A1300090F8392090F83800101A704790F83830AD
:10A1400090F839209A4205D95A1C034480F83820E7
:10A15000187E70474FF0FF30704700BF90F83830DE
:10A1600090F839209A4286BF1B18187E4FF0FF30B6
:10A17000704700BF704700BF38B50546B0F85E00B5
:10A1800090B195F85D301446C3F1210294420CD889
:10A1900005F13B001844224600F0FCF895F85D30CC
:10A1A000234485F85D30204638BD012014462871CF
:10A1B000EEE700BFB0F85E306BB190F85D30202B59
:10A1C00007D8C218013380F85D30012082F83B10B7
:10A1D0007047012303710020704700BF10B502696A
:10A1E000D378DBB2D90604463DD510215806D1708C
:10A1F00038D503F0040303F0FF02002B51D03D4992
:10A20000626E00230B7084F85D30002A5BD09047AB
:10A2100094F85D30002B56D02369D0229A702369C0
:10A2200094F83B201A712369012284F85C200222F1
:10A23000DA7010BD304B84F860009C424AD02F4B3E
:10A240009C4252D094F8391013791F29DBB207D8F9
:10A250002848007820B16018013184F8391003765D
:10A260000223D37010BD5906C3D4917801F01001B8
:10A2700001F0FF000029DDD013F001031ED194F896
:10A280005C1094F85D00884281BF4B1C091984F86A
:10A290005C3091F83B3013712369D0229A702269A7
:10A2A000DEE7236984F83920C0229A702369114AB5
:10A2B0001979012111700222DA7010BDC023937048
:10A2C00022691379CCE70122002384F85D2084F809
:10A2D0003B30A1E7626994F86130094913440322D5
:10A2E000187A00F029FB2269ACE7626994F86130C2
:10A2F0000449F3E758DEFF1F08A6FF1F74A6FF1FDF
:10A3000065A3000071A300000369DB7803F020035C
:10A3100073B190F860300133DBB2012B80F860300C
:10A320001AD9426990F861301344187A00F080BB62
:10A3300070B5426903F0FF0590F86130134404469C
:10A34000187A00F075FBA36E5BB184F8385094F86E
:10A350003900BDE87040184790F85F30002BE0D01E
:10A36000704770BD0148FFF7CFBF00BF08A6FF1FB1
:10A370000148FFF7C9BF00BF74A6FF1F0148FFF7E0
:10A380002DBF00BF08A6FF1F0148FFF727BF00BF72
:10A3900074A6FF1F844641EA000313F003036DD146
:10A3A000403A41D351F8043B40F8043B51F8043B98
:10A3B00040F8043B51F8043B40F8043B51F8043B9F
:10A3C00040F8043B51F8043B40F8043B51F8043B8F
:10A3D00040F8043B51F8043B40F8043B51F8043B7F
:10A3E00040F8043B51F8043B40F8043B51F8043B6F
:10A3F00040F8043B51F8043B40F8043B51F8043B5F
:10A4000040F8043B51F8043B40F8043B51F8043B4E
:10A4100040F8043B51F8043B40F8043B51F8043B3E
:10A4200040F8043B403ABDD2303211D351F8043BDE
:10A4300040F8043B51F8043B40F8043B51F8043B1E
:10A4400040F8043B51F8043B40F8043B103AEDD28D
:10A450000C3205D351F8043B40F8043B043AF9D2DE
:10A46000043208D0D2071CBF11F8013B00F8013BB1
:10A4700001D30B8803806046704700BF082A13D3BE
:10A480008B078DD010F003038AD0C3F10403D21AD6
:10A49000DB071CBF11F8013B00F8013B80D331F80A
:10A4A000023B20F8023B7BE7043AD9D3013A11F88A
:10A4B000013B00F8013BF9D20B7803704B784370F5
:10A4C0008B78837060467047374A384913681B069B
:10A4D000FCD40B6813F08003F8D172B634490A78C3
:10A4E000002A5FD0334A3448F0B4344C1768066809
:10A4F0002568D4680C303E44143200681268304F2E
:10A5000035442C4420440244C2F34E022D4E2E48C2
:10A510002E4D2F4C42F400423A60376806682D6891
:10A520002C4A24680C303E44006812682A4F354497
:10A530002C4420440244C2F34E02284E2848294DA0
:10A54000294C42F400423A60376806682D68274A71
:10A5500024680C303E4400681268254F35442C4472
:10A5600020440244C2F34E02224E2348234D244C81
:10A5700042F400423A60376806682D68214A246830
:10A580000C303E440068126835442C442044024498
:10A59000C2F34E021C4842F4004202600B7062B6E5
:10A5A000F0BC704762B6704724B0034024B00B4043
:10A5B0005ADEFF1F38B003403CB0034040B00340B8
:10A5C0002CB0034058B003405CB0034060B003407F
:10A5D00064B003406CB0034030B0034038B00B406F
:10A5E0003CB00B4040B00B4044B00B404CB00B4073
:10A5F0002CB00B4058B00B405CB00B4060B00B402F
:10A6000064B00B406CB00B4030B00B4030B4294804
:10A61000294A2A4B2A4D6024E121047011701B78CD
:10A62000284C082B30D00A2B2748284937D00C2B30
:10A630000CBF35223D2212232A60236002600B608A
:10A64000234B24491B78244ABBB101230B601360C0
:10A65000224B23491B78234A012B26D9042B0FD9DF
:10A66000082B1ED9102B94BF862387230B60136001
:10A670001D4B01221A7030BC70470B601360E7E776
:10A6800084230B601360F3E700F58E200F49083038
:10A69000012213232A60236002600B60D0E7392275
:10A6A000F7E785230B601360E2E780230B601360FC
:10A6B000DEE700BF0040074001400740E0A6FF1F63
:10A6C00008B003400CB0034008B00B400CB00B4086
:10A6D0005DDEFF1F20B0034020B00B40E1A6FF1F4E
:10A6E00024B0034024B00B405ADEFF1F28282FD887
:10A6F000334B2DE9F0411E5CFF2E2BD0314B1B78E4
:10A70000002B2AD132062CD472B62F4D2F4C2F4657
:10A71000012326602B7062B672B623681B060CD428
:10A720003B781BB9F4E72B78002BF1D062B602F02E
:10A73000C7F972B623681806F5D5254B1B680022A9
:10A740002A7062B6234A107843FA00F0BDE8F0811F
:10A75000002070470020BDE8F081FFF7B5FE32060B
:10A76000D2D572B61C4DDFF87C801C4C06F0400739
:10A77000FFB206F03F06D8F80030DFB123F0100337
:10A78000C8F8003001232660134A2B7062B672B6F7
:10A79000236819060CD413781BB9ECE72B78002B2F
:10A7A000E9D062B602F08CF972B623681B06F5D5C3
:10A7B0000B4BC3E743F01003C8F80030E2E700BFDB
:10A7C000580601005ADEFF1F5CDEFF1F00B0034089
:10A7D00010B0034059DEFF1F5BDEFF1F00B00B40CF
:10A7E00010B00B400CB00B4008B5104C08E02368CB
:10A7F00059050DD423681A050FD42368DB0411D43E
:10A8000023685803F3D500F07DFC23685905F1D582
:10A8100000F018FB23681A05EFD502F0D5F923687C
:10A82000DB04EDD502F066FAEAE700BF34800440AD
:10A8300008B5FFF7D9FF00BF014B10221A807047FF
:10A8400000200540704700BF094908B50B6830B1CA
:10A850006A461844A2F58052904202D20860184617
:10A8600008BD03F0B1FA0C2303604FF0FF3008BDC0
:10A87000E4A6FF1FFEE700BF704700BF10B40F4BF8
:10A8800053F8302092F880422CB1012369B182F84C
:10A89000803010BC704703EBC0035B681A6841B995
:10A8A00022F002021A6010BC704782F8003110BC1E
:10A8B000704742F003021A6010BC70478406010022
:10A8C0001C4A02EBC00301295B6811D004291BD08C
:10A8D00052F83000002280F8802229B1022920D0CD
:10A8E000032922D01A6070474FF480721A607047B3
:10A8F00052F830004FF4A27280F880121A601A6881
:10A9000022F020021A60704752F830104FF4A27201
:10A91000012081F880021A601A6842F020021A6051
:10A92000704740F203121A6070474FF481721A6048
:10A93000704700BF84060100212848D8F8B5042AD2
:10A9400044D8DFE802F0484B4E0345004FF4102690
:10A950002B4B03EBC0030D465C68216811F4E061EA
:10A9600048D0284B284A2949C3F89C2104F1404289
:10A970002748C3F8A411A2F59221264FC3F8A001DD
:10A980007C292548C3F8A871C3F8AC012CD9A2F5DD
:10A9900094237C2B2AD9A2F596237C2B28D9A2F5C7
:10A9A00098237C2B29D9A2F59A227C2A27D81B48E8
:10A9B00072B6236823F4702343F08072C4F38401D9
:10A9C0001643236040F82150266062B6F8BD7047F8
:10A9D0004FF43026BCE74FF40026B9E74FF4402689
:10A9E000B6E74FF42026B3E70D48E1E70D48DFE76F
:10A9F0000D48DDE7FFF764FFB3E70C48D8E7F8BD83
:10AA0000840601000092FF1FD197FF1F7997FF1F57
:10AA1000A597FF1F4D97FF1F2197FF1FC0A7FF1F7F
:10AA2000E8A6FF1F20A7FF1F70A7FF1FA0A7FF1FFB
:10AA30001A4B03EBC00010B4426802F14043A3F587
:10AA400092217C2923D9A3F594217C290DD9A3F542
:10AA500096217C291FD9A3F598217C2919D9A3F522
:10AA60009A237C2B11D80E4C00E00E4C72B6136862
:10AA70000D4823F08773C2F3840123F4803343F03D
:10AA80008073136044F8210062B610BC7047074C15
:10AA9000ECE7074CEAE7074CE8E700BF8406010053
:10AAA000C0A7FF1F20A7FF1F79A80000E8A6FF1F6F
:10AAB000A0A7FF1F70A7FF1F30B4054B054D064C24
:10AAC000002210211A602A602060196030BC704793
:10AAD00014D0034004D0034000D00340212801D803
:10AAE000FFF7CCBE704700BF212806D8044B53F8AF
:10AAF000303093F80002C0B270470020704700BFAA
:10AB000084060100212801D8FFF7DABE704700BF94
:10AB100072B60C490C4B0D4A1B680868126862B685
:10AB2000520102D5322B88BF01300949C3F5BB332E
:10AB30004FF47A72FF33A1FB031302FB00F000EB2A
:10AB40009310704760DEFF1F18E000E004ED00E0A6
:10AB5000ABAAAAAA2DE9F843054672B6204F214BAD
:10AB6000214A1B683C68126862B6520102D5322B3A
:10AB700088BF013495B3C3F5BB331C4EDFF8649036
:10AB8000DFF86480FF334FF47A72A6FB031302FBF5
:10AB900004F404EB931472B6D9F800103A68D8F8AC
:10ABA00000E062B6C1F5BB33FF33A6FB03031EF022
:10ABB000806FC4EB93134FF47A7002D0322988BFB0
:10ABC000013200FB0233B3F57A7F04D3013D05D097
:10ABD00004F57A74DFE701F073FFDCE7BDE8F88382
:10ABE00060DEFF1F18E000E004ED00E0ABAAAAAAB7
:10ABF000F8B52D4B2D49DFF8D0E0DFF8D0C02C4E52
:10AC00002C4D2D4C2D4A2E4F4FF4000018604FF064
:10AC1000807018604FF0007018604FF0806018600E
:10AC20004FF0006018600020086028234BF6FF7189
:10AC3000CCF80010CEF80030336013602B60236036
:10AC40003B60B3629362092245F8242CC4F8D80F04
:10AC500005F57F65C7F8D41F07F5FF2707F5FA67E5
:10AC6000C6F8F83F2B6006F5FF26C4F8D42F05F58B
:10AC7000FD2504F5FF24386006F2F47611483160B2
:10AC800005F5FF6504F5FD642B6023600260FFF7A6
:10AC9000BDFC1920FFF75EFF00F09CFF40F213108F
:10ACA000BDE8F840FFF756BF08E100E0048003402C
:10ACB00014800340248003402C8003401C80034008
:10ACC0003480034000800B400C8003400880034028
:10ACD0002B4A2C491368F0B543F4806313600A785B
:10ACE000294F2A4E2A4D2B4C2B4900233B703370A1
:10ACF0002B7023700B70002A3DD0152A21D0274BD2
:10AD00001B78012B25D0052B30D01F2827D80020F9
:10AD100002460125224B234C1A7023495D70042200
:10AD20004FF0020E88273C26402598729A704FF407
:10AD3000005083F813E05A751F74DE7025700860A8
:10AD4000F0BD1A4B40F213321A60144B1B78012BE2
:10AD5000D9D1174B4FF451721F281A60D7D9C0F3BD
:10AD60004432C0F3471500F01F00D3E7114B4FF4F6
:10AD700051721A60C9E7104B40F213321A60BEE7F5
:10AD800034800440ACDEFF1F68DEFF1F69DEFF1F5A
:10AD9000F8DEFF1FF1DEFF1FF0DEFF1FC8A7FF1F59
:10ADA00000A006402DE400E004E100E018C00440EB
:10ADB00044A004401CC0044040A00440054A064B87
:10ADC00010781B78C0B2DBB2984238BF4030C01A4E
:10ADD000704700BF68DEFF1F69DEFF1F30B4154BF0
:10ADE000154C1A782378D2B2DBB29A421ED00133C6
:10ADF0003F2B0ED91149124B087819680023C0B2B5
:10AE0000237021B1D31A1A2B01DC00230B7030BC44
:10AE100070470A480A49C05C0968DDB2C0B22570B3
:10AE20000029F4D09A4238BF4032EBE74FF0FF30B0
:10AE3000EDE700BF68DEFF1F69DEFF1FB0DEFF1F0A
:10AE400064DEFF1FF0B4384B1A7912F0300F2CD0AB
:10AE500072B6997D01F0FF0200293DD062B6334FF2
:10AE6000334938780D78334E1C46C0B2EDB2431CDE
:10AE7000402BE17928BF0023AB4202F1FF32C9B277
:10AE80001CBFF154184612F0FF02F0D12A4B1B6888
:10AE9000C2B23A704BB1A84236BFC5F14005401B63
:10AEA00040192728C4BF01221A701F49CA78D2B29C
:10AEB000150616D452060DD51B4B1B795B0609D51A
:10AEC0001E4B1F491B6800220A7003B11A70164BF3
:10AED0003C22DA70F0BC70474022D9795A7462B6CD
:10AEE000E3E70B791C06E5D5164B174E1C78337833
:10AEF000E4B2DBB29C420ED0144D01E0A3420AD072
:10AF00000133402B28BF00230879E85CC0B2C87128
:10AF1000087D0728F2D9DBB2034933700B79180694
:10AF200044BF7C23CB70C5E700A0064068DEFF1F4E
:10AF300069DEFF1FB0DEFF1F64DEFF1FF4DEFF1FB0
:10AF4000F0DEFF1FF8DEFF1FF1DEFF1F6CDEFF1FCC
:10AF5000431E032B14D872B60A4951F8230068B176
:10AF600070B4094C058834F81320466841F8236012
:10AF7000521B24F8132062B670BC704762B670474B
:10AF80000020704754DFFF1F7CE1FF1F01380328BA
:10AF90000BD872B6074B53F8203043B100205B68E2
:10AFA0000130002BFBD162B6704700207047184675
:10AFB000F9E700BFA8DFFF1F30B472B62B4A137841
:10AFC0001D0706D52A4B196A002936D0996A00292F
:10AFD00041D053781C0706D5254B196C00293ED06B
:10AFE000996C002939D09378190705D5204B196E33
:10AFF000002936D0996E89B1D3781B0707D51C4B31
:10B00000D3F880207AB3D3F8882011213AB162B600
:10B01000184B00221A7030BC00F068BE0D21154C90
:10B02000154D227843F8315003EBC1030830013A43
:10B030005860227062B630BC704704220D4C0F4D30
:10B04000217843F8325003EBC20308304A1E58609F
:10B05000227062B6EFE70521E1E70921DFE7082268
:10B06000ECE70C22EAE71022E8E700BFCC0701007A
:10B070000080FF1FD1DFFF1FC80040008800400094
:10B08000431E032B1DD81B4A400140F0100030B472
:10B09000104472B6184CE25C032A1BD8DFE802F0B9
:10B0A0000212151703220D88E25410F0080F14BF86
:10B0B000C823882343EA054308310360416062B630
:10B0C00030BC704708300222EDE70522EBE708307C
:10B0D0000422E8E7094A52F8230038B1084A52F836
:10B0E0002300416042F8231062B6E9E742F82310DA
:10B0F000034AF7E70080FF1FE0DFFF1FA8DFFF1F05
:10B10000B8DFFF1F2DE9F04FDFF80CB3DFF80CA319
:10B1100087B044E0AB4F4FEA930807EBC809013E04
:10B12000D9F8042003F00803F6B2A2F1080003F0F6
:10B13000FF04002B40F0028157F838301B0C99B205
:10B1400022F8081C002B00F0F0809F4B22F8064CE0
:10B1500042F8044C53F82620002A00F0C5829B4D8B
:10B1600055F8263058609A4C45F8260034F81630C9
:10B17000194424F8161000F099FD002800F0AD8263
:10B18000944A954B19F0080F00F1080018BF1346B8
:10B19000C9F8040047F8383008238BF800309BF8D2
:10B1A0000040E4B261071AD58C4B1B78A3B18C49DF
:10B1B0000A7802F0FF0322B1013BDBB20B7003B946
:10B1C00000BE88490A7802F0FF032AB1013BDBB2D6
:10B1D0000B70002B00F0578204238BF8003004F032
:10B1E000080303F0FF02002B00F0CC809AF8003037
:10B1F000DBB21E098ED19C08DFF8C89159F83420C3
:10B2000009EBC401C2F38302013A49680C2A00F237
:10B210008880DFE802F07C7C868686868686478684
:10B22000868607000868704D4A68704F704E286027
:10B2300081B240F28160674B6A604FF0010E0022DC
:10B24000814249F834303A60C9F81020C9F8182012
:10B2500086F800E05B4C00F2E380B1F5D06F80F03F
:10B260004683B1F5817F00F0FC8200F28D82802957
:10B2700000F07783822940F0FA82A98801F07F01EB
:10B28000042900F2F4825B485B4C89000844227078
:10B2900062700278930740F1588484F800E04FF020
:10B2A000020E42E3514F3A6832B3544B504E544968
:10B2B000188834780D784028864645F0020828BF63
:10B2C0004FF0400E002C84F001043470CEEB0000EF
:10B2D0000CBF8824C82409EBC80680B285F001059C
:10B2E00044EA0E447260188049F8384072440D7088
:10B2F000002800F045813A603B4B1A88B2F5A06FF8
:10B300000FD100219A7859703E4B1A7009E0364AE5
:10B31000108842F22102904200F037812D4A49F80C
:10B320003420394A0123137036E72A4A2A4B19F090
:10B33000080F18BF134647F838302DE700F0D6FC49
:10B34000324A334952F82630002B00F0D181586838
:10B350008C5D42F8260003F10802C9F80420032C92
:10B3600005D8DFE804F02C02292602228A551A8823
:10B3700019F0080F0CBF8823C82343EA024347F89B
:10B38000383009E7E00700F18181210600F1F28100
:10B39000A20706D51F4A204913780220DBB213709A
:10B3A0000870E30602D51C4B10221A7007B0BDE8E6
:10B3B000F08F04228A55DAE705228A55D7E703225F
:10B3C0008A55D4E70080FF1F54DFFF1F00DFFF1FF7
:10B3D0007CE1FF1FC800400088004000DCDFFF1F49
:10B3E00065DFFF1FE4DFFF1FC8DFFF1FFCDEFF1F5D
:10B3F00064DFFF1FC0200740D4DFFF1F10DFFF1FE7
:10B40000D0DFFF1F9820074094200740A8DFFF1FD0
:10B41000E0DFFF1F88200740802007409020074082
:10B4200042F22100814200F02A8100F2D880B1F579
:10B43000086F00F07682B1F5106F40F01882226A32
:10B44000B349A8780870120600F13A83D9F8282089
:10B45000B049130600F10C83D9F83020AD49150628
:10B4600000F10183D9F83820AA49140600F1F682C8
:10B47000D9F84020A749100600F14A83D9F848209E
:10B48000A449120600F13F83D9F85020A1491306C0
:10B4900000F13483D9F858209E49150600F129831C
:10B4A000D9F860209B49140600F11E83D9F8682062
:10B4B0009849100600F11383D9F8702095491206B7
:10B4C00000F10883D9F878209249130600F1FD8233
:10B4D000D9F880208F49150600F13183D9F88820EA
:10B4E0008C49140600F12583D9F89020894910066B
:10B4F00000F11983D9F898208649120600F10D83CE
:10B500008548864A864901908648874D874C04972E
:10B5100000230596029580460F4616461D46039465
:10B52000306828B1446800F0E1FB2046002CF9D1D6
:10B5300000233360029B38681A46002342F8253006
:10B5400028B1446800F0D2FB2046002CF9D100223B
:10B550003A60019A98F800301146002241F8042B15
:10B56000039A0191023B4FF0000122F81510032BC2
:10B5700000F22B81DFE813F0700125017001250135
:10B58000BEF1400F18BF0022B5E6694A0D78487831
:10B59000157050708D78C8789570D07010680D79DE
:10B5A000157186284D7989795571917100F09B81CB
:10B5B0006049614E0A78307882F00105002842F037
:10B5C00002020D700CBF8821C82149F8321009EB26
:10B5D000C20280F001000021307051609EE642F20C
:10B5E0002120814240F0CB81544B554C5549A878DD
:10B5F0001D682560CDF804E00870002002908046A8
:10B60000844604464B490D7845F0020E09EBCE0303
:10B610000393019B002B039B5C600CBF8824C82410
:10B6200044EA080385F0010449F83E3032700C709A
:10B63000DFF8E0E0404BDFF8FC80002840F01E819E
:10B64000BCF1400F1BD144F0020C09EBCC03029C6F
:10B65000DFF8C0E05C60002A40F02681020442F07E
:10B6600088029DF804304EF83C20044433700D707D
:10B670002346402803D10020334A3B601080334AE0
:10B68000012313704DE600F09DFCA5E5214B2F48EA
:10B6900028491A614FF0020E80F800E02C4F0A7022
:10B6A0002C49196099602C4E2C4D2D4C9A610D211E
:10B6B0003970FF213170DFF8B8E029702270294D10
:10B6C000294A8EF800109F27012406F8047C5D604B
:10B6D0000470DA6007B0BDE8F08F244A47F83800FC
:10B6E00013780133137057E543F826000E4D3AE501
:10B6F0008B5D032B00F2F08001A252F823F000BF13
:10B7000099B1000099B10000BDB70000B7B70000C3
:10B71000DCDFFF1F0080FF1FB8DFFF1F54DFFF1FAC
:10B72000A8DFFF1FE0DFFF1F00DFFF1F7CE1FF1F1F
:10B7300084E1FF1FD0DFFF1F64DFFF1F60DEFF1FFC
:10B740008CE1FF1FF4DFFF1F10DFFF1F9420074075
:10B75000C020074088004000882007408020074024
:10B760009820074014DFFF1F68DFFF1FD1DFFF1F96
:10B770008C200740C149C24B80220D2008701A70EE
:10B78000A2077FF50EAE05E640F20232914240F08C
:10B79000EE80A98801F07F01042968D86A88002A10
:10B7A00065D1B648CDF804E089000844017841F03D
:10B7B0000201017021E701238B55EDE400238B5535
:10B7C000EAE44FF0010388F800300135042D06F15A
:10B7D000040607F1040708F101087FF4A1AEA94CA3
:10B7E000A94B2278A94D049F059E002129701A704B
:10B7F000130700F105816278A549DFF8A0820A707D
:10B8000010074FF00001C9F83010C9F8381000F1E6
:10B81000E080A049A2780A700021C9F85010C9F848
:10B8200058101107DFF8748200F10181E2789A491B
:10B830009A4C0A7000211207C9F87010C9F87810E4
:10B8400000F1B08033780193002183F00102C9F840
:10B850009010C9F89810D0E64FF0000388F8003037
:10B86000B3E7A98801F07F01042940F28D80834A63
:10B870000F2313708A4A0123137052E540287FF684
:10B88000E2AE44F002040EEBC401029E4E60BAB177
:10B890009DF80410834A19703346403888F80050E8
:10B8A00040334EF83420E7E69DF80430337002044C
:10B8B000029B0D7042F0C80203444EF83C20D8E6CB
:10B8C0009DF804101970029B774A88F800504038A0
:10B8D00040334EF83420CFE619F0080F0CBF022396
:10B8E00003238B5558E4714A0F21117060E6704AAA
:10B8F0005468002CBBD06888B5F804E003E00C3233
:10B900005468002CB3D013888342F8D15388734510
:10B91000F5D1000A03280CBF94F800E0B2F808E063
:10B9200003E0644A644C12782270E888704580F025
:10B930003F8162490D784028844645F0020E28BFB9
:10B940004FF0400C04EB0C0309EBCE0202930123F1
:10B950005460CCEB00004FEA0C4800220193C8244D
:10B960005EE6554C4FF0020E22706270DDE7B1F5D5
:10B97000A06F7FF47CAF0123002201933DE642F2E9
:10B9800021329142F7D072E76A88002A7FF46FAFC4
:10B990003A48CDF804E089000844017821F002011A
:10B9A00001702AE600F082F9002800F0EF800830EC
:10B9B0003D4AC4F88400C4F8802000F077F90028DC
:10B9C00000F0DE800830374AC9F88C00C9F88820BA
:10B9D00038E700F06BF9002800F0C0800830324AE8
:10B9E000C8F84400C8F8402000F060F9002800F0D2
:10B9F000AF8008302B4AC9F84C00C9F8482008E746
:10BA000000F054F9002800F0CD800830264AC9F82B
:10BA10002400C9F8202000F049F9002800F0BC807B
:10BA20000830204AC9F82C00C9F82820E3E600F0C5
:10BA30003DF9002800F09E8008301B4AC8F86400D9
:10BA4000C8F8602000F032F9002800F08D8008303E
:10BA5000144AC9F86C00C9F86820E7E6C86B0838D2
:10BA600000F044F904E5486B083800F03FF9F9E4C8
:10BA7000C86A083800F03AF9EEE400BFC020074079
:10BA800080200740CC070100C4200740D1DFFF1F02
:10BA9000C8200740CC200740D02007400080FF1F6F
:10BAA00094200740C80040008800400065DFFF1F69
:10BAB000D0070100DCDFFF1FD4DFFF1FD0DFFF1F37
:10BAC000606A083800F012F9C0E4C86F083800F066
:10BAD0000DF9FDE4486F083800F008F9F2E4C86E8B
:10BAE000083800F003F9E7E4486E083800F0FEF883
:10BAF000DCE4C86D083800F0F9F8D1E4486D083886
:10BB000000F0F4F8C6E4C86C083800F0EFF8BBE4C5
:10BB1000486C083800F0EAF8B0E4D1F89C00083826
:10BB200000F0E4F8ECE4D1F89400083800F0DEF816
:10BB3000E0E4D1F88C00083800F0D8F8D4E4D1F86B
:10BB40008400083800F0D2F8C8E44FF0020EECE6AA
:10BB50002A78C9F8480001322A705AE62A78C8F8CB
:10BB6000400001322A703FE72A78C9F868000132A4
:10BB70002A705BE62A78C8F8600001322A7061E713
:10BB80002A78C9F8880001322A705BE62A78C4F85E
:10BB9000800001322A7010E72A78C9F828000132A3
:10BBA0002A7028E62A78C9F8200001322A7032E784
:10BBB000BEF1400FF44628BF4FF0400C04EB0C03DD
:10BBC00002930123CCEB0E004FEA0C4800220193B4
:10BBD00018E500BFF8B501F0F9F8294B29482A4CBF
:10BBE0002A4F2B4DDFF8BCC0DFF8BCE0294E002205
:10BBF0001A605A609A60DA601A615A619A61DA6171
:10BC00001A625A629A62DA621A635A639A63DA6350
:10BC10001A645A649A64DA641A655A659A65DA6530
:10BC20001A665A669A66DA661A675A679A67DA6710
:10BC3000C3F880200168C3F8842041F480210160AA
:10BC4000C3F307212170C3F30740134938701B0E5B
:10BC50002B70FF238CF80030104D8EF80030104808
:10BC60000B700123337084F8642070264FF4007445
:10BC7000102207F82C3C2E70046081F8F820F8BDE3
:10BC80000080FF1F348004409C200740B020074004
:10BC9000B4200740942007401020074049E400E00A
:10BCA00008E100E0802007408820074072B60D4878
:10BCB0000268B2FA82F30B2B10DC4FF00041D9403E
:10BCC00022EA0102026062B6074803EBC303DB000D
:10BCD000C2180021C15010465160704762B6002062
:10BCE000704700BFCCA7FF1FBC93FF1F0D4B0E4A30
:10BCF000C31AA2FB03231B090B2B0CD80B4A127887
:10BD000052B972B60A484FF00041026821FA03F3B3
:10BD10001A43026062B67047064A1278002AF0D0D1
:10BD2000FFF74AB9BC93FF1F398EE338D1DFFF1FFD
:10BD3000CCA7FF1FDCDFFF1F38B50F4D286878B197
:10BD400043880288C118013393420C7A02D243809F
:10BD5000204638BDFFF7CAFF002320462B6038BDC0
:10BD6000064B1B782BB10320FFF7F2F82860002860
:10BD7000E6D14FF0FF3038BDF0DFFF1FDCDFFF1FE3
:10BD800010B5094C206818B143881844007A10BDDA
:10BD9000064B1B782BB10320FFF7DAF82060002850
:10BDA000F2D14FF0FF3010BDF0DFFF1FDCDFFF1FCF
:10BDB000044B054A1B6890881BB11A885B88D31A0C
:10BDC00018447047F0DFFF1F7CE1FF1F0B4B1B780F
:10BDD0009BB110B50A4C206848B1FFF787FF0023DC
:10BDE00003202360FFF7B4F830B1FFF77FFF032093
:10BDF000FFF7AEF80028F8D110BD7047DCDFFF1F59
:10BE0000F0DFFF1F2DE9F04FDFF8F89083B001223B
:10BE100089F80020019169B3DFF8EC80364F019E6C
:10BE20008346D8F80000B0B3344D4488C4F14001D3
:10BE3000B14228BF314604EB010E00221FFA8EFEEC
:10BE40002A70761AA0F802E000F1080251B1013C14
:10BE5000224459441BF8014B02F8014F8B45F9D19C
:10BE6000B0F802E0BEF13F0F0BD8254A0521117052
:10BE7000002ED6D10198002389F8003003B0BDE828
:10BE8000F08F4022028001460420FFF7F9F80022DB
:10BE9000C8F80020E9E73A782AB3184D4AF2F924A5
:10BEA0004FF0010A07E0013C16D02A78A2B900F051
:10BEB00007FE3A78BAB10420FFF768F80728F2D8ED
:10BEC00089F800A0FFF7F2FEC8F800000028ACD106
:10BED0000C4B013C1870E8D101234FF0FF302B7060
:10BEE00003B0BDE8F08F00234FF0FF3089F8003039
:10BEF00003B0BDE8F08F00BFDCDFFF1FECDFFF1FEA
:10BF0000E4DFFF1FE5DFFF1FE8DFFF1F00B583B0A1
:10BF100002AB012103F8010D1846FFF773FF03B0D0
:10BF20005DF804FB38B50E4D0E4C286801232370D4
:10BF300028B1408800232370C0F1400038BD0A4B6F
:10BF40001B7813B90020207038BD0420FFF71EF8BD
:10BF50000728F7D8FFF7AAFE28600028E9D1F1E703
:10BF6000E8DFFF1FE5DFFF1FDCDFFF1FF8B5114B28
:10BF70001B788BB1104E114D346801272F7064B1BE
:10BF80000F4A638800271770214623800420FFF79B
:10BF900077F8376000232B70F8BDFFF787FE084B5A
:10BFA00028B1014604201C70FFF76AF8F2E71F7001
:10BFB000F0E700BFDCDFFF1FE8DFFF1FE5DFFF1F4B
:10BFC000E4DFFF1F38B50E4B1B7873B90D4C2168A9
:10BFD00061B103F0FF054B880B800420FFF750F898
:10BFE000256038BD084B01221A7038BDFFF75EFE90
:10BFF0000028F7D00146BDE838400420FFF740B8DC
:10C00000E5DFFF1FE8DFFF1FE4DFFF1FC029F0B4FB
:10C0100028BFC02172B6124B124E134A186000237B
:10C02000138033607360B360F36033617361012721
:10C0300099B15D0903F01F0456F8252007FA04F4AE
:10C04000013322438B4246F82520F2D1002343805E
:10C0500001338B4200F58270F9D162B6F0BC7047B3
:10C0600000E0FF1F08E0FF1F22E0FF1FF0B472B6E0
:10C07000234F244E3C8806F1180306EB84009842B7
:10C0800012D256F8241099B9021D06F11B05631C43
:10C09000AD1A03EB950503E052F8041B41B90133D7
:10C0A000AB421C461046F7D162B60020F0BC704788
:10C0B000B1FA81F34FF00042DA4021EA0201016057
:10C0C00001B9013410493C800A88013294B20C80D5
:10C0D00062B6801B8010C3EB401000EB8010830021
:10C0E0000A480B49006803F5FB531C330125C5546E
:10C0F0000D88AA42184488BF0C80F0BC704700BF6E
:10C1000022E0FF1F08E0FF1F24E0FF1F00E0FF1FE9
:10C11000FCDFFF1F428872B60378012B03D9013B75
:10C12000037062B67047531170B40C4C0C4D54F848
:10C1300023102E88D2434FF0004002F01F0220FA55
:10C1400002F21143074A44F82310B34238BF2B8050
:10C150001388013B138062B670BC704708E0FF1F74
:10C1600022E0FF1F24E0FF1FC368B3B130B401E039
:10C17000DB688BB1187A9042FAD158685C7A006912
:10C1800050F82450002DF3D140F8241008780130E5
:10C190000870DB68002BEDD130BC7047437A8B42CE
:10C1A00006D90369002253F8210043F82120704783
:10C1B0000020704738B5437A8B421AD9036953F887
:10C1C0002140002243F821209CB12378012B0ED975
:10C1D000FFF74CFF054628B14FF48072211D043053
:10C1E000FEF7D8F82378013B2370284638BD204657
:10C1F00038BD002038BD00BF037C23BB4368427AB2
:10C200005B7A9A421FD830B472B60468E3682BB3E5
:10C21000DA6832B119688C4216D01346DA68002AFF
:10C22000F8D1D8600023C360A37A0133A3720268F7
:10C230004168012313728A7A1A448A72426813721F
:10C24000037462B630BC70475D6841688D42E4D1CA
:10C25000198903899942F4D01346DFE7E060E1E7EA
:10C26000037C10B5002B32D04368427A5B7A9A4245
:10C270002DD872B60268D36843B3984202D129E040
:10C28000984202D0DB68002BFAD14368417A1B69DF
:10C29000044653F8210048B1FFF73CFF72B66368CB
:10C2A000627A1B69002143F822102268937A013BCD
:10C2B000937223689A7A02B91A726268937A013B80
:10C2C000937263689A7A1AB10023237462B610BD20
:10C2D0001A72F9E7C368D360D7E700BF084B1A7832
:10C2E00062B930B407480849D02505704FF0804442
:10C2F00001220C6010461A7030BC70470020704755
:10C3000004E0FF1F5EE400E008E100E01A491B4A78
:10C310001B48F8B50B681B4D046843F080730B6035
:10C32000136843F0010313602E6814B915E06469C3
:10C330009CB1237A002BFAD023682F681B68204613
:10C3400098472B68E188DB1B1B099AB28B42A280BD
:10C3500088BFE2806469002CEBD10A4B0A4A1B6853
:10C3600010880A4C9B1B1B0999B28342218001D97A
:10C370001180F8BDF8BD00BFFCED00E0001000E04A
:10C38000F8DFFF1F041000E020E0FF1F26E0FF1F82
:10C39000F0B572B699B902688AB103790F2B0ED83D
:10C3A000274C218841FA03F5ED070AD503F1007304
:10C3B00003F59063B2EB431F03D162B6F0BD204C8E
:10C3C0002188002341FA03F212F0010207D0013361
:10C3D000102BF7D162B6002203710260F0BD012577
:10C3E0009D402943218062B6164E174D174FDFF846
:10C3F00064E0D9B20171346844F0020434602C68FE
:10C4000044F002042C60A6F580268224A5F5802540
:10C4100003F100733C6003F59063223E243D0C4C15
:10C420008EF800105B0131702970217003601A6072
:10C430005A609A60DA601A615A619A61DA61F0BDF5
:10C4400028E0FF1F408004403C8004400080004002
:10C450001F8000401A80004003790F2B11D8094A31
:10C4600010B4137072B6084904790A880123A340F6
:10C4700022EA03030B8062B61022002310BC027173
:10C48000036070471A80004028E0FF1F10B4EFF3EC
:10C49000108272B6437F33B9017F012907D0032987
:10C4A0000FD00123437702B962B610BC7047124C1B
:10C4B0002168A1B1114943610B688361086058612B
:10C4C000EFE70F4C216881B10E4943610B6883612E
:10C4D000086058610C4B4FF080511960E1E7074B41
:10C4E0004161816120601860DBE7064B4161816139
:10C4F00020601860EEE700BF3CE0FF1F38E0FF1F40
:10C500002CE0FF1F30E0FF1F04ED00E070B5EFF3FB
:10C51000108272B60C4C206880B10C4E0025436925
:10C52000236073B19D6102B962B64577836898470D
:10C53000EFF3108272B620680028F0D102B962B61B
:10C5400070BD3360EFE700BF2CE0FF1F30E0FF1F3E
:10C55000FFF7DCBF184A30B41468002C27D00368FA
:10C5600021688B420ED2CB1A00218460C160236007
:10C57000E06010600223037530BC704711688B4285
:10C58000144608D3A2685B1A0360002AF6D18260C1
:10C59000C460A060EEE7D268C2608460E060C568F5
:10C5A000CB1A0222A8602360027530BC70478460F9
:10C5B000C4601060DEE700BF34E0FF1FF8B5224E14
:10C5C00034682CB32368002B3AD1204F1D4604E079
:10C5D0003468ECB12368002B32D1A36803B1DD606D
:10C5E00020693360036825751B68BB4221D1037F36
:10C5F0004560022BC46020D0FFF748FF6368002B22
:10C60000E6D023602046FFF7A5FF3468002CE1D177
:10C61000EFF3108372B60E4A00211068116003B95F
:10C6200062B628B18468FFF795FF20460028F9D14B
:10C63000F8BD224600219847E0E783689847DDE788
:10C64000013B2360E4E700BF34E0FF1F4D820000A0
:10C6500044E0FF1F024A136801331360FFF7AEBFC7
:10C6600060DEFF1F2DE9F0438C688BB0ECB1002534
:10C67000064689462F462B46212201A9484600F04E
:10C68000E7F93268202C234628BF2023D2F8048003
:10C6900001A91A4630461D44E41AC0470744002C3D
:10C6A000E9D138460BB0BDE8F0832746F9E700BF73
:10C6B00000B5064A036812885B6883B001A9ADF82B
:10C6C00004200222984703B05DF804FB94070100A0
:10C6D000F0B507468BB0002A33D0012A08BF0A22E2
:10C6E00051B3212400E0F4B2B1FBF2F502FB1511C5
:10C6F000C8B2092900F1300198BFC8B20AA988BFA1
:10C700003730214488BFC0B201F8240C661E294688
:10C71000002DE8D133B1013CE4B20AAB23442D2211
:10C7200003F8242C3B6801AA11195B683846C4F150
:10C73000220298470BB0F0BD30228DF8252021242D
:10C74000E8E70368C9B21B6898470BB0F0BD00BFAB
:10C750000029BABF49422D2300230A22FFF7B8BFA0
:10C760002DE9F04385B080461946104616461F460F
:10C770009DF8305000F0C4FF002840F0B18027F051
:10C780000044304621464FF0FF32594B00F0B8FFCD
:10C7900098B9304621464FF0FF32554B00F092FFDA
:10C7A00058B9D8F8003053495B684046032298478F
:10C7B0008146484605B0BDE8F083304639464FF023
:10C7C00060424D4B00F092FF002870D13046394650
:10C7D0004FF06042494B00F06BFF002867D13046B4
:10C7E00039460022002300F063FF002863D1814610
:10C7F000002D65D0424B00240022104619463AA372
:10C80000D3E9002300F0E2FC01340B46E1B28D4293
:10C810000246F2D83046394600F026FB0F4606465F
:10C8200000F084FF044600F05BFC02460B463046F5
:10C83000394600F017FB4B4606460F460A222146B2
:10C840004046FFF745FF0F2D28BF0F2501352E234A
:10C850008146EDB28DF8003001240022294B30468C
:10C86000394600F0B3FC0F46064600F05FFF04AB0C
:10C870002344C0B200F1300203F8102C00F040FC59
:10C8800002460B463046394600F0ECFA0134E4B279
:10C89000AC4206460F46E0D1D8F8003022465B682D
:10C8A000404669469847484605B0BDE8F083D8F849
:10C8B0000030154978E707F100474FF0010997E785
:10C8C00000220F4B3046394600F0CEFA00F02EFF22
:10C8D0004B4601460A224046FFF7FAFE814668E7CA
:10C8E000D8F8003009495FE7000000A09999B93FE6
:10C8F000FFFFEF7FA0070100FFFFEF41FFFFEFC148
:10C900000000E03F000024409C0701009807010060
:10C91000F0B5164D2A680AB31549164BDFF85CE0EE
:10C9200082FB016781FB0214D617D1191444C6EBB0
:10C930002141C6EB244403FB04F40EFB112244F214
:10C94000A71303FB0243002B02DA03F10043013B70
:10C95000B3FBF0F22B6000FB1230F0BD064B2B60F6
:10C96000B3FBF0F200FB1230F0BD00BF48E0FF1F48
:10C970005F0B4E83ECF4FFFF42CE0C1F1DF3010052
:10C9800008B1014B1860704748E0FF1F08B1FFF77E
:10C99000BFBF7047884206DA10B50446081AFFF791
:10C9A000B7FF204410BD704710B50446006801F081
:10C9B0007FFA204610BD00BF38B543688B4201D3D3
:10C9C000012038BD0D4604460131006801F02EFEFD
:10C9D0000028F6D0A36884E82100002BF0D1037072
:10C9E000EEE700BFF8B50446154632B9036803B157
:10C9F0001A700023A3602046F8BD0E461146FFF7CB
:10CA0000DBFF074648B9206810B101F051FA2760F2
:10CA100000236360A3602046F8BDA560314620680E
:10CA200002F00CFAE7E700BF38B5002304460360C4
:10CA300043608360037341B108460D4602F060FA1B
:10CA4000294602462046FFF7CDFF204638BD00BFED
:10CA5000B2B1A9B138B584689C420ED9E41A013A42
:10CA60000D469442016828BF1446194422462846C0
:10CA700002F0B4FA00232B5538BD00230B7038BDEB
:10CA8000704700BF08B5F8F76BFFF9F779F900F0C8
:10CA900017F8FAE7FFF79AB9FFF772B9FFF74CB941
:10CAA000FFF786B9FFF762BAFFF73CBA08461146AE
:10CAB000FFF7A8B90846FFF729BA00BF704700BFC3
:10CAC00038B5224C237803B138BD01232370FFF71A
:10CAD0006FF970BBFEF772F940BB00F065F810BB50
:10CAE00000F0F8F8E0B900232370EFF30583002B82
:10CAF000EAD1EFF3108172B6154B1868E0B1154C0E
:10CB00002278CAB945691D6001232370C5B1AA61A5
:10CB100001B962B600254577836898472570D3E749
:10CB200000F09AF9DFE700F095F9D9E700F090F905
:10CB3000D3E7FFF7C3FFCDE70029C5D162B638BD03
:10CB4000054B1D600029E5D1E3E700BF4DE0FF1F65
:10CB50003CE0FF1F40E0FF1F38E0FF1FF0B44D1E18
:10CB60002E46002400E00134B0FBF2F302FB130078
:10CB7000092800F130078ABF3730F8B2C0B206F892
:10CB8000010F1846002BEED10A1953704CB11078E2
:10CB900015F8016F28700133E01A834202F8016929
:10CBA000F5DB0846F0BC7047054A064B10781B7849
:10CBB000C0B2DBB2984238BF4030C01A704700BFE5
:10CBC000C0E0FF1F55E0FF1FF0B4384B1A7912F098
:10CBD000300F2CD072B6997D01F0FF0200293DD0B4
:10CBE00062B6334F334938780D78334E1C46C0B2A5
:10CBF000EDB2431C402BE17928BF0023AB4202F188
:10CC0000FF32C9B21CBFF154184612F0FF02F0D136
:10CC10002A4B1B68C2B23A704BB1A84236BFC5F16D
:10CC20004005401B40192728C4BF01221A701F4924
:10CC3000CA78D2B2150616D452060DD51B4B1B79F5
:10CC40005B0609D51E4B1F491B6800220A7003B101
:10CC50001A70164B3C22DA70F0BC70474022D9792A
:10CC60005A7462B6E3E70B791C06E5D5164B174EEE
:10CC70001C783378E4B2DBB29C420ED0144D01E054
:10CC8000A3420AD00133282B28BF00230879E85C8F
:10CC9000C0B2C871087D0728F2D9DBB203493370EE
:10CCA0000B79180644BF7C23CB70C5E700B0064063
:10CCB000C0E0FF1F55E0FF1F80E0FF1F50E0FF1F97
:10CCC000C4E0FF1F54E0FF1FC8E0FF1FC1E0FF1FCB
:10CCD00058E0FF1F054A064B10781B78C0B2DBB244
:10CCE000984238BF4030C01A704700BFD0E0FF1FE5
:10CCF000D1E0FF1F30B42B4B1A7994061FD52A4878
:10CD0000DA790378294901333F2B0978C8BF00231A
:10CD10008B42D2B203D0264CD9B2E2540170254ADC
:10CD2000116861B1244A1278D2B2934236BFC2F17F
:10CD300040029B1A9B18272BC4BF01230B70194A72
:10CD4000D378DBB2180611D45A060DD5154B1B79D2
:10CD50005B0609D5194B1A491B6800220A7003B1FA
:10CD60001A70104B2C22DA7030BC7047117909060A
:10CD7000EAD5144910480C780178C9B28C420DD01C
:10CD80004A1C272A84BF00210A460F4D054C98BF34
:10CD9000D1B2AA5CD2B2E2710170D5E76C21D17038
:10CDA000D2E700BF00C00640D0E0FF1FD1E0FF1F68
:10CDB000FCE0FF1FCCE0FF1F3DE1FF1F40E1FF1F34
:10CDC0003CE1FF1F44E1FF1FD4E0FF1F70B584B0BA
:10CDD00072B6194B194D1A48702241260F24802132
:10CDE0001A702E701A460470197013781B06FCD541
:10CDF000144B186862B6144B144C984298BF00EB61
:10CE0000800001A998BF40000A22FFF7A7FE01A9F0
:10CE10002046002311F8012B01333AB10A2B20F8E8
:10CE2000022FF7D11623237004B070BD5B00DBB274
:10CE3000237004B070BD00BF000002400700024034
:10CE400006000240080002407F9698006CA8FF1F71
:10CE5000704700BF704700BF704700BF81F00041BE
:10CE600002E000BF83F0004330B54FEA41044FEACF
:10CE7000430594EA050F08BF90EA020F1FBF54EA6A
:10CE8000000C55EA020C7FEA645C7FEA655C00F006
:10CE9000E2804FEA5454D4EB5555B8BF6D420CDDD7
:10CEA0002C4480EA020281EA030382EA000083EA5A
:10CEB000010180EA020281EA0303362D88BF30BDFA
:10CEC00011F0004F4FEA01314FF4801C4CEA113150
:10CED00002D0404261EB410113F0004F4FEA0333AF
:10CEE0004CEA133302D0524263EB430394EA050F3A
:10CEF00000F0A780A4F10104D5F1200E0DDB02FAA9
:10CF00000EFC22FA05F2801841F1000103FA0EF23C
:10CF1000801843FA05F359410EE0A5F120050EF102
:10CF2000200E012A03FA0EFC28BF4CF0020C43FA33
:10CF300005F3C01851EBE37101F0004507D54FF040
:10CF4000000EDCF1000C7EEB00006EEB0101B1F590
:10CF5000801F1BD3B1F5001F0CD349085FEA3000D6
:10CF60004FEA3C0C04F101044FEA445212F5800FE1
:10CF700080F09A80BCF1004F08BF5FEA500C50F17E
:10CF8000000041EB045141EA050130BD5FEA4C0C61
:10CF9000404141EB010111F4801FA4F10104E9D1EA
:10CFA00091F0000F04BF01460020B1FA81F308BFE1
:10CFB0002033A3F10B03B3F120020CDA0C3208DDAD
:10CFC00002F1140CC2F10C0201FA0CF021FA02F188
:10CFD0000CE002F11402D8BFC2F1200C01FA02F1F8
:10CFE00020FA0CFCDCBF41EA0C019040E41AA2BF1D
:10CFF00001EB0451294330BD6FEA04041F3C1CDAE5
:10D000000C340EDC04F11404C4F1200220FA04F004
:10D0100001FA02F340EA030021FA04F345EA0301AE
:10D0200030BDC4F10C04C4F1200220FA02F001FA70
:10D0300004F340EA0300294630BD21FA04F02946F2
:10D0400030BD94F0000F83F4801306BF81F480118B
:10D050000134013D4EE77FEA645C18BF7FEA655CFE
:10D0600029D094EA050F08BF90EA020F05D054EAD0
:10D07000000C04BF1946104630BD91EA030F1EBFD5
:10D080000021002030BD5FEA545C05D140004941D9
:10D0900028BF41F0004130BD14F580043CBF01F5CC
:10D0A000801130BD01F0004545F0FE4141F47001B2
:10D0B0004FF0000030BD7FEA645C1ABF194610468D
:10D0C0007FEA655C1CBF0B46024650EA013406BF8E
:10D0D00052EA033591EA030F41F4002130BD00BF4D
:10D0E00090F0000F04BF0021704730B54FF480640A
:10D0F00004F132044FF000054FF0000150E700BF8B
:10D1000090F0000F04BF0021704730B54FF48064E9
:10D1100004F1320410F0004548BF40424FF00001D6
:10D120003EE700BF42004FEAE2014FEA31014FEA19
:10D1300002701FBF12F07F4393F07F4F81F0605168
:10D14000704792F0000F14BF93F07F4F704730B5D7
:10D150004FF4607401F0004521F0004120E700BF6A
:10D1600050EA010208BF704730B54FF000050AE0F1
:10D1700050EA010208BF704730B511F0004502D5F2
:10D18000404261EB41014FF4806404F132045FEAF4
:10D19000915C3FF4DCAE4FF003025FEADC0C18BF99
:10D1A00003325FEADC0C18BF033202EBDC02C2F18F
:10D1B000200300FA03FC20FA02F001FA03FE40EA21
:10D1C0000E0021FA02F11444C1E600BF70B54FF021
:10D1D000FF0C4CF4E06C1CEA11541DBF1CEA135503
:10D1E00094EA0C0F95EA0C0F00F0DEF82C4481EA6B
:10D1F000030621EA4C5123EA4C5350EA013518BF8B
:10D2000052EA033541F4801143F4801338D0A0FB77
:10D2100002CE4FF00005E1FB02E506F00042E0FB24
:10D2200003E54FF00006E1FB03569CF0000F18BF2A
:10D230004EF0010EA4F1FF04B6F5007F64F54074D2
:10D2400004D25FEA4E0E6D4146EB060642EAC62165
:10D2500041EA55514FEAC52040EA5E504FEACE2ED2
:10D26000B4F1FD0C88BFBCF5E06F1ED8BEF1004FD5
:10D2700008BF5FEA500E50F1000041EB045170BD51
:10D2800006F0004646EA010140EA020081EA030195
:10D29000B4EB5C04C2BFD4EB0C0541EA045170BD91
:10D2A00041F480114FF0000E013C00F3AB8014F10B
:10D2B000360FDEBF002001F0004170BDC4F1000454
:10D2C000203C35DA0C341BDC04F11404C4F12005D5
:10D2D00000FA05F320FA04F001FA05F240EA020030
:10D2E00001F0004221F0004110EBD37021FA04F666
:10D2F00042EB06015EEA430E08BF20EAD37070BD20
:10D30000C4F10C04C4F1200500FA04F320FA05F07E
:10D3100001FA04F240EA020001F0004110EBD37080
:10D3200041F100015EEA430E08BF20EAD37070BDF0
:10D33000C4F1200500FA05F24EEA020E20FA04F3C9
:10D3400001FA05F243EA020321FA04F001F0004178
:10D3500021FA04F220EA020000EBD3705EEA430EE9
:10D3600008BF20EAD37070BD94F0000F0FD101F018
:10D370000046400041EB010111F4801F08BF013C51
:10D38000F7D041EA060195F0000F18BF704703F08F
:10D390000046520043EB030313F4801F08BF013D16
:10D3A000F7D043EA0603704794EA0C0F0CEA1355D2
:10D3B00018BF95EA0C0F0CD050EA410618BF52EA8C
:10D3C0004306D1D181EA030101F000414FF0000092
:10D3D00070BD50EA410606BF1046194652EA4306A0
:10D3E00019D094EA0C0F02D150EA013613D195EA14
:10D3F0000C0F05D152EA03361CBF104619460AD15C
:10D4000081EA030101F0004141F0FE4141F4700165
:10D410004FF0000070BD41F0FE4141F4780170BD55
:10D4200070B54FF0FF0C4CF4E06C1CEA11541DBFBA
:10D430001CEA135594EA0C0F95EA0C0F00F0A7F8BC
:10D44000A4EB050481EA030E52EA03354FEA0131E9
:10D4500000F088804FEA03334FF0805545EA1313FC
:10D4600043EA12634FEA022245EA111545EA1065C4
:10D470004FEA00260EF000419D4208BF964244F15B
:10D48000FD0404F5407402D25B084FEA3202B61A7A
:10D4900065EB03055B084FEA32024FF480104FF44E
:10D4A000002CB6EB020E75EB030E22BFB61A7546C2
:10D4B00040EA0C005B084FEA3202B6EB020E75EB55
:10D4C000030E22BFB61A754640EA5C005B084FEABD
:10D4D0003202B6EB020E75EB030E22BFB61A75468A
:10D4E00040EA9C005B084FEA3202B6EB020E75EB95
:10D4F000030E22BFB61A754640EADC0055EA060E56
:10D5000018D04FEA051545EA16754FEA06164FEA98
:10D51000C30343EA52734FEAC2025FEA1C1CC0D144
:10D5200011F4801F0BD141EA00014FF000004FF0D1
:10D53000004CB6E711F4801F04BF01430020B4F192
:10D54000FD0C88BFBCF5E06F3FF6AFAEB5EB030C4A
:10D5500004BFB6EB020C5FEA500C50F1000041EB47
:10D56000045170BD0EF0004E4EEA113114EB5C0414
:10D57000C2BFD4EB0C0541EA045170BD41F48011E7
:10D580004FF0000E013C90E645EA060E8DE60CEAEF
:10D59000135594EA0C0F08BF95EA0C0F3FF43BAF0C
:10D5A00094EA0C0F0AD150EA01347FF434AF95EAC3
:10D5B0000C0F7FF425AF104619462CE795EA0C0FA7
:10D5C00006D152EA03353FF4FDAE1046194622E774
:10D5D00050EA410618BF52EA43067FF4C5AE50EA4E
:10D5E00041047FF40DAF52EA43057FF4EBAE12E73E
:10D5F0004FF0FF3C06E000BF4FF0010C02E000BF1F
:10D600004FF0010C4DF804CD4FEA410C7FEA6C5C01
:10D610004FEA430C18BF7FEA6C5C1BD001B050EAA4
:10D62000410C0CBF52EA430C91EA030F02BF90EA8F
:10D63000020F0020704710F1000F91EA030F58BF4E
:10D64000994208BF90422CBFD8176FEAE37040F0B0
:10D65000010070474FEA410C7FEA6C5C02D150EA4E
:10D66000013C07D14FEA430C7FEA6C5CD6D152EA09
:10D67000033CD3D05DF8040B704700BF84461046CE
:10D6800062468C461946634600E000BF01B5FFF7CD
:10D69000B7FF002848BF10F1000F01BD4DF808ED9D
:10D6A000FFF7F4FF0CBF012000205DF808FB00BF6E
:10D6B0004DF808EDFFF7EAFF34BF012000205DF8C8
:10D6C00008FB00BF4DF808EDFFF7E0FF94BF012015
:10D6D00000205DF808FB00BF4DF808EDFFF7CEFF16
:10D6E00094BF012000205DF808FB00BF4DF808ED55
:10D6F000FFF7C4FF34BF012000205DF808FB00BF26
:10D700004FEA410C7FEA6C5C02D150EA013C0AD13D
:10D710004FEA430C7FEA6C5C02D152EA033C02D12F
:10D720004FF0000070474FF0010070474A0011D2DF
:10D7300012F5001211D20DD56FF47873B3EB62526B
:10D740000ED44FEAC12343F0004343EA505323FA77
:10D7500002F070474FF00000704750EA013002D1EC
:10D760004FF0FF3070474FF00000704780F00040EE
:10D7700002E000BF81F0004142001FBF5FEA4103A9
:10D7800092EA030F7FEA226C7FEA236C6AD04FEAA9
:10D790001262D2EB1363C1BFD218414048404140EE
:10D7A000B8BF5B42192B88BF704710F0004F40F4A0
:10D7B000000020F07F4018BF404211F0004F41F4BC
:10D7C000000121F07F4118BF494292EA030F3FD088
:10D7D000A2F1010241FA03FC10EB0C00C3F120039B
:10D7E00001FA03F100F0004302D5494260EB40002A
:10D7F000B0F5000F13D3B0F1807F06D340084FEA95
:10D80000310102F10102FE2A51D2B1F1004F40EB89
:10D81000C25008BF20F0010040EA030070474900F1
:10D8200040EB000010F4000FA2F10102EDD1B0FABC
:10D8300080FCACF1080CB2EB0C0200FA0CF0AABFB1
:10D8400000EBC25052421843BCBFD040184370474F
:10D8500092F0000F81F4000106BF80F40000013255
:10D86000013BB5E74FEA41037FEA226C18BF7FEA2C
:10D87000236C21D092EA030F04D092F0000F08BF6E
:10D880000846704790EA010F1CBF0020704712F055
:10D890007F4F04D1400028BF40F00040704712F194
:10D8A00000723CBF00F50000704700F0004343F0F9
:10D8B000FE4040F4000070477FEA226216BF08462F
:10D8C0007FEA23630146420206BF5FEA412390EAF2
:10D8D000010F40F4800070474FF0000304E000BFE8
:10D8E00010F0004348BF40425FEA000C08BF704799
:10D8F00043F0964301464FF000001CE050EA01025D
:10D9000008BF70474FF000030AE000BF50EA010271
:10D9100008BF704711F0004302D5404261EB41015E
:10D920005FEA010C02BF84460146002043F0B64383
:10D9300008BFA3F18053A3F50003BCFA8CF2083AA8
:10D94000A3EBC25310DB01FA02FC634400FA02FCB1
:10D95000C2F12002BCF1004F20FA02F243EB0200B8
:10D9600008BF20F00100704702F1200201FA02FC1A
:10D97000C2F1200250EA4C0021FA02F243EB02000D
:10D9800008BF20EADC7070474FF0FF0C1CEAD05251
:10D990001EBF1CEAD15392EA0C0F93EA0C0F6FD012
:10D9A0001A4480EA010C400218BF5FEA41211ED0F0
:10D9B0004FF0006343EA501043EA5111A0FB0131DC
:10D9C0000CF00040B1F5000F3EBF490041EAD371B1
:10D9D0005B0040EA010062F17F02FD2A1DD8B3F12D
:10D9E000004F40EBC25008BF20F00100704790F09C
:10D9F000000F0CF0004C08BF49024CEA502040EAEE
:10DA000051207F3AC2BFD2F1FF0340EAC2507047B3
:10DA100040F400004FF00003013A5DDC12F1190FF1
:10DA2000DCBF00F000407047C2F10002410021FA63
:10DA300002F1C2F1200200FA02FC5FEA310040F17B
:10DA4000000053EA4C0308BF20EADC70704792F0F4
:10DA5000000F00F0004C02BF400010F4000F013A2C
:10DA6000F9D040EA0C0093F0000F01F0004C02BF27
:10DA7000490011F4000F013BF9D041EA0C018FE796
:10DA80000CEAD15392EA0C0F18BF93EA0C0F0AD09C
:10DA900030F0004C18BF31F0004CD8D180EA0100C2
:10DAA00000F00040704790F0000F17BF90F0004F5B
:10DAB000084691F0000F91F0004F14D092EA0C0F3D
:10DAC00001D142020FD193EA0C0F03D14B0218BFD0
:10DAD000084608D180EA010000F0004040F0FE4016
:10DAE00040F40000704740F0FE4040F440007047B2
:10DAF0004FF0FF0C1CEAD0521EBF1CEAD15392EA31
:10DB00000C0F93EA0C0F69D0A2EB030280EA010C20
:10DB100049024FEA402037D04FF0805343EA1111B9
:10DB200043EA10130CF000408B4238BF5B0042F117
:10DB30007D024FF4000C8B4224BF5B1A40EA0C00BC
:10DB4000B3EB510F24BFA3EB510340EA5C00B3EBEE
:10DB5000910F24BFA3EB910340EA9C00B3EBD10FDC
:10DB600024BFA3EBD10340EADC001B0118BF5FEA2E
:10DB70001C1CE0D1FD2A3FF650AF8B4240EBC25057
:10DB800008BF20F0010070470CF0004C4CEA502018
:10DB90007F32C2BFD2F1FF0340EAC250704740F467
:10DBA00000004FF00003013A37E792F0000F00F059
:10DBB000004C02BF400010F4000F013AF9D040EAD7
:10DBC0000C0093F0000F01F0004C02BF490011F46B
:10DBD000000F013BF9D041EA0C0195E70CEAD15363
:10DBE00092EA0C0F08D142027FF47DAF93EA0C0F4A
:10DBF0007FF470AF084676E793EA0C0F04D14B022E
:10DC00003FF44CAF08466EE730F0004C18BF31F0DF
:10DC1000004CCAD130F000427FF45CAF31F00043D9
:10DC20007FF43CAF5FE700BF4FF0FF3C06E000BF72
:10DC30004FF0010C02E000BF4FF0010C4DF804CD95
:10DC40004FEA40024FEA41037FEA226C18BF7FEAA5
:10DC5000236C11D001B052EA530C18BF90EA010FA7
:10DC600058BFB2EB030088BFC81738BF6FEAE17036
:10DC700018BF40F0010070477FEA226C02D15FEAD2
:10DC8000402C05D17FEA236CE4D15FEA412CE1D03E
:10DC90005DF8040B704700BF844608466146FFE705
:10DCA0000FB5FFF7C9FF002848BF10F1000F0FBDE7
:10DCB0004DF808EDFFF7F4FF0CBF012000205DF8E0
:10DCC00008FB00BF4DF808EDFFF7EAFF34BF012065
:10DCD00000205DF808FB00BF4DF808EDFFF7E0FFFE
:10DCE00094BF012000205DF808FB00BF4DF808ED4F
:10DCF000FFF7D2FF94BF012000205DF808FB00BFB2
:10DD00004DF808EDFFF7C8FF34BF012000205DF893
:10DD100008FB00BF4FEA4002B2F1FE4F0FD34FF0B5
:10DD20009E03B3EB12620DD94FEA002343F0004388
:10DD300010F0004F23FA02F018BF404270474FF036
:10DD40000000704712F1610F01D1420205D110F0BD
:10DD5000004008BF6FF0004070474FF00000704770
:10DD600042000ED2B2F1FE4F0BD34FF09E03B3EB45
:10DD7000126209D44FEA002343F0004323FA02F071
:10DD800070474FF00000704712F1610F01D142025D
:10DD900002D14FF0FF3070474FF00000704700BFD6
:10DDA0000B460146184600F009B800BF0A220021C0
:10DDB00001F0E4B90A22002101F0E0B913460A4655
:10DDC0000146022001F008BB014B1868704700BFF4
:10DDD000B0ACFF1F70B50F4E0F4D761BB61018BFBD
:10DDE000002405D0013455F8043B9847A642F9D1E8
:10DDF0000A4E0B4D761B02F0B3FDB61018BF00247F
:10DE000006D0013455F8043B9847A642F9D170BDBD
:10DE100070BD00BF6C0901006C090100B809010068
:10DE20006C09010010B5044600F030F82044407839
:10DE300000F0080010BD00BF931E222B10D80A2A44
:10DE400010B506D000230C46194401F077FA20469D
:10DE500010BD0028F6DA2D230B7040420123F2E7B3
:10DE600000200870704700BFFFF7E6BF034A044B6D
:10DE70001268506B002808BF18467047B0ACFF1FEF
:10DE8000B4ACFF1FD0F8EC00704700BF08B5034BDF
:10DE90001868FFF7EBFFD0F8EC0008BDB0ACFF1F2F
:10DEA000024B0146186800F00BB800BFB0ACFF1F72
:10DEB000024B0146186801F053BB00BFB0ACFF1F16
:10DEC0002DE9F04F01F10B05162D83B0064640F207
:10DED0009F8035F0070500F1BF80A94200F2BC80A9
:10DEE00000F0A0FBB5F5FC7FC0F09C826B0A00F04F
:10DEF000BA80042B00F28381A80900F1390E4FEAA1
:10DF00004E033830C44F07EB8303A3F108015C686C
:10DF1000A14207D1ACE0002A80F2AC80E468A142C3
:10DF200000F0A680636823F003035A1B0F2AF2DD7A
:10DF3000B9493C6901F1080E744500F0B38163688A
:10DF400023F003035A1B0F2A00F39981002AC1F81A
:10DF500014E0C1F810E080F29E80B3F5007F80F0FD
:10DF60006781DB0803F1010C01229B1002FA03F325
:10DF70004A6851F83C80C4F8088001EBCC091A4388
:10DF8000A9F10803E3604A6041F83C40C8F80C403E
:10DF9000831001249C40944200F28A80144206D1EE
:10DFA00020F003006400144200F10400FAD007EBF3
:10DFB000C009CC468046DCF80C108C4507D173E1D3
:10DFC000002A80F28181C9688C4500F06D814B6820
:10DFD00023F003035A1B0F2AF2DD0C46D1F80CC0C4
:10DFE00054F8088F4B1945F001054D6042F00101CE
:10DFF000C8F80CC03046CCF808807B613B61C3F8A0
:10E000000CE0C3F808E059609A5000F00DFB1FE0E7
:10E01000102921D800F006FB1025062302207E4F90
:10E0200007EB8303A3F108025C68944200F045818A
:10E030006368E168A56823F00303234430465A6807
:10E04000E96042F001028D605A6000F0EDFA083498
:10E05000204603B0BDE8F08F00240C232046336037
:10E0600003B0BDE8F08F80234FF0400E3F2049E71A
:10E0700070465DE72344E1685A68A56842F00102F2
:10E08000E96030468D605A6000F0CEFA08342046D0
:10E0900003B0BDE8F08F234430465A6842F00102D5
:10E0A0005A6000F0C1FA0834204603B0BDE8F08F92
:10E0B000BC68636823F00308A84504D3C5EB0803D4
:10E0C0000F2B00F38C80554BDFF860911A68D9F85C
:10E0D000003001332A4404EB080A00F0608102F5A5
:10E0E00080520F3222F47F6222F00F021146304636
:10E0F000019200F093FCB0F1FF3F8346019A00F0DB
:10E100005881824500F2FC80454B1968DA4511447C
:10E11000196000F05381D9F80000DFF810E10130F8
:10E120001BBFCAEB0B0A5144CEF800B019601BF0BC
:10E13000070100F01781C1F10800C1F58051834447
:10E1400008315A44C2F30B02C2EB0109494630467A
:10E15000019300F063FC431C019B00F03F81CBEB7B
:10E1600000024A4442F001021968C7F808B0494465
:10E17000BC42CBF804201960DFF8A49016D0B8F1A7
:10E180000F0F40F2FD806268A8F10C0323F0070333
:10E19000E01802F001024FF0050E1A430F2B6260E7
:10E1A000C0F804E0C0F808E000F21C811D4BBC6818
:10E1B0001A68914288BF19601B4B1A6891426268C5
:10E1C00088BF196022F003029542A2EB050301D833
:10E1D0000F2B04DC304600F027FA002438E76219E0
:10E1E00043F0010345F0010565603046BA605360B5
:10E1F00000F01AFA0834204603B0BDE8F08F142B63
:10E2000071D9542B00F2A480280B00F16F0E4FEA55
:10E210004E036E3076E600BF20AEFF1F50E1FF1FB9
:10E2200054E1FF1F4CE1FF1F48E1FF1F2CB2FF1F0D
:10E230005A0A042A5ED9142A00F2B38002F15C0162
:10E2400049005B3207EB810C57F82110DFF8DC81C5
:10E25000ACF1080C8C4500F088804A6822F003027B
:10E26000934202D289688C45F7D1D1F80CC07A6804
:10E27000C4F80CC0A160CCF80840CC6088E66319F3
:10E2800042F0010745F00105656030464B610B61C6
:10E29000C3F80CE0C3F808E05F609A50083400F05F
:10E2A000C3F9D5E64A6873E608F1010818F0030FD0
:10E2B0000CF1080C7FF47FAE30E0DC68A34208BFAD
:10E2C00002303FF435AEB3E60B440C465A68C968D9
:10E2D00054F8085F42F001025A603046E9608D60F0
:10E2E00000F0A2F9B4E603F15C0E03F15B004FEA23
:10E2F0004E0307E69A0902F1390149003832A1E7D5
:10E30000BC424A4B3FF400AF9C68626822F00302B3
:10E310005AE759F80839994540F0828010F0030F08
:10E3200000F1FF30F5D17B6823EA04037B606400D1
:10E330009C423FF6BDAE002C3FF4BAAE1C424046B4
:10E340007FF435AE64001C4200F10400FAD02EE6E2
:10E35000B3F5AA7F18D8E80B00F1780E4FEA4E0308
:10E360007730CFE54FF48051EBE60121D8F8043047
:10E37000921001FA02F21A43C8F80420614677E7C6
:10E380000123CBF8043025E740F25452934220D8C1
:10E39000A80C00F17D0E4FEA4E037C30B2E510323E
:10E3A000A4E6542A26D81A0B02F16F0149006E32F6
:10E3B00048E7BC68626822F0030205E7CAF30B0075
:10E3C00000287FF4A8AE4244BB6842F001025A60C4
:10E3D000ECE6FE234FF07F0E7E2093E501224FF006
:10E3E0000009C1E604F10801304601F0B9F8D9F896
:10E3F0000010DBE6B2F5AA7F05D8DA0B02F178014E
:10E40000490077321EE740F254518A4205D89A0CEF
:10E4100002F17D0149007C3214E7FE217E2211E7E2
:10E420007B6884E7E808431C5B00F8E520AEFF1F2B
:10E4300082B049B15AB16BB113780B601278101CDD
:10E4400018BF012002B0704701A9002AF3D110467D
:10E4500002B070476FF00100F4E700BF032A70B408
:10E4600026D940EA01039B0711D004780D78AC420D
:10E4700022D10244431C05E013F8014B11F8015F5F
:10E48000AC4219D19342F7D1002070BC70470C46C2
:10E4900003461E682568AE421846214603F1040370
:10E4A00004F10404E1D1043A032A18462146F0D8C5
:10E4B000002ADAD11046E8E7601B70BC704700BF45
:10E4C0008842F0B50DD98B1898420AD28118002ADB
:10E4D00051D09A1A13F8014D01F8014D9342F9D128
:10E4E000F0BD0F2A48D941EA00039B0746D100F14D
:10E4F000100401F11003154653F8106C44F8106C29
:10E5000053F80C6C44F80C6C53F8086C44F8086C25
:10E51000103D53F8046C44F8046C0F2D03F1100304
:10E5200004F11004E8D8A2F1100323F00F0302F065
:10E530000F0E1033BEF1030F1944034421D91E1FDF
:10E540000D467446043C55F8047B46F8047F032CC2
:10E55000F8D8AEF1040424F0030404342344214425
:10E5600002F0030262B1013B0A4411F8014B03F8C7
:10E57000014F8A42F9D1F0BD0346F3E70346F2E7C3
:10E58000F0BD7246EEE700BF70B4840746D0541E5B
:10E59000002A41D0CDB2034602E0621EE4B3144625
:10E5A00003F8015B9A07F8D1032C2ED9CDB245EAC6
:10E5B00005250F2C45EA054519D903F11002264619
:10E5C000103E0F2E42F8105C42F80C5C42F8085CDA
:10E5D00042F8045C02F11002F2D8A4F1100222F019
:10E5E0000F0204F00F041032032C13440DD91E4601
:10E5F0002246043A032A46F8045BFAD8221F22F086
:10E6000003020432134404F003042CB1C9B21C44C5
:10E6100003F8011BA342FBD170BC704714460346AC
:10E62000C2E700BF704700BF704700BF024B0A46F9
:10E630000146186800F002B8B0ACFF1F2DE9F04F9A
:10E64000174683B0002900F0C1800E46814607F1CD
:10E650000B05FFF7E7FF56F804EC162D2EF0030428
:10E66000A6F1080840D810221546AF4241D894427E
:10E6700075DAC94B996808EB04008842416800F0DC
:10E68000D98021F0010303445B68DB077DD51EF0D0
:10E69000010F35D039464846FFF712FC0746E0B176
:10E6A00056F8043C23F001034344A0F108029A42C7
:10E6B00000F04481221F242A00F23181132A00F243
:10E6C00004810346324611681960516859609268A6
:10E6D0009A603146484600F043FF4846FFF7A4FFE2
:10E6E000384603B0BDE8F08F25F00705002D2A4617
:10E6F000BBDA0C230020C9F8003003B0BDE8F08F6E
:10E7000056F8083CC3EB080ADAF8043023F0030C8F
:10E7100004EB0C039342BDDB5746DAF80C1057F8B4
:10E72000080F221F242AC160886000F21781132A73
:10E7300040F212813168CAF808107168CAF80C10EA
:10E740001B2A00F22B8108360AF110023168116091
:10E7500071685160B16891603E461C46D046631BAB
:10E760000F2B1DD8D8F8043003F001032343444491
:10E77000C8F80430636843F0010363604846FFF75C
:10E7800053FF304603B0BDE8F08F21F00301214470
:10E79000914221DBC36882680C46D3609A60DEE751
:10E7A000D8F8042008EB050102F00102154343F0FC
:10E7B00001020B44C8F804504A605A6842F0010252
:10E7C00008315A60484600F0CBFED7E7114603B047
:10E7D000BDE8F04FFFF774BB1EF0010F7FF45AAF96
:10E7E00056F8083CC3EB080ADAF8043023F0030CAF
:10E7F00001EB0C0E96458BDBC36882685746D360ED
:10E800009A6057F8081FDAF80C30CB60221F242AD0
:10E81000996000F29980132A62D93368CAF80830E7
:10E820007368CAF80C301B2A00F2A08008360AF17F
:10E83000100356E021F0030BA34405F110008345BB
:10E8400059DA1EF0010F7FF425AF56F8081CC1EB12
:10E85000080ADAF8041021F0030CE34458453FF7A6
:10E8600057AF5746DAF80C1057F8080F221F242A22
:10E87000C160886000F2B480132A40F2A58031683C
:10E88000CAF808107168CAF80C101B2A00F2AF8091
:10E8900008360AF110023168116071685160B16880
:10E8A00091600AEB0501C5EB0B0242F00102996091
:10E8B0004A60DAF8043003F001031D434846CAF801
:10E8C0000450FFF7B1FE38465CE7336803607368B5
:10E8D00043601B2A27D800F1080306F10802F2E67C
:10E8E0003B4632681A6072685A60B2689A603E4667
:10E8F0007446D04633E708EB0501C5EB0B0B4BF034
:10E90000010299604A6056F8043C03F001031D437C
:10E91000484646F8045CFFF787FE304632E731464A
:10E92000FFF7CEFDD5E6B3688360F368C360242AA1
:10E9300028D000F1100306F11002C4E650F8043CA0
:10E9400023F003031C440AE7314638467446D04698
:10E95000FFF7B6FD3E4602E73A46F7E6314638464F
:10E960001C46D046FFF7ACFD3E46F8E6B368CAF851
:10E970001030F368CAF81430242A1BD010360AF17C
:10E980001803AEE7336903617369436106F1180246
:10E9900000F1180397E600BF20AEFF1FB168CAF868
:10E9A0001010F168CAF81410242A0FD010360AF19A
:10E9B0001802CBE63369CAF818307369CAF81C30FC
:10E9C00018360AF120038CE73A4664E73269CAF840
:10E9D00018207269CAF81C2018360AF12002B5E620
:10E9E000314638460193FFF76BFD019B59E7B1684B
:10E9F000CAF81010F168CAF81410242A03D010368F
:10EA00000AF1180247E73269CAF818207269CAF891
:10EA10001C2018360AF120023DE700BF38B5074C2C
:10EA20000023054608462360FBF70EFF431C00D079
:10EA300038BD2368002BFBD02B6038BD90E1FF1F51
:10EA4000F8B507460E4617F8014BFFF71FFA2044AA
:10EA50002546437803F00303012B08BF04F120058A
:10EA600016F8014BFFF712FA2044437803F0030332
:10EA7000012B04D0281B01D1002CE4D1F8BD203497
:10EA8000281BE0D0F8BD00BF70B411F0FF0434D0F3
:10EA900085070FD00378002B5AD09C422BD0431C03
:10EAA00005E013F8012B002A4FD0944223D09A0797
:10EAB0001846F6D10E0206F47F462643036846EA5E
:10EAC000064601E050F8043F86EA0305A5F101324D
:10EAD000A3F1013122EA050221EA0303134313F0F3
:10EAE000803FEFD0037823B932E010F8013F002BCC
:10EAF0002ED09C42F9D170BC704784070BD00378AC
:10EB0000002BF8D0431C03E002780133002AF2D036
:10EB100099071846F8D10268A2F1013323EA0203EB
:10EB200013F0803F08D150F8042FA2F1013323EAFB
:10EB3000020313F0803FF6D00378002BDBD010F8EF
:10EB4000013F002BFBD170BC7047104670BC704772
:10EB5000184670BC704700BFFFFFFFFFFFFFFFFFBD
:10EB6000A2EB0300704700BF02780B78012A28BF90
:10EB70009A42F5D16DE9044540EA0104CDE9026706
:10EB80006FF0000C4FEA447212B380EA010414F0F3
:10EB9000070F6AD100F0070420F0070004F0030516
:10EBA00021F007014FEAC505F0E8042314F0040F33
:10EBB000F1E804670CFA05F462EA040266EA040666
:10EBC0000AD063EA0403624667EA0407664603E084
:10EBD000F0E80423F1E8046782FA4CF582EA0604BF
:10EBE000A4FA8CF46CBB83FA4CF583EA0705A5FA0A
:10EBF0008CF595B950E9022351E9026782FA4CF588
:10EC000082EA0604A4FA8CF483FA4CF583EA070539
:10EC1000A5FA8CF52543DBD09CB92DBAB5FA85F45D
:10EC200024F0070427FA04F1DDE9026723FA04F36C
:10EC300003F0FF0001F0FF01FDE80445A0EB010037
:10EC4000704724BAB4FA84F424F0070426FA04F1D5
:10EC5000DDE9026722FA04F202F0FF0001F0FF0191
:10EC6000FDE80445A0EB0100704714F0030F3CD110
:10EC700010F0030428D150F8082B51F8083B82FA11
:10EC80004CF582EA0305A5FA8CF55DB950F8042C21
:10EC900051F8043C82FA4CF582EA0305A5FA8CF59A
:10ECA000002DE8D02DBAB5FA85F424F0070423FA34
:10ECB00004F122FA04F202F0FF0001F0FF01FDE886
:10ECC0000445A0EB010070474FEAC40420F00300A4
:10ECD00050F8082B21F0030151F8083B0CFA04F41A
:10ECE00062EA040263EA0403C9E710F003041AD0DD
:10ECF000A1EB040120F00300E40750F8042B06D038
:10ED00000FD28B785FFAA2F4E41A06D12BB1CB783C
:10ED10005FFAB2F4E41A00D11BB920465DF8104B3B
:10ED2000704701F1040150F8042BCC0721F00301D6
:10ED300051F8043B48D824D222F07F4482FA4CF5A3
:10ED400094EA1325A5FA8CF50AD165B951F8043B6C
:10ED500084EA0204B4EB036F0ED150F8042BEBE706
:10ED60004FEA132355E035F07F454DD10878FDE893
:10ED70000445C0F1000070474FEA126203F0FF0340
:10ED800047E002EA1C4482FA4CF594EA1345A5FADE
:10ED90008CF50AD165B951F8043B84EA0204B4EB5E
:10EDA000034F0CD150F8042BEBE74FEA134330E04C
:10EDB00015EA1C4528D10B884FEA124229E04FEA98
:10EDC000124203EA1C4324E002F0FF0482FA4CF5ED
:10EDD00094EA1365A5FA8CF50AD165B951F8043B9C
:10EDE00084EA0204B4EB032F09D150F8042BEBE7BB
:10EDF0004FEA13630DE015F0FF0F05D10B684FEAE2
:10EE0000122223F07F4304E04FF00000FDE80445A8
:10EE1000704712BA1BBA82FA4CF482EA0304A4FACD
:10EE20008CF5B5FA85F402FA04F203FA04F34FEA1A
:10EE30001260FDE80445A0EB1360704780EA010210
:10EE4000844612F0030F4FD111F0030F32D14DF869
:10EE5000044D11F0040F51F8043B0BD0A3F1013223
:10EE60009A4312F0803F04BF4CF8043B51F8043B36
:10EE700016D100BF51F8044BA3F101329A4312F0AE
:10EE8000803FA4F101320BD14CF8043BA24312F0B5
:10EE9000803F04BF51F8043B4CF8044BEAD02346B2
:10EEA0000CF8013B13F0FF0F4FEA3323F8D15DF864
:10EEB000044B704711F0010F06D011F8012B0CF82C
:10EEC000012B002A08BF704711F0020FBFD031F8A4
:10EED000022B12F0FF0F16BF2CF8022B8CF800202B
:10EEE00012F47F4FB3D1704711F8012B0CF8012BAE
:10EEF000002AF9D1704700BFFFFFFFFFFFFFFFFFB0
:10EF000090F800F06DE9024520F007016FF0000C69
:10EF100010F0070491F820F040F049804FF0000411
:10EF20006FF00700D1E9002391F840F000F10800EC
:10EF300082FA4CF2A4FA8CF283FA4CF3A2FA8CF324
:10EF40004BBBD1E9022382FA4CF200F10800A4FA8B
:10EF50008CF283FA4CF3A2FA8CF3E3B9D1E90423DF
:10EF600082FA4CF200F10800A4FA8CF283FA4CF316
:10EF7000A2FA8CF37BB9D1E9062301F1200182FAD0
:10EF80004CF200F10800A4FA8CF283FA4CF3A2FAD6
:10EF90008CF3002BC6D0002A04BF04301A4612BAE4
:10EFA000B2FA82F2FDE8024500EBD2007047D1E9E7
:10EFB000002304F00305C4F100004FEAC50514F076
:10EFC000040F91F840F00CFA05F562EA05021CBF47
:10EFD00063EA050362464FF00004A9E740EA010333
:10EFE0009B0770B42BD1032A29D90C46034621462E
:10EFF00054F8046BA6F1013525EA060515F0803FAB
:10F0000006D1043A032A43F8046B2146EFD8A2B193
:10F010000C781C70013A013301313CB16AB111F82E
:10F02000014B03F8014B013A002CF7D12AB11A44E5
:10F03000002103F8011B9A42FBD170BC70470346C4
:10F04000E5E700BF2DE9F84FDDF828900F46804630
:10F0500016461D468B4600E0A3465C46484614F81B
:10F0600001ABFEF70FFF5044417801F0080101F0B9
:10F07000FF0C0029F0D152462D2A61D02B2A04BF63
:10F080009BF801200BF10204002D43D0102D65D018
:10F09000A946BCF1000F0CBF6FF0004A4FF0004AC8
:10F0A0000021BAFBF9FE084609FB1EAA05E029D09B
:10F0B00009FB0030012114F8012BA2F13003092BC8
:10F0C00005D9A2F14103192B0AD8A2F137039D42B9
:10F0D0000EDD4A1CEFD08645E9D24FF0FF31EAE75A
:10F0E000A2F16103192B03D8A2F157039D42F0DC72
:10F0F0004B1C15D0BCF1000F10D14EB1E1B93760F7
:10F10000BDE8F88F9A45D3DA70464FF0FF31D2E769
:10F11000BDE8F88F302A1AD00A25B9E74042ECE75B
:10F12000BCF1000F4FF022030CBF6FF000404FF016
:10F130000040C8F80030F6B1671E3760BDE8F88FB0
:10F140000BF102049BF801204FF0010C9CE723789F
:10F1500003F0DF03582B08D0082599E7302A97D110
:10F16000237803F0DF03582B92D14FF01009627817
:10F170004D4602348DE7BDE8F88F00BF30B5084C2E
:10F18000084B25686C6B83B0002C08BF1C460094AC
:10F1900013460A4601462846FFF754FF03B030BD28
:10F1A000B0ACFF1FB4ACFF1F2DE9F84FDDF828907D
:10F1B0000E460746154698468B4600E0A3465C4639
:10F1C000484614F801ABFEF75DFE5044407800F06D
:10F1D000080000F0FF0C0028F0D151462D2961D025
:10F1E0002B2904BF9BF801100BF10204B8F1000FAA
:10F1F0000CD0B8F1100F5CD04FF0FF33B3FBF8F335
:10F2000008FB03FA6FEA0A0AC14607E0302961D019
:10F210004FF00A083D4BC1464FF0050A4FF0000E73
:10F22000704606E02FD009FB00204FF0010E14F8C5
:10F23000011BA1F13002092A05D9A1F14102192AC5
:10F240000BD8A1F1370290450FDDBEF1FF3FEED0A4
:10F250009842E7D94FF0FF3EE9E7A1F16102192A90
:10F2600003D8A1F157029045EFDCBEF1FF3F11D06A
:10F27000BCF1000F00D0404255B1BEF1000F0DD1DE
:10F280002E60BDE8F88F5245CDDD4FF0FF3ECEE752
:10F29000BDE8F88F22233B60704645B3661E2E60A2
:10F2A000BDE8F88F0BF102049BF801104FF0010C40
:10F2B0009CE730291DD1237803F0DF03582B1ED1A2
:10F2C0004FF010096178C8464FF00F0A02346FF012
:10F2D0007043A3E7237803F0DF03582BF0D04FF0FF
:10F2E0000808C1464FF0070A6FF0604396E7BDE893
:10F2F000F88F4FF00F0A6FF07043C1468EE7C1469A
:10F300004FF00F0A6FF0704388E700BF9999991981
:10F3100030B5084C084B25686C6B83B0002C08BFD7
:10F320001C46009413460A4601462846FFF73CFF58
:10F3300003B030BDB0ACFF1FB4ACFF1FF0B5DFF8B9
:10F3400078E0164604460F46BEE80F008BB06D46C7
:10F350000FC5BEE80F000FC59EE80300B31E45F8B9
:10F36000040B222B297022D87D1E2846002200E0A3
:10F370001A46B4FBF6F10AAB06FB114423440C46D3
:10F3800013F8283C00F8013F531C0029F0D1F95430
:10F39000BB184AB1197815F8010F29700134111BF7
:10F3A0008C4203F80109F5DB38460BB0F0BD0020B4
:10F3B00038700BB0F0BD00BF3408010021B1FF2A46
:10F3C00004D80A7001207047084670478A230360FA
:10F3D0004FF0FF30704700BF2DE9F047254C2568FE
:10F3E000D5F848410646884692469946C4B36068B7
:10F3F0001F2817DC431C76B104EB80050122C5F8F9
:10F4000088A0D4F8881182401143022EC4F88811D4
:10F41000C5F808911ED00230636044F820800020B7
:10F42000BDE8F087144B03B34FF4C870FEF738FD06
:10F430000446D0B1D5F84831002780E88800C5F8E7
:10F44000484138460123C4F88871C4F88C71002EF5
:10F45000E1D0D1E7D4F88C110A43C4F88C21DAE763
:10F4600005F5A674C5F84841C1E74FF0FF30BDE887
:10F47000F08700BF24080100A1DE0000024B13B199
:10F48000024800F005B87047000000009DF400003D
:10F49000002301461A461846FFF79EBF38B5074DB0
:10F4A000074C2C1BA41005D0013C55F8043D98478F
:10F4B000002CF9D1BDE8384001F07EBA0000000010
:10F4C00000000000F8B5234F0C460646FFF7AAF8E7
:10F4D000BB685D6825F00305291B01F6EF7121F477
:10F4E0007F6121F00F01A1F58054B4F5805F07DB47
:10F4F00000213046FFF792FABB682B44984204D0B3
:10F500003046FFF791F80020F8BD61423046FFF722
:10F5100085FA01300DD0104BBA6819682D1B45F0E3
:10F5200001053046091B55601960FFF77DF8012081
:10F53000F8BD00213046FFF771FABA68831A0F2B25
:10F54000DEDD064C0449246843F00103001B5360D0
:10F550000860D5E720AEFF1F54E1FF1F2CB2FF1F4C
:10F56000002945D02DE9F0410D468046FFF75AF8B5
:10F5700055F8047C6A4927F00103A5F10804E21854
:10F580008E685068B24220F0030062D0FE075060DF
:10F590000BD455F8087CE41B01F1080EA5687545ED
:10F5A0003B446FD0E768EF60BD6015186D68ED07EC
:10F5B00042D543F001026260E350B3F5007F18D2F8
:10F5C000DB085A1C4D6851F83270A76001209B106F
:10F5D00000FA03F301EBC2001D430838E0604D6000
:10F5E00041F83240FC604046BDE8F041FFF71CB8EE
:10F5F00070475A0A042A53D89A0902F139077F0042
:10F6000002F1380501EB870051F8272044490838FA
:10F6100090424DD0516821F003018B4202D2926892
:10F620009042F7D1D068E060A2608460D460404628
:10F63000BDE8F041FEF7F8BF95683A4FBD4203447C
:10F640003FD0D068E86043F0010285606260E3501B
:10F65000B3E7FF07034407D455F8082CA41A134452
:10F66000A068E268C26090602F4A126843F001000F
:10F67000934260608C60B6D32C4B40461968FFF70C
:10F6800021FFB0E711184968C90744D49168D268CE
:10F69000CA60034443F0010091606060E350A2E758
:10F6A000142A17D802F15C077F0002F15B05A9E775
:10F6B000AA104B68012505FA02F213434B6002467B
:10F6C000B1E743F001024C610C61E560A560626046
:10F6D000E35088E7542A06D81A0B02F16F077F001F
:10F6E00002F16E058EE7B2F5AA7F06D8DA0B02F1B9
:10F6F00078077F0002F1770584E740F25450824298
:10F7000006D89A0C02F17D077F0002F17C0579E7AB
:10F71000FE277E2576E743F001026260E35062E750
:10F7200020AEFF1F28AEFF1F28B2FF1F50E1FF1FB2
:10F73000000000000000000075A80000E803D007EA
:10F74000E803DC05D007FFFF596573005371756549
:10F75000616B200020616761696E20696E20000086
:10F76000206D5300537461727420706C6179696EFE
:10F770006720000020696E20465820736C6F74204B
:10F7800000000000202849443A2000002900000021
:10F7900053746F702020706C6179696E672000006F
:10F7A00020696E20456E67696E6520736C6F7420EA
:10F7B00000000000456E67696E6520736F756E64AA
:10F7C000732064697361626C6564202D2066696CC6
:10F7D0006573206D697373696E67000054726163AD
:10F7E0006B206F7665726C617920736F756E6473D0
:10F7F0002070726573656E7400000000547261635E
:10F800006B204F7665726C617920736F756E6473CF
:10F810002064697361626C6564202D206E6F2066C0
:10F82000696C657320666F756E6400003A000000B5
:10F830002D00000048415244574152452056455240
:10F8400053494F4E3A2000004649524D57415245C8
:10F850002056455253494F4E3A200000302E39333E
:10F860002E353000534F554E442046494C452049D3
:10F870004E464F0046696C656E616D652020202004
:10F88000202020202020204D4D3A53533A6D532004
:10F89000202020205072696F726974790000000086
:10F8A000202D2000207C20005452554500000000EF
:10F8B00046414C53450000004E6F00004849474800
:10F8C000000000004C4F570025000000566F6C757B
:10F8D0006D657300456E67696E6520766F6C756D3A
:10F8E000653A20004566666563747320766F6C75B3
:10F8F0006D653A2000000000547261636B204F7602
:10F9000065726C617920766F6C756D653A200000C8
:10F9100053717565616B2053657474696E6773000C
:10F92000204D696E3D000000204D61783D000000D3
:10F9300020456E61626C65643D0000005371756521
:10F94000616B206D696E2073706565643D00000019
:10F950004C6967687420000020466C61736820540D
:10F96000696D653A2000000020426C696E6B204F83
:10F970006E2054696D653A200000000020426C69D9
:10F980006E6B204F66662054696D653A200000005A
:10F99000536F756E642042616E6B20413A20000007
:10F9A000536F756E642042616E6B20423A200000F6
:10F9B00050726573656E7420284175746F2D6C6F7D
:10F9C0006F703A20000000005468726F74746C65A8
:10F9D0002F456E67696E652053657474696E677331
:10F9E000000000004175746F2053746172742045EB
:10F9F0006E67696E652077697468205468726F74E9
:10FA0000746C653A200000004175746F2053746F68
:10FA10007020456E67696E6520416674657220547A
:10FA2000696D652061742049646C653A20000000AE
:10FA3000206D696E75746573000000004E2F4100E3
:10FA40005468726F74746C6520537469636B2049D9
:10FA5000646C652061743A2000000000537469638F
:10FA60006B2043656E746572000000005374696317
:10FA70006B20456E6400000049646C65204465613C
:10FA80006462616E643A2000536572766F2053653C
:10FA90007474696E67730000536572766F205265E7
:10FAA0007665727365643A200000000054696D65E4
:10FAB00020746F207265636F696C3A20000000004B
:10FAC00054696D6520746F2072657475726E3A208A
:10FAD00000000000456E6420706F696E74733A20F8
:10FAE0000000000025207265636F696C6564202842
:10FAF00000000000207553292C20000025206261A1
:10FB00007474657279202800207553290000000064
:10FB1000456E67696E652053746172740000000061
:10FB2000456E67696E652053746F7000456E676936
:10FB30006E6520546F67676C6500000043616E6EF0
:10FB40006F6E200020466972650000004D61636899
:10FB5000696E652047756E200000000020537461B7
:10FB6000727400002053746F7000000020546F679F
:10FB7000676C6500204F6E00204F66660000000035
:10FB800020537461727420626C696E6B696E6700D9
:10FB900020546F67676C6520626C696E6B696E6775
:10FBA0000000000020466C617368000055736572A8
:10FBB00020536F756E64200020506C617900000046
:10FBC0002052657065617400536F756E64204261E8
:10FBD0006E6B2000410000004200000020506C616C
:10FBE000792F53746F70000020506C6179204E653E
:10FBF0007874000020506C61792050726576696FCE
:10FC00007573000020506C61792052616E646F6DD5
:10FC1000000000004368616E6E656C205479706569
:10FC2000730000004368616E6E656C200000000088
:10FC300053776974636820280000000020706F7398
:10FC40006974696F6E7329005661726961626C65CF
:10FC500020496E707574202D200000004E756C6C6C
:10FC600000000000456E67696E652053706565642D
:10FC7000000000004D617374657220566F6C756DE5
:10FC800065000000556E6B6E6F776E00202843682C
:10FC9000616E6E656C2052657665727365642900CD
:10FCA0004368616E6E656C20547269676765727334
:10FCB0000000000020506F7320000000206F6E00D5
:10FCC000206F66660000000020746F67676C652017
:10FCD0006F6E000020746F67676C65206F6666004A
:10FCE00020737461727420626C696E6B696E670058
:10FCF0002073746F7020626C696E6B696E670000B0
:10FD000020666C61736800006368315F66756E63BE
:10FD1000000000006368616E6E656C5F66756E63FF
:10FD2000000000006368325F66756E6300000000CB
:10FD30006368335F66756E63000000006368345F5C
:10FD400066756E63000000006368355F66756E63FC
:10FD5000000000006368315F72657665727365004C
:10FD60006368616E6E656C5F7265766572736564FB
:10FD7000000000006368325F72657665727365002B
:10FD80006368335F72657665727365006368345FBC
:10FD900072657665727365006368355F7265766556
:10FDA000727365006368315F706F73006368616EC2
:10FDB0006E656C5F706F735F636F756E74000000CB
:10FDC0006368325F706F73006368335F706F7300D6
:10FDD0006368345F706F73006368355F706F7300C2
:10FDE0006368616E6E656C5F706F735F7472696774
:10FDF000676572730000000073316D696E0000006A
:10FE000073717565616B5F73657474696E67730098
:10FE100073316D61780000007331656E0000000081
:10FE200073326D696E00000073326D6178000000FE
:10FE30007332656E0000000073336D696E00000060
:10FE400073336D61780000007333656E000000004D
:10FE500073346D696E00000073346D6178000000CA
:10FE60007334656E0000000073356D696E0000002C
:10FE700073356D61780000007335656E0000000019
:10FE800073366D696E00000073366D617800000096
:10FE90007336656E000000006D696E737065656491
:10FEA00000000000656E67696E650000766F6C7516
:10FEB0006D65730065666665637473006F76657261
:10FEC0006C6179006C315F666C61736800000000E2
:10FED0006C696768747300006C315F626C696E6B8B
:10FEE0006F6E00006C315F626C696E6B6F666600EE
:10FEF0006C325F666C617368000000006C325F6298
:10FF00006C696E6B6F6E00006C325F626C696E6B59
:10FF10006F6666006C335F666C617368000000009A
:10FF20006C335F626C696E6B6F6E00006C335F6286
:10FF30006C696E6B6F6666005342415F6C6F6F70E9
:10FF400000000000736F756E6462616E6B000000EC
:10FF50005342425F6C6F6F700000000073657276F1
:10FF60006F5F726576657273650000007365727607
:10FF70006F00000074696D655F7265636F696C0086
:10FF800074696D655F72657475726E0065705F721D
:10FF900065636F696C00000065705F626174746511
:10FFA000727900006175746F73746172740000007F
:10FFB0006175746F73746F700000000063656E7418
:10FFC00065727468726F74746C6500007468726F27
:10FFD00074746C650000000069646C65646561643C
:10FFE00062616E6400000000537461727420456E9B
:10FFF00067696E650000000053687574646F776E02
:020000021000EC
:1000000020456E67696E650053746F70205371757B
:1000100065616B730000000053746172742053714A
:100020007565616B730000004552524F523A20597A
:100030006F75206E65656420746F207570646174DF
:10004000652074686520434F554E545F544F5441AA
:100050004C5F534F554E4446494C4553206E756D89
:1000600062657221000000004572726F723A204E84
:1000700065787420736F756E642062616E6B2066A4
:10008000696C65206E6F7420666F756E6400000089
:100090005354415254205445535420524F555449BF
:1000A0004E45000046696C656E616D65202020201C
:1000B000202020202020204D4D3A53533A6D5300EC
:1000C000454E44205445535420524F5554494E45B3
:1000D00000000000506C6179696E672E2E2E202082
:1000E000000000004E6F7420666F756E64000000A3
:1000F000446F6E6500000000566F6C756D6520439F
:100100006F6E74726F6C20536F757263653A205313
:10011000657269616C000000566F6C756D652043F7
:100120006F6E74726F6C20536F757263653A2052F4
:1001300043000000566F6C756D6520436F6E7472DE
:100140006F6C20536F757263653A204B6E6F62005F
:10015000556E61626C6520746F20616363657373B3
:10016000207468652053442063617264202D2063ED
:100170006865636B20616E64207265626F6F7420C6
:100180006465766963650000496E692066696C651F
:10019000202800002920646F6573206E6F7420652D
:1001A000786973740000000029206E6F74207661F6
:1001B0006C69643A20000000496E692066696C65CC
:1001C00020657869737473202D2053657474696E8B
:1001D0006773204C6F616465643A0000284F6E6C51
:1001E00079207573656420696E205243206D6F64B9
:1001F00065290000446576696365206D6F64653A22
:1002000020524320696E7075740000004465766961
:100210006365206D6F64653A2053657269616C2077
:10022000696E7075740000002F6F70736F756E6467
:100230002E696E6900FFFFFFE80335058306080796
:10024000E803E204DC05D6060807FFFFE803B00474
:10025000780540060807D007747275650000000035
:10026000796573003100000066616C736500000001
:100270006E6F0000300000006E6F206572726F724A
:100280000000000066696C65206E6F7420666F75F3
:100290006E64000066696C65206E6F74206F706517
:1002A0006E00000062756666657220746F6F207361
:1002B0006D616C6C000000007365656B2065727287
:1002C0006F72000073656374696F6E206E6F7420C7
:1002D000666F756E640000006B6579206E6F742028
:1002E000666F756E64000000656E64206F66206640
:1002F000696C6500756E6B6E6F776E206572726FDC
:1003000072000000756E6B6E6F776E206572726F93
:10031000722076616C7565000000010004000B001E
:1003200013001E002C003C004E0063007B00950073
:10033000B100D000F10014013A0163018E01BB014C
:10034000EA011D0251028802C102FC023A037B034A
:10035000BD03020449049304DF042D057D05D00587
:1003600024067C06D50630078E07EE075008B40831
:100370001A098309ED095A0AC90A390BAC0B210C79
:10038000980C100D8B0D080E860E070F890F0D109F
:1003900093101B11A5113112BE124D13DE137014F0
:1003A00004159A153216CB16651701189F183E19B9
:1003B000DF19811A251BCA1B711C181DC21D6C1E5A
:1003C000181FC51F73202321D42186223923ED2332
:1003D000A22458250F26C82681273B28F628B229B3
:1003E0006F2A2D2BEC2BAB2C6B2D2C2EED2EAF2F43
:1003F00072303531F931BD32823348340E35D4355F
:100400009B3662372938F138B939813A493B123C79
:10041000DB3CA43D6D3E363FFF3FC84091415A4210
:100420002343EB43B4447C4545460C47D4479C48A2
:100430006349294AF04AB64B7B4C404D044EC84EA6
:100440008C4F4E501051D251935253531254D0549A
:100450008E554B560757C2577C583659EE59A55AF8
:100460005C5B115CC55C785D2A5EDB5E8A5F39602F
:10047000E66091613C62E5628D633364D9647C65BA
:100480001E66BF665F67FC6798683369CC69646AFB
:10049000F96A8E6B206CB16C406DCD6D596EE26E59
:1004A0006A6FF06F7570F7707871F6717372EE7233
:1004B0006673DD735274C5743675A47511767B76D8
:1004C000E4764A77AE7710787078CE782979837998
:1004D000DA792F7A817AD27A207B6C7BB57BFC7BB0
:1004E000417C847CC47C027D3E7D777DAE7DE27D57
:1004F000147E447E717E9C7EC47EEA7E0E7F2F7FBA
:100500004E7F6A7F847F9B7FB07FC37FD37FE17FF5
:10051000EC7FF47FFB7FFE7FFF7FFFFF000000008A
:1005200000000000597400000000000000000000FE
:10053000FD750000000000000000000009770000C9
:100540000000000000000000DD7F0000000000004F
:10055000000000007D8100003C800440001000008D
:10056000041A0000FF7F0000111000005D840000ED
:100570000C08000000020000000200000B07000051
:1005800040020000000200000D0E000040020000CA
:10059000000200000A020906141715160F000000D9
:1005A0000002000000020000000200000002000043
:1005B0000002000000020000000200000002000033
:1005C00000020000010102020404080810000000FB
:1005D00000000000000000008D9500007D930000E9
:1005E000198F00008D930000719500004195000067
:1005F0000995000034800440400000001211FFFF04
:10060000FF02020000001310FFFFFF0202000000C3
:100610001800000034800440800000001EFFFFFF2F
:10062000FF02000000001DFFFFFFFF0200000000AE
:10063000190000000000000000000000B5A100004B
:1006400079A10000198F000075A1000031A1000000
:100650003DA100005DA10000050E08090D0C060774
:100660000F0400130393050E08090D0C06070F0471
:10067000FFFFC585848687C4FFFF001303931A928A
:1006800017FFFFFF4008FE4340A004404408FE431C
:1006900044A004400018FE4300C004403000FE4364
:1006A000309004403400FE43349004401C18FE4354
:1006B0001CC004401018FE4310C004400818FE433C
:1006C00008C004400C18FE430CC004400C10FE434C
:1006D0000CB004401010FE4310B004401810FE434C
:1006E00018B004401C10FE431CB004401410FE431C
:1006F00014B004400418FE4304C004400010FE433C
:1007000000B004400008FE4300A004400408FE437B
:1007100004A004400C08FE430CA004400808FE435B
:1007200008A004401418FE4314C004401818FE43E7
:1007300018C004400410FE4304B004400810FE43F7
:1007400008B004401400FE43149004404C08FE43DB
:100750004CA004400420FE4304D004402410FE4377
:1007600024B004402010FE4320B004402810FE4373
:1007700028B004402C10FE432CB004400020FE435F
:1007800000D004404808FE4348A004401000FE4347
:10079000109004400D0AFFFF6E616E006F766600D8
:1007A000696E66000000000000000000B5CA00008D
:1007B000ADCA0000A9CA0000A5CA0000A1CA000075
:1007C0009DCA000099CA000095CA000000151915BD
:1007D00000010000E0A7FF1F12000000000200005F
:1007E0000CA8FF1F430000000003000068A8FF1FC3
:1007F0000000000001030904F4A7FF1F000000002F
:100800000203090450A8FF1F0000000003030904AD
:100810006CA8FF1F000000000000000000000000A6
:100820000000000088A8FF1F504F534958000000E7
:100830002E00FFFF303132333435363738396162BC
:10084000636465666768696A6B6C6D6E6F70717200
:10085000737475767778797A000000000020202084
:100860002020202020202828282828202020202060
:100870002020202020202020202020202088101030
:10088000101010101010101010101010100404048C
:10089000040404040404041010101010101041414A
:1008A0004141414101010101010101010101010138
:1008B000010101010101010110101010101042424C
:1008C0004242424202020202020202020202020208
:1008D00002020202020202021010101020000000A8
:1008E0000000000000000000000000000000000008
:1008F00000000000000000000000000000000000F8
:1009000000000000000000000000000000000000E7
:1009100000000000000000000000000000000000D7
:1009200000000000000000000000000000000000C7
:1009300000000000000000000000000000000000B7
:1009400000000000000000000000000000000000A7
:1009500000000000000000000000000000FFFFFF9A
:10096000F8B500BFF8BC08BC9E4670477DF4000097
:1009700035040000455F0000557500006D750000EE
:100980009D750000B5750000CD750000E57500008F
:10099000F1760000317900004979000061790000AA
:1009A0007979000091790000A9790000C1790000EF
:0809B0001D9B0000419B0000AB
:0409B800F8B500BFCF
:1009BC0038B5084B1C681C6054B1074D94FAA4F36D
:1009CC00B3FA83F355F823309847631E1C40F5D1D6
:1009DC0038BD00BFA0D00440C0A7FF1F38B5084BDE
:1009EC001C681C6054B1074D94FAA4F3B3FA83F35A
:1009FC0055F823309847631E1C40F5D138BD00BF15
:100A0C00A0C00440A0A7FF1F38B5084B1C681C6091
:100A1C0054B1074D94FAA4F3B3FA83F355F8233089
:100A2C009847631E1C40F5D138BD00BFA0B00440F0
:100A3C0070A7FF1F38B5084B1C681C6054B1074DDC
:100A4C0094FAA4F3B3FA83F355F823309847631E52
:100A5C001C40F5D138BD00BFA0A0044020A7FF1F4B
:100A6C0038B5084B1C681C6054B1074D94FAA4F3BC
:100A7C00B3FA83F355F823309847631E1C40F5D125
:100A8C0038BD00BFA0900440E8A6FF1F0000000086
:100A9C0075736572312E77617600000000000000DE
:100AAC00000000000400000075736572322E77613F
:100ABC0076000000000000000000000004000000B0
:100ACC0075736572332E77617600000000000000AC
:100ADC00000000000400000075736572342E77610D
:100AEC007600000000000000000000000400000080
:100AFC0075736572352E776176000000000000007A
:100B0C00000000000400000075736572362E7761DA
:100B1C00760000000000000000000000040000004F
:100B2C0075736572372E7761760000000000000047
:100B3C00000000000400000075736572382E7761A8
:100B4C00760000000000000000000000040000001F
:100B5C0075736572392E7761760000000000000015
:100B6C0000000000040000007573657231302E77B0
:100B7C00617600000000000000000000040000008E
:100B8C007573657231312E776176000000000000BC
:100B9C0000000000040000007573657231322E777E
:100BAC00617600000000000000000000040000005E
:100BBC007573657231332E7761760000000000008A
:100BCC0000000000040000007573657231342E774C
:100BDC00617600000000000000000000040000002E
:100BEC007573657231352E77617600000000000058
:100BFC0000000000040000007573657231362E771A
:100C0C0061760000000000000000000004000000FD
:100C1C007573657231372E77617600000000000025
:100C2C0000000000040000007573657231382E77E7
:100C3C0061760000000000000000000004000000CD
:100C4C007573657231392E776176000000000000F3
:100C5C0000000000040000007573657232302E77BE
:100C6C00617600000000000000000000040000009D
:100C7C0002010100656E7374617274322E776176B5
:100C8C000000000000000000010000000000FF0058
:100C9C00D0070000656E6163636C312E776176005E
:100CAC00000000000000000001000000656E6163A0
:100CBC00636C322E776176000000000000000000AB
:100CCC0001000000656E6163636C332E7761760002
:100CDC00000000000000000001000000656E616370
:100CEC00636C342E77617600000000000000000079
:100CFC0001000000656E6163636C352E77617600D0
:100D0C0000000000000000000100000002000000D4
:100D1C00656E72756E312E776176000000000000F2
:100D2C000000000001000000656E72756E322E77B7
:100D3C0061760000000000000000000001000000CF
:100D4C00656E72756E332E776176000000000000C0
:100D5C000000000001000000656E72756E342E7785
:100D6C00617600000000000000000000010000009F
:100D7C00656E72756E352E7761760000000000008E
:100D8C000000000001000000656E72756E362E7753
:100D9C00617600000000000000000000010000006F
:100DAC00656E72756E372E7761760000000000005C
:100DBC000000000001000000656E72756E382E7721
:100DCC00617600000000000000000000010000003F
:100DDC00656E72756E392E7761760000000000002A
:100DEC000000000001000000656E72756E31302E3F
:100DFC007761760000000000000000000100000098
:100E0C00656E73746F702E776176000000000000C1
:100E1C000000000001000000FFFF640164050C02EB
:100E2C000F000000280201000000FF00656E6964DD
:100E3C006C65312E77617600000000000000000028
:100E4C0001000000656E69646C65322E7761760076
:100E5C00000000000000000001000000656E6964E5
:100E6C006C65332E776176000000000000000000F6
:100E7C0001000000656E69646C65342E7761760044
:100E8C00000000000000000001000000656E6964B5
:100E9C006C65352E776176000000000000000000C4
:100EAC00010000000F190000656E6465636C312E43
:100EBC0077617600000000000000000001000000D7
:100ECC00656E6465636C322E7761760000000000FD
:100EDC000000000001000000656E6465636C332E39
:100EEC0077617600000000000000000001000000A7
:100EFC00656E6465636C342E7761760000000000CB
:100F0C000000000001000000656E6465636C352E06
:100F1C007761760000000000000000000100000076
:100F2C0074725F73746172742E77617600000000C6
:100F3C0000000000010000007475727265742E7759
:100F4C0061760000000000000000000001000000BD
:100F5C0074725F73746F702E7761760000000000FE
:100F6C00000000000100000074725F737472746DF5
:100F7C002E776176000000000000000001000000E8
:100F8C007475727265745F6D2E7761760000000067
:100F9C00000000000100000074725F73746F706DCC
:100FAC002E776176000000000000000001000000B8
:100FBC0062725F73746172742E7761760000000048
:100FCC00000000000100000062617272656C2E77F7
:100FDC00617600000000000000000000010000002D
:100FEC0062725F73746F702E776176000000000080
:100FFC0000000000010000006D675F737461727483
:10100C002E77617600000000000000000300000055
:10101C006D672E7761760000000000000000000074
:10102C0000000000030000006D675F73746F702E8A
:10103C007761760000000000000000000300000053
:10104C006D673273746172742E77617600000000E4
:10105C0000000000030000006D67322E77617600FF
:10106C000000000000000000000000000300000071
:10107C006D673273746F702E77617600000000001C
:10108C0000000000030000006D673373746172741C
:10109C002E776176000000000000000003000000C5
:1010AC006D67332E776176000000000000000000B1
:1010BC0000000000030000006D673373746F702E26
:1010CC0077617600000000000000000003000000C3
:1010DC0063616E6E6F6E662E7761760000000000A5
:1010EC00000000000100000063616E6E6F6E6632DE
:1010FC002E77617600000000000000000100000067
:10110C0063616E6E6F6E66332E7761760000000041
:10111C00000000000100000063616E6E6F6E682EAF
:10112C007761760000000000000000000100000064
:10113C006D676869742E776176000000000000000E
:10114C00000000000100000064657374726F792E5A
:10115C007761760000000000000000000100000034
:10116C006C69676874312E776176000000000000AE
:10117C0000000000010000006C69676874322E7773
:10118C00617600000000000000000000010000007B
:10119C006C69676874332E7761760000000000007C
:1011AC0000000000010000007265706169722E770A
:1011BC00617600000000000000000000010000004B
:1011CC00626565702E7761760000000000000000FB
:1011DC0000000000090000006272616B652E7761EF
:1011EC00760000000000000000000000010000007C
:1011FC007478656E676167652E7761760000000014
:10120C000000000001000000747864656761676588
:10121C002E77617600000000000000000100000045
:10122C0073717565616B312E77617600000000007B
:10123C00000000000100000073717565616B322EB7
:10124C007761760000000000000000000100000043
:10125C0073717565616B332E776176000000000049
:10126C00000000000100000073717565616B342E85
:10127C007761760000000000000000000100000013
:10128C0073717565616B352E776176000000000017
:10129C00000000000100000073717565616B362E53
:1012AC0077617600000000000000000001000000E3
:1012BC000400000074726B73746F702E776176008B
:1012CC0000000000000000000200000072656C6F5E
:1012DC0061645F312E776176000000000000000031
:1012EC000100000072656C6F61645F322E7761766D
:1012FC0000000000000000000100000072656C6F2F
:10130C0061645F332E7761760000000000000000FE
:10131C000100000072656C6F61645F342E7761763A
:10132C0000000000000000000100000072656C6FFE
:10133C0061645F352E7761760000000000000000CC
:10134C000100000074726B73746172742E77617695
:10135C000000000000000000020000000D00000072
:10136C00615F62616E6B312E776176000000000068
:10137C000000000004000000615F62616E6B322EA1
:10138C0077617600000000000000000004000000FF
:10139C00615F62616E6B332E776176000000000036
:1013AC000000000004000000615F62616E6B342E6F
:1013BC0077617600000000000000000004000000CF
:1013CC00615F62616E6B352E776176000000000004
:1013DC000000000004000000615F62616E6B362E3D
:1013EC00776176000000000000000000040000009F
:1013FC00615F62616E6B372E7761760000000000D2
:10140C000000000004000000615F62616E6B382E0A
:10141C00776176000000000000000000040000006E
:10142C00615F62616E6B392E77617600000000009F
:10143C000000000004000000615F62616E6B3130DF
:10144C002E77617600000000000000000400000010
:10145C00615F62616E6B31312E7761760000000046
:10146C000000000004000000615F62616E6B3132AD
:10147C002E776176000000000000000004000000E0
:10148C00615F62616E6B31332E7761760000000014
:10149C000000000004000000615F62616E6B31347B
:1014AC002E776176000000000000000004000000B0
:1014BC00615F62616E6B31352E77617600000000E2
:1014CC000000000004000000615F62616E6B313649
:1014DC002E77617600000000000000000400000080
:1014EC00615F62616E6B31372E77617600000000B0
:1014FC000000000004000000615F62616E6B313817
:10150C002E7761760000000000000000040000004F
:10151C00615F62616E6B31392E776176000000007D
:10152C000000000004000000615F62616E6B3230ED
:10153C002E7761760000000000000000040000001F
:10154C00625F62616E6B312E776176000000000085
:10155C000000000004000000625F62616E6B322EBE
:10156C00776176000000000000000000040000001D
:10157C00625F62616E6B332E776176000000000053
:10158C000000000004000000625F62616E6B342E8C
:10159C0077617600000000000000000004000000ED
:1015AC00625F62616E6B352E776176000000000021
:1015BC000000000004000000625F62616E6B362E5A
:1015CC0077617600000000000000000004000000BD
:1015DC00625F62616E6B372E7761760000000000EF
:1015EC000000000004000000625F62616E6B382E28
:1015FC00776176000000000000000000040000008D
:10160C00625F62616E6B392E7761760000000000BC
:10161C000000000004000000625F62616E6B3130FC
:10162C002E7761760000000000000000040000002E
:10163C00625F62616E6B31312E7761760000000063
:10164C000000000004000000625F62616E6B3132CA
:10165C002E776176000000000000000004000000FE
:10166C00625F62616E6B31332E7761760000000031
:10167C000000000004000000625F62616E6B313498
:10168C002E776176000000000000000004000000CE
:10169C00625F62616E6B31352E77617600000000FF
:1016AC000000000004000000625F62616E6B313666
:1016BC002E7761760000000000000000040000009E
:1016CC00625F62616E6B31372E77617600000000CD
:1016DC000000000004000000625F62616E6B313834
:1016EC002E7761760000000000000000040000006E
:1016FC00625F62616E6B31392E776176000000009B
:10170C000000000004000000625F62616E6B32300A
:10171C002E7761760000000000000000040000003D
:10172C00656E7374617274312E77617600000000FF
:10173C0000000000010000000A000000656E6964F2
:10174C006C655F642E77617600000000000000007D
:10175C00010000000000803F0000803F0000803F3F
:10176C000000000001010000E803000074726163D6
:10177C006B73312E776176000000000000000000D2
:10178C0001000000747261636B73322E7761760016
:10179C000000000000000000010000007472616392
:1017AC006B73332E776176000000000000000000A0
:1017BC0001000000747261636B73342E77617600E4
:1017CC000000000000000000010000007472616362
:1017DC006B73352E7761760000000000000000006E
:1017EC0001000000747261636B73362E77617600B2
:1017FC000000000000000000010000007472616332
:10180C006B73372E7761760000000000000000003B
:10181C0001000000747261636B73382E776176007F
:10182C000000000000000000010000007472616301
:10183C006B73392E77617600000000000000000009
:10184C0001000000747261636B7331302E77617626
:10185C00000000000000000001000000020C00006D
:10186C0000C002405805010000000000000000000C
:10187C00000000000000000000000000000000005C
:10188C00000000000000000000000000000000004C
:10189C0000000000000000003C06010000000000F9
:1018AC00E80300000000000000600640F4050100A1
:1018BC00000000000000000000000000000000001C
:1018CC00000000000000000000000000000000000C
:1018DC0000000000000000000000000000000000FC
:1018EC0000000000000000000000000000000000EC
:1018FC0000000000000000000000000000000000DC
:10190C00000000003C06010000000000E80300009D
:10191C0000000000007006401406010000000000EA
:10192C0000000000000000000000000000000000AB
:10193C00000000000000000000000000000000009B
:10194C00000000000000000000000000000000008B
:10195C00000000000000000000000000000000007B
:10196C00000000000000000000000000000000006B
:10197C000A04000094E1FF1F79A8000079A8000078
:10198C0079A8000079A8000079A8000079A80000C7
:10199C0079A8000079A8000079A8000079A80000B7
:1019AC0079A8000079A8000079A8000079A80000A7
:1019BC0079A8000079A8000079A8000079A8000097
:1019CC0079A8000079A8000079A8000079A8000087
:1019DC0079A8000079A8000079A8000079A8000077
:1019EC0079A8000079A8000079A8000079A8000067
:1019FC0079A8000079A8000079A8000079A8000057
:101A0C0079A8000079A8000079A8000079A8000046
:101A1C0079A8000079A8000079A8000079A8000036
:101A2C0079A8000079A8000079A8000079A8000026
:101A3C0079A8000079A8000079A8000079A8000016
:101A4C0079A8000079A8000079A8000079A8000006
:101A5C0079A8000079A8000001000000FFFFFFFF3B
:101A6C00AC07010000000000E803000000000000CB
:101A7C001201100102000040C0168304750201021D
:101A8C000301000018035400650065006E0073002C
:101A9C0079006400750069006E006F000902430054
:101AAC00020100C0320904000001020201000524F9
:101ABC00001001052401010104240206052406007E
:101ACC00010705820310004009040100020A00000E
:101ADC0000070503024000000705840240000000D7
:101AEC00160355005300420020005300650072009D
:101AFC00690061006C000000040309040C03000081
:101B0C0000000000000000000000000000000000C9
:101B1C0000000000000000000000000074ABFF1F7C
:101B2C00DCABFF1F44ACFF1F0000000000000000F6
:101B3C000000000000000000000000000000000099
:101B4C000000000000000000000000000000000089
:101B5C000000000000000000000000000000000079
:101B6C000000000000000000000000000000000069
:101B7C000000000000000000000000000000000059
:101B8C000000000000000000000000000000000049
:101B9C000000000000000000000000000000000039
:101BAC000000000000000000000000000000000029
:101BBC000000000000000000000000000000000019
:101BCC0001000000000000000E33CDAB34126DE6B6
:101BDC00ECDE05000B00000000000000000000001F
:101BEC0000000000000000000000000000000000E9
:101BFC0000000000000000000000000000000000D9
